:020000040800F2
:1000000008AD012061020008D360000867500008B5
:1000100089600008A90B000889750008000000002D
:10002000000000000000000000000000A101000826
:10003000270D000800000000FD01000865660008AB
:100040007B0200087B0200087B0200087B0200089C
:100050007B0200087B0200087B020008290D0008D3
:100060007B0200087B0200087B0200087B0200087C
:100070007B0200087B0200087B0200087B0200086C
:10008000AD0B0008BD0B00087B0200087B020008D6
:100090007B0200087B0200087B0200087B0200084C
:1000A0007B020008096900087B0200087B02000847
:1000B00019690008296900087B0200087B02000812
:1000C0007B0200087B0200087B0200087B0200081C
:1000D0007B0200083D750008517500086575000831
:1000E0007B0200087B0200087B0200087B020008FC
:1000F000616900087B0200087B0200087B0200089F
:100100007B0200087B0200087B0200087B020008DB
:100110007B0200087B020008396900085169000869
:10012000CD0B0008DD0B0008ED0B00087B0200087A
:100130007B0200087B0200087B0200087B020008AB
:100140007B0200087B0200087B0200087B0200089B
:100150007B020008FD0B00080D0C000875750008F7
:100160007B0200087B0200087B0200087B0200087B
:100170007B0200087B0200087B02000800000000F0
:100180007B0200087B020008DFF810D000F0CCFBF7
:1001900000480047C1C80208AFF3008008AD012045
:1001A0002C4B19680868B0E8F04F80F30988BFF35A
:1001B0006F8F4FF0000080F311887047000000003F
:1001C00008480068006880F308884FF0000080F35A
:1001D000148862B661B6BFF34F8FBFF36F8F00DF35
:1001E00000BF00BF08ED00E0DFF80C00016841F43B
:1001F00070010160704700BF88ED00E0EFF30980F7
:10020000BFF36F8F134B1A681EF0100F08BF20ED5D
:10021000108A20E9F04F106009B44FF0500080F3CD
:100220001188BFF34F8FBFF36F8F43F0FDFB4FF08B
:10023000000080F3118809BC19680868B0E8F04F25
:100240001EF0100F08BFB0EC108A80F30988BFF3CE
:100250006F8F704744C00120EFF3058070470000A6
:100260000648804706480047FEE7FEE7FEE7FEE750
:10027000FEE7FEE7FEE7FEE7FEE7FEE74967000868
:10028000890100082DE9F05F0546002092469B4653
:1002900088460646814640241BE02846414647469C
:1002A000224600F022FA53465A46C01A914110D312
:1002B00011461846224600F009FA2D1A67EB01088C
:1002C0004F4622460120002100F000FA17EB0009FA
:1002D0004E41201EA4F10104DFDC484631462A4687
:1002E0004346BDE8F09F10B5431A934209D28318E4
:1002F000881803E010F8011D03F8011D521EF9D201
:1003000010BD40EA01039B0703D009E008C9121F92
:1003100008C0042AFAD203E011F8013B00F8013BBF
:10032000521EF9D210BDD2B201E000F8012B491ED5
:10033000FBD270470022F6E710B513460A46044682
:100340001946FFF7F0FF204610BD421E12F8013F8C
:10035000002BFBD111F8013B02F8013B002BF9D136
:10036000704710B5044604E00B7800F8013B03B178
:10037000491C521EF8D2204610BD421C10F8011B29
:100380000029FBD1801A704710B5002200E0521CF2
:10039000835C8C5CA34201D1002BF8D1D8B2E1B2CE
:1003A000401A10BD034611F8012B00F8012B002A5A
:1003B000F9D1184670472DE9FE4F804681EA0300C7
:1003C000C00F0C46009021F0004123F00045B8EB2F
:1003D0000200A94105D24046214690461C460B46E4
:1003E000024623F00040104347D0270DC7F30A0010
:1003F000C3F30A510290401A019040286BDAC3F30C
:10040000130040F4801B0098924620B10023D2EBE9
:10041000030A63EB0B0B01985946C0F140025046AA
:1004200000F054F906460D4650465946019A00F030
:100430006CF910EB08006141002487EA115284EA4C
:10044000E7731A4340D0009A62B3019A012A4FEA37
:10045000075215DC001B61EB02014FF0004202EA7B
:100460000752CDE90042001C41F5801132462B466F
:1004700000F06CF903B0BDE8F08F40462146F9E783
:10048000001B61EB0201001C41F5801300185B4169
:100490002018A2F5001747EB030140EAD570B61902
:1004A0006D4111E06D084FEA360645EAC0754FEA26
:1004B0000752001B61EB0201001C41F58011490845
:1004C0004FEA30000019514132462B4603B0BDE8D7
:1004D000F04F00F02CB90098012240000023D0EB2F
:1004E000020263EBE073009821464FEAE074B8EB38
:1004F000000061EB0401E9E783F000435BE781F072
:10050000004158E72DE9FE4F81EA030404F000445E
:1005100021F0004100944FF0000B23F0004350EA1B
:1005200001045ED052EA03045BD0C3F30A54C1F362
:100530000A552C44A4F2F3340194A0FB0254C1F3F5
:10054000130141F48011C3F3130343F4801301FB3F
:10055000024400FB034E840A970A44EA815447EAA6
:100560008357A4FB076802958D0A05FB07854FEAB0
:10057000932C04FB0C542705029D4FEA065847EACA
:100580001637B5EB08056EEB070C870E920E47EA9F
:10059000811742EA8312A7FB0201B6EB0B0164EB61
:1005A00000042B0D43EA0C335E1844EB1C50DA4672
:1005B0005146E7FB0201C5F313044FEA0B3343EA4C
:1005C00014534FEA0432019C43EA0603A4F10C04DD
:1005D0000294009CCDE900B400F0B8F803B0BDE887
:1005E000F08F00200146F9E70EB5C10F80EAE070F8
:1005F0000844CA07002140F233438DE80E000A4642
:100600000B4600F0A3F803B000BD70B5C1F30A5269
:1006100001F000450024C1F3130140F2FF3341F41F
:1006200080119A4201DA002070BD40F233439A42B1
:10063000A2F2334203DC524200F057F800E090404F
:100640002C43F1D0404270BD00F0004230F0004039
:100650000AD0C10D01F56071C0F3160042EA0151E4
:10066000C208400711437047002001467047000050
:1006700030B5041E71F1000404DB4FF00044404229
:1006800064EB0101141E73F1000405DB1C464FF0FE
:100690000043524263EB04038B4208BF824230BDE9
:1006A00030B50B46014600202022012409E021FA42
:1006B00002F59D4205D303FA02F5491B04FA02F53F
:1006C0002844151EA2F10102F1DC30BD202A04DB12
:1006D000203A00FA02F1002070479140C2F1200355
:1006E00020FA03F3194390407047202A04DB203A94
:1006F00021FA02F00021704721FA02F3D040C2F142
:1007000020029140084319467047202A06DBCB1788
:10071000203A41FA02F043EAE07306E041FA02F3BC
:10072000D040C2F12002914008431946704710B5ED
:10073000141E73F1000408DA401C41F10001921804
:100740005B411A4301D120F0010010BD2DE9F04DAD
:1007500092469B4611B1B1FA81F202E0B0FA80F202
:1007600020329046FFF7B2FF04460F4640EA0A00E7
:1007700041EA0B0153465A46084313D0114653EA47
:10078000010019D0C8F140025046FFF7AEFF054600
:100790000E46504659464246FFF798FF084305D09B
:1007A000012004E020463946BDE8F08D00200543D5
:1007B00046EAE0762C4337430A986305E40AA0EB47
:1007C00008000022FD0A44EA47540A3002D50020FE
:1007D0000146E9E7010510196941DDE908450019FD
:1007E0006941BDE8F04DA2E72DE9F04D81EA03042F
:1007F00004F0004B21F0004514464FF0000A23F0AE
:10080000004150EA050220D054EA01021DD0C5F390
:100810000A570246C5F31303C1F31300C1F30A5686
:1008200040F4801543F48013A7EB0608101BD6464E
:1008300008F2FD3873EB050002D308F1010801E06E
:1008400092185B41B8F1000F03DA00200146BDE8C1
:10085000F08D00204FF48011064684460EE0171BF1
:1008600073EB050705D3121B63EB050306434CEA44
:10087000010C49084FEA300092185B4150EA010729
:10088000EDD152EA030012D082EA040083EA0501A6
:10089000084305D0101BAB4106D20122002306E01D
:1008A00000224FF0004302E06FF0010253101AEBF8
:1008B00006004CEB085110EB0A0041EB0B01BDE8C0
:1008C000F04DFFF734BFC1F30A52C1F3130140F2F8
:1008D000FF3341F480119A4202DA0020014670474A
:1008E00040F233439A42A2F2334202DC5242FFF713
:1008F000FCBEFFF7EBBE000030B5041E71F1000432
:1009000004DB4FF00044404264EB0101141E73F11C
:10091000000405DB1C464FF00043524263EB040326
:10092000994208BF904230BD064C074D06E0E06892
:1009300040F0010394E8070098471034AC42F6D326
:10094000FFF726FC74280608B428060870B58C1832
:1009500010F8015B15F0070301D110F8013B2A11D3
:1009600006D110F8012B03E010F8016B01F8016BC0
:100970005B1EF9D12B0705D40023521E0DD401F8BC
:10098000013BFAE710F8013BCB1A921C03E013F885
:10099000015B01F8015B521EF9D5A142D8D30020BA
:1009A00070BD70B50546AC6B206C00F0500050BBBC
:1009B000206C40F4007020642068806800F0405093
:1009C000E8B9207ED8B92068C06A00F4700020B170
:1009D0002068806800F4806088B92068406820F052
:1009E000200021684860206C20F480702064206C16
:1009F00000F4805018B9206C40F0010020642046BB
:100A000000F0ACFA0BE0206C00F0100018B12046AA
:100A100000F0A6FA03E0A06BC16C2846884770BDC1
:100A200070B50546AC6B40202064606C40F004005B
:100A30006064204600F094FA70BD70B50446A56B62
:100A4000284600F08CFA70BD55494A6822F44032BD
:100A50004A604A6843681A434A600268526822F44E
:100A6000807203685A6002685368026943EA02228E
:100A700003685A600268526822F0407203685A6044
:100A80000268526883681A4303685A600268926871
:100A900022F4006203689A6002689268C3681A438D
:100AA00003689A603F4B826A9A4218D00268926843
:100AB00022F0706203689A6002689268836A1A433F
:100AC00003689A600268926822F0405203689A6054
:100AD00002689268C36A1A4303689A600BE002686E
:100AE000926822F0706203689A600268926822F04D
:100AF000405203689A600268926822F0020203681A
:100B00009A6002689368027E43EA420203689A6030
:100B10002022125CA2B10268526842F400620368AB
:100B20005A600268526822F4604203685A600268A0
:100B30005368426A521E43EA423203685A6005E033
:100B40000268526822F4006203685A600268D26A3E
:100B500022F470020368DA620268D36A828B521E42
:100B600043EA02520368DA620268926822F4007271
:100B700003689A600268936890F8302043EA422242
:100B800003689A600268926822F4806203689A603F
:100B900002689368426943EA822203689A60704758
:100BA000002301400100000F00BFFEE710B502481E
:100BB00000F0E0FC10BD0000DCDA012010B50248B6
:100BC00000F0D8FC10BD00007CDA012010B502480E
:100BD00000F0D0FC10BD00000CD4012010B502487C
:100BE00000F0C8FC10BD00009CDB012010B50248DD
:100BF00000F0C0FC10BD00001CDA012010B5024856
:100C000000F0B8FC10BD00003CDB012010B502482C
:100C100000F0B0FC10BD0000BCD9012001460878EE
:100C200010381823B0FBF3F20848805CC865032A2B
:100C300005D908686FF30900001D886503E008689E
:100C40006FF309008865886D7047000060480408EC
:100C5000014600208A6A8B69CBB932B1012A0DD0D6
:100C6000022A03D0032A10D10EE000BFCB6A03F0A2
:100C70008073B3F1807F00D1012007E0CB6AB3F12C
:100C8000C07F00D1012001E000E000BF34E08B69AB
:100C9000B3F5005F1AD132B1012A07D0022A03D07E
:100CA000032A11D10AE000BF01200EE0CB6A03F055
:100CB0008073B3F1807F00D1012006E0CB6AB3F1ED
:100CC000C07F00D1012000E000BF15E032B1012A51
:100CD00005D0022A04D0032A0CD103E000BF00BFD4
:100CE000012008E0CB6A03F08073B3F1807F00D16C
:100CF000012000E000BF00BF704730B504682468E1
:100D000024F4802405682C60046863608468402CA7
:100D100004D10468A2600468E16003E00468A16093
:100D20000468E26030BD704710B5022000F01EFE7E
:100D300010BD72B600BFFEE701460846024B33F80D
:100D4000100002B290B270471C090020014608460C
:100D5000024B33F8100002B290B27047FC0800203A
:100D600030B50246D41702EB5474E410094D2B5DE4
:100D70000246D41702EB5474E410A2EBC40501241C
:100D8000AC401C4014B101220A7001E000220A703C
:100D900030BD000034C0012030B50246D41702EB4C
:100DA0005474E410094D2B5D0246D41702EB5474C1
:100DB000E410A2EBC4050124AC401C4014B1012294
:100DC0000A7001E000220A7030BD000036C0012028
:100DD00038B502460020009000BF92F83C00012880
:100DE00001D1022038BD012082F83C0000BF086814
:100DF000092816D91068C0680C780A3C04EB440531
:100E00000724AC40A0431468E0600C780A3C04EB73
:100E100044048868A0401468E46820431468E060D3
:100E200013E0106800690C7804EB44050724AC401B
:100E3000A043146820610C7804EB44048868A04047
:100E4000146824692043146820614868072817D271
:100E50001068406B0C79641E04EB84051F24AC40C1
:100E6000A04314686063088880B20C79641E04EBA8
:100E70008404A0401468646B20431468606331E00C
:100E800048680D2817D21068006B0C79E41F04EB3A
:100E900084051F24AC40A04314682063088880B2F6
:100EA0000C79E41F04EB8404A0401468246B2043F5
:100EB0001468206316E01068C06A0C790D3C04EBDE
:100EC00084051F24AC40A0431468E062088880B207
:100ED0000C790D3C04EB8404A0401468E46A2043C0
:100EE0001468E062194B1A4C1068A04206D10868D9
:100EF000122803D1586840F480005860144C1068E0
:100F0000A0421CD10868102802D00868112816D108
:100F1000586840F400005860086810280FD10D4848
:100F200000680D4CB0FBF4F000EB80004000009036
:100F300002E00098401E009000980028F9D100BF00
:100F4000002082F83C0000BF00BF4BE700230140B7
:100F50000020014040C0012040420F007047704710
:100F60007047000070B5044600250CB9012070BD23
:100F70001549A06A884200D000BF206C30B92046D5
:100F800000F024F80020606484F83C00206C00F03D
:100F9000100088B9206C20F4885040F002002064D2
:100FA0002046FFF751FD00206064206C20F0020015
:100FB00040F00100206400E0012500BF002084F81B
:100FC0003C0000BF2846D2E70100000F10B586B0F4
:100FD0000446142101A8FFF7ADF92849206888428A
:100FE0004AD100BF002000902548006840F480707E
:100FF000234908600846006800F48070009000BF34
:1010000000BF00BF002000901D481438006840F069
:1010100001001B49143908600846006800F001000F
:10102000009000BF00BF022001900320029000202A
:10103000039001A9134800F0A7FC13481349086066
:1010400000204860002111488160C1604FF4806138
:10105000016149004161890081614911C16100213B
:101060000162416200F0A6FB08B1FFF762FE00BF1B
:101070000648A063846300BF06B010BD0020014095
:101080004438024000000240106402400CD40120A9
:10109000F8B504460D4616460020009000BF94F8AF
:1010A0003C00012801D10220F8BD012084F83C0059
:1010B00000BF2068806800F00100A0B92068806847
:1010C00040F0010021688860554800685549B0FB30
:1010D000F1F000EB4000009002E00098401E00900C
:1010E00000980028F9D12068806800F48070B0F57D
:1010F000807F05D12068806820F480702168886036
:101100002068806800F0010000287ED0206C40F24A
:101110000161884340F4807020642068406800F4D6
:10112000806028B1206C20F4005040F4805020648E
:10113000206C00F48050B0F5805F04D1606C20F02A
:101140000600606401E00020606400BF002084F8B5
:101150003C0000BF344F3548A16BC8633448A16BD5
:1011600008643448A16BC8646FF0220021680860ED
:101170002068406840F0806021684860206880688E
:1011800040F4807021688860226802F14C01334687
:101190002A46A06B00F084FB786800F01F0018BBA3
:1011A00025492068884213D024492068884204D108
:1011B000381D006800F01F0050B1214920688842A6
:1011C0002BD11948001D006800F01F00102824D200
:1011D0002068806800F04050F8B92068806840F0CE
:1011E00080402168886018E013492068884214D143
:1011F0002068806800F0405078B92068806840F02E
:1012000080402168886008E0FFE7206C40F0100013
:101210002064606C40F001006064002044E700003E
:1012200040C0012040420F0000230140A3090008F4
:101230003B0A0008210A000800200140002101406B
:10124000002201407047F0B50346002603B109B9FA
:101250000120F0BD00BF5879012801D10220F8E734
:101260000120587100BF022018711868046802F04C
:10127000100740F6FE70B8408443D1E9000740EA09
:10128000070502F0100005FA00F004431868046036
:101290001868006802F0100CC02707FA0CF7B84372
:1012A0001F6838600120187100BF0020587100BF0E
:1012B0003046CEE7704770B5044620680568206860
:1012C000466B05F40050B0F5005F17D106F40050EE
:1012D000B0F5005F12D104202071206940F00100B8
:1012E00020614FF40050216848632068006820F4B2
:1012F0008050216808602046FFF7DCFF05F00050B1
:10130000B0F1005F17D106F00050B0F1005F12D1CC
:1013100004202071206940F0020020614FF000504D
:10132000216848632068006820F0805021680860C8
:101330002046FFF787FF70BD10B504460CB90120A9
:1013400010BD207920B900206071204600F008F817
:101350000220207100202061012020710020EFE791
:1013600010B586B00446142101A8FEF7E3FF1D491D
:101370002068884233D100BF002000901A480068DE
:1013800040F00050184908600846006800F000501E
:10139000009000BF00BF00BF00200090124810382E
:1013A000006840F0010010491039086008460068E4
:1013B00000F00100009000BF00BF1020019003204A
:1013C00002900020039001A9084800F0DDFA0022F5
:1013D0000521362001F06AF8362001F053F806B0F6
:1013E00010BD000000740040403802400000024080
:1013F00038B50446002000900CB9012038BD2068A3
:10140000009029B902F10800009D2844009004E0F2
:1014100002F11400009D2844009000980360002011
:10142000ECE710B502460AB9012010BD00BF5079A3
:10143000012801D10220F8E70120507100BF0220ED
:1014400010711068006801F010040123A3401843D4
:101450001368186061B91068006800F03C003C280F
:1014600016D11068406840F00100136858600FE022
:101470001068006800F4701301F010043C20A040D4
:10148000834205D11068406840F00200136858603C
:101490000120107100BF0020507100BF00BFC4E7E1
:1014A00070B50446A56D00F077FB064694F835004C
:1014B000022808D08020606500BF002084F8340036
:1014C00000BF012070BD2068006820F01600216870
:1014D00008602068406920F0800021684861206C25
:1014E00008B9A06C28B12068006820F008002168C5
:1014F00008602068006820F001002168086010E0A2
:1015000000F04AFB801B05280BD9202060650320D2
:1015100084F8350000BF002084F8340000BF0320A9
:10152000D0E72068006800F001000028E8D194F8B6
:101530005C103F208840A860012084F8350000BF7F
:10154000002084F8340000BF00BFBBE7014691F8DB
:101550003500022803D0802048650120704705200F
:1015600081F835000868006820F001000A68106002
:101570000020F3E7F8B50446002000908C4800688E
:101580004FF41651B0FBF1F7A56D2E6894F85C107E
:1015900008208840304098B12068006800F00400BE
:1015A00070B12068006820F004002168086094F899
:1015B0005C1008208840A860606D40F00100606504
:1015C00094F85C1001208840304068B12068406980
:1015D00000F0800040B194F85C1001208840A860C1
:1015E000606D40F00200606594F85C100420884053
:1015F000304068B12068006800F0020040B194F803
:101600005C1004208840A860606D40F004006065B4
:1016100094F85C1010208840304078B3206800684F
:1016200000F0080050B394F85C1010208840A860C7
:101630002068006800F4802080B12068006800F411
:10164000002028B9206CC8B12046216C884715E0DD
:10165000A06C98B12046A16C88470FE02068006814
:1016600000F4807028B92068006820F00800216824
:101670000860206C10B12046216C884794F85C10FB
:10168000202088403040002865D02068006800F0A5
:10169000100000285FD094F85C1020208840A860DB
:1016A00094F83500052828D12068006820F016003D
:1016B000216808602068406920F080002168486146
:1016C000206C08B9A06C28B12068006820F00800E0
:1016D0002168086094F85C103F208840A8600120D1
:1016E00084F8350000BF002084F8340000BF206D6E
:1016F00010B12046216D8847F8BD2068006800F4CD
:10170000802080B12068006800F4002028B9606C57
:1017100010B12046616C88471DE0E06BD8B12046CF
:10172000E16B884717E02068006800F4807068B9B2
:101730002068006820F0100021680860012084F80B
:10174000350000BF002084F8340000BFE06B10B10A
:101750002046E16B8847606D38B3606D00F0010092
:10176000F0B1052084F835002068006820F0010001
:101770002168086000BF0098401C0090B84200D962
:1017800005E02068006800F001000028F3D100BFE8
:10179000012084F8350000BF002084F8340000BF29
:1017A000E06C10B12046E16C884700BFA4E7000060
:1017B00040C001202DE9F0410446002500F0ECF97D
:1017C000074614B90120BDE8F081606A00B100BF8E
:1017D000022084F8350000BF002084F8340000BFE8
:1017E0002068006820F00100216808600AE000F02D
:1017F000D3F9C01B052805D920206065032084F893
:101800003500E0E72068006800F001000028EED114
:101810002068056821480540D4E901010843E168D2
:1018200008432169084361690843A1690843E169E4
:101830000843216A08430543606A042803D1D4E9B8
:101840000B0108430543206805602068456925F0C1
:101850000705606A0543606A04280DD1A06A054344
:10186000E06A48B12046FFF7F3F928B140206065EF
:10187000012084F83500A6E7206845612046FFF77F
:10188000CDF9064694F85C103F208840B0600020F7
:101890006065012084F83500002094E73F8010F057
:1018A0002DE9F04704460D4616461F464FF0000846
:1018B000D4F8589000BF94F83400012802D10220D7
:1018C000BDE8F087012084F8340000BF94F83500AB
:1018D000012825D1022084F83500002060653B46B0
:1018E000324629462046FFF708FA94F85C103F205C
:1018F0008840C9F808002068006840F01600216898
:101900000860206C28B12068006840F00800216859
:1019100008602068006840F001002168086006E067
:1019200000BF002084F8340000BF4FF0020840469A
:10193000C6E7000070B5044600F02EF906462546BD
:10194000681C10B104480078054400BF00F024F979
:10195000801BA842FAD370BD00010020022802D1EA
:101960000121014A11707047D900002010B50446CA
:1019700004480068204020B1024804602046FFF778
:10198000EDFF10BD143C0140F8B502460B460025A2
:10199000002400200021D6E0012606FA01F51E6889
:1019A00006EA0504AC4274D11E7906F00306012E46
:1019B00004D01E7906F00306022E13D190684F0062
:1019C0000326BE40B0434F00DE68BE403043906007
:1019D000506801268E40B0431E79C6F300168E4033
:1019E000304350601E7906F00306032E09D0D068FC
:1019F0004F000326BE40B0434F009E68BE403043B8
:101A0000D0601E7906F00306022E13D1CF0802F132
:101A1000200656F827004E07F70E0F26BE40B043AB
:101A20004F07FF0E1E69BE403043CF0802F120066B
:101A300046F8270010684F000326BE40B0431E79C9
:101A400006F003064F00BE40304310605E6806F4A7
:101A50004036002E76D000BF002600963C4E3668F9
:101A600046F480463A4F3E603E46366806F480466D
:101A7000009600BF00BF374E8F0856F827008E072C
:101A8000370F0F26BE40B043334EB24202D100267C
:101A900024E057E0314EB24201D101261EE0304E23
:101AA000B24201D1022619E02E4EB24201D10326E4
:101AB00014E02D4EB24201D104260FE02B4EB2426B
:101AC00001D105260AE02A4EB24201D1062605E0E0
:101AD000284EB24201D1072600E008268F073F0FAB
:101AE000BE4030431B4E8F0846F82700224E306818
:101AF000A0435E6806F4801606B120431E4E306097
:101B0000361D3068A0435E6806F4001606B1204317
:101B1000194E361D3060184E361F3068A0435E687F
:101B200006F4003606B12043134E361F3060361FD0
:101B30003068A0435E6806F4803606B120430E4E3E
:101B4000083E3060491C1029FFF426AFF8BD0000A4
:101B500044380240083801400000024000040240BE
:101B600000080240000C0240001002400014024035
:101B700000180240001C0240083C01400246136964
:101B80000B400BB1012000E0002070470AB18161D9
:101B900001E00B0483617047014800687047000052
:101BA000F800002070B504460CB9012070BD94F80F
:101BB0003D0028B9002084F83C00204600F018FBC6
:101BC000242084F83D002068006820F0010021688E
:101BD00008602068006840F40040216808602068C0
:101BE000006820F400402168086000F09BFD054675
:101BF0005C496068884206D85B48854201D2012072
:101C000007E0002005E05948854201D2012000E0AC
:101C10000020012800D1C9E75548B5FBF0F620683F
:101C2000406820F03F003043216848604D496068BB
:101C3000884201D8701C07E04FF4967070434FF44F
:101C40007A71B0FBF1F0401C2168096A21F03F0174
:101C500008432168086243496068884214D8681EB6
:101C600061684900B0FBF1F0401CC0F30B00042890
:101C700001D204203DE0681E61684900B0FBF1F02C
:101C8000401CC0F30B0034E0A06838B9681E6168DE
:101C900001EB4101B0FBF1F0401C0AE0681E6168F5
:101CA00001EBC10202EB0111B0FBF1F0401C40F46A
:101CB0008040C0F30B0008B901201AE0A06848B9C1
:101CC000681E616801EB4101B0FBF1F0401CC0F3FC
:101CD0000B000CE0681E616801EBC10202EB011110
:101CE000B0FBF1F0401CC0F30B0040F4804040F426
:101CF00000402168C9694CF6FF729143084321688E
:101D0000C861D4E9070108432168096821F0C001CE
:101D1000084321680860D4E90310084321688968F2
:101D200048F2FF329143084321688860D4E90501F5
:101D300008432168C96821F0FF0108432168C86091
:101D40002068006840F001002168086000202064DD
:101D5000202084F83D000020206384F83E0000BF6E
:101D600024E70000A086010080841E0000093D00D9
:101D700040420F002DE9F84304468946174698462D
:101D8000089EFFF709FF054694F83D0020287DD105
:101D900019230122B7492046009503F0B4FA10B187
:101DA0000220BDE8F88300BF94F83C00012801D16F
:101DB0000220F6E7012084F83C0000BF206800689C
:101DC00000F0010028B92068006840F00100216897
:101DD00008602068006820F4006021680860222004
:101DE00084F83D00102084F83E00002020646762E3
:101DF000A4F82A80608D20859F48E0622B463246F9
:101E00004946204603F050F908B10120C9E7208D6A
:101E100088B900BF002000902068406900902068C9
:101E20008069009000BF00BF2068006840F4007027
:101E30002168086047E0208D012817D120680068DC
:101E400020F480602168086000BF002000902068B6
:101E50004069009020688069009000BF00BF206842
:101E6000006840F40070216808602CE0208D022892
:101E700018D12068006820F480602168086020681C
:101E8000006840F400602168086000E0EFE000BFF7
:101E900000200090206840690090206880690090D0
:101EA00000BF10E02068006840F48060216808608E
:101EB00000BF002000902068406900902068806981
:101EC000009000BF00BFC3E0208D03287ED8208D86
:101ED000012815D12A463146204603F0F0FA08B110
:101EE00001205EE720680069616A0870606A401C32
:101EF0006062208D401E2085608D401E6085A7E0B9
:101F0000208D02282AD1334600225C4920460095C4
:101F100003F0F9F908B1012043E72068006840F4B4
:101F200000702168086020680069616A0870606A52
:101F3000401C6062208D401E2085608D401E6085A3
:101F400020680069616A0870606A401C6062208DC8
:101F5000401E2085608D401E608579E0334600225A
:101F600046492046009503F0CEF908B1012018E754
:101F70002068006820F4806021680860206800699B
:101F8000616A0870606A401C6062208D401E208576
:101F9000608D401E608533460022384920460095FA
:101FA00003F0B1F908B10120FBE62068006840F4B5
:101FB00000702168086020680069616A0870606AC2
:101FC000401C6062208D401E208500E010E0608D86
:101FD000401E608520680069616A0870606A401C64
:101FE0006062208D401E2085608D401E60852FE040
:101FF0002A463146204603F062FA08B10120D0E6B5
:1020000020680069616A0870606A401C6062208D07
:10201000401E2085608D401E608520684069C0F3A9
:102020008000A8B1208D032805D12068006820F425
:1020300080602168086020680069616A0870606AD1
:10204000401C6062208D401E2085608D401E608592
:10205000208D00287FF438AF202084F83D00002038
:1020600084F83E0000BF84F83C0000BF99E60220DF
:1020700097E60000020010000000FFFF04000100CE
:102080002DE9F8430446894616461F46DDF82080B0
:10209000FFF782FD054694F83D0020287ED11923E4
:1020A000012251492046009503F02DF910B102207C
:1020B000BDE8F88300BF94F83C00012801D102205C
:1020C000F6E7012084F83C0000BF2068006800F0BB
:1020D000010028B92068006840F00100216808600C
:1020E0002068006820F4006021680860212084F8DE
:1020F0003D00102084F83E00002020646662678561
:10210000608D20853948E0622B464246494620468C
:1021100003F066F808B10120CAE700BF0020009074
:1021200020684069009020688069009000BF00BF6F
:1021300044E02A464146204603F006FA50B1206C9E
:10214000042805D12068006840F400702168086008
:102150000120ADE7606A007821680861606A401C70
:102160006062608D401E6085208D401E2085206845
:102170004069C0F3800070B1208D60B1606A007862
:1021800021680861606A401C6062608D401E608545
:10219000208D401E20852A46414600E022E0204650
:1021A00003F07EF850B1206C042805D12068006847
:1021B00040F4007021680860012079E7208D002834
:1021C000B7D12068006840F40070216808602020C2
:1021D00084F83D00002084F83E0000BF84F83C00F5
:1021E00000BF65E7022063E7020010000000FFFF68
:1021F00010B586B00446142101A8FEF79BF84449A7
:10220000206888422FD100BF00200090414800681C
:1022100040F002003F4908600846006800F00200F4
:10222000009000BF00BFC02001901220029000204B
:102230000390032004900420059001A93648FFF77D
:10224000A3FB00BF0020009032481030006840F42B
:1022500000103049103108600846006800F4001092
:10226000009000BF51E02D49206888424DD100BF49
:10227000002000902748006840F0040025490860CD
:102280000846006800F00400009000BF00BF00BFD7
:10229000002000900846006840F0010008600846F1
:1022A000006800F00100009000BF00BF48150190D9
:1022B0001220029000200390032004900420059037
:1022C00001A91748FFF760FB4FF4807001901220BE
:1022D000029000200390032004900420059001A99F
:1022E0001048FFF751FB00BF002000900948103054
:1022F000006840F400000749103108600846006893
:1023000000F40000009000BF00BF06B010BD000048
:10231000005400403038024000040240005C00409D
:1023200000080240000002400348006803490978A1
:102330000844014908607047F800002000010020AF
:1023400010B50D48006840F400700B49086008465D
:10235000006840F4806008600846006840F48070BF
:102360000860032000F0E0F80F2000F007F800F00C
:102370005FF8002010BD0000003C02402DE9F04154
:1023800088B004460027B84600BF002001902348CB
:10239000006840F02000214908600846006800F00D
:1023A0002000019000BF00BF02A903A800F092F92D
:1023B000069F1FB900F0B6F9054602E000F0B2F939
:1023C00045001748B5FBF0F0A0F101081548164983
:1023D000086040F2E7311448C160C0F80480002171
:1023E00001618160816101F0B7F9064696B90E4836
:1023F00001F0FCFA06466EB9372000F043F8102CC5
:1024000007D200222146372000F050F80748046028
:1024100000E00126304608B0BDE8F08140380240B7
:1024200040420F0000140040FCDB0120FC000020B3
:1024300008B500BF002000901148006840F48040BB
:102440000F4908600846006800F48040009000BF13
:1024500000BF00BF00200090081F006840F08050BF
:10246000091F08600846006800F08050009000BF17
:1024700000BF00220F21901E00F018F808BD0000D8
:10248000443802400146084600280DDB00BF00BF6B
:1024900000F01F0301229A4043099B0003F1E0234F
:1024A000C3F8002100BF00BF00BF70472DE9F05FF7
:1024B00080460D461646002705F0D0F807463946F7
:1024C0002A46334601F00700C0F1070ABAF1040FAB
:1024D00002D94FF0040A01E0C0F1070AD14600F129
:1024E000040ABAF1070F02D24FF0000A01E0A0F18E
:1024F000030AD4464FF0010A0AFA09FAAAF1010ABE
:102500000AEA020A0AFA0CFA4FF0010B0BFA0CFB6A
:10251000ABF1010B0BEA030B4AEA0B0421464046E0
:1025200005F0A4F8BDE8F09F00BF00F00702064BDD
:1025300019684FF6FF031940044B0B4343EA02218D
:10254000014B196000BF70470CED00E00000FA0578
:1025500070B504460D460CB9012070BD584800689E
:1025600000F00700A84209D255490D7008460068DE
:1025700000F00700A84201D00120EEE7207800F02B
:10258000020002281DD1207800F00400042805D1A3
:102590004C48006840F4E0504A490860207800F058
:1025A0000800082805D14748006840F460404549C4
:1025B00008604448006820F0F000A16808434149E1
:1025C0000860207800F00100A8B36068012807D1F6
:1025D0003C4808380068C0F34040B8B90120BCE767
:1025E0006068022802D06068032807D1354808389F
:1025F0000068C0F3406048B90120AEE731480838B0
:102600000068C0F3400008B90120A6E72D48006823
:1026100020F00300616808432A490860FFF7BCFA0C
:10262000064609E0FFF7B8FA801B41F2883188427C
:1026300002D9032091E707E02248006800F00C006F
:102640006168B0EB810FEDD11D48006800F0070014
:10265000A84209D91A490D700846006800F0070021
:10266000A84201D0012078E7207800F00400042877
:1026700007D11448006820F4E050E168084311498C
:102680000860207800F00800082808D10D4800688C
:1026900020F46040216940EAC1000A49086000F066
:1026A00061F808490968C1F30311074A515CC84041
:1026B0000649086006480068FFF760FE00204CE706
:1026C000003C0240083802406848040840C001202D
:1026D000FC0000200F2202600D4A126802F0030283
:1026E00042600B4A126802F0F0028260084A1268E7
:1026F00002F4E052C260064A126802F46042D20854
:102700000261044A126802F007020A607047000082
:1027100008380240003C0240014800687047000051
:1027200040C0012000B5FFF7F7FF04490968C1F375
:102730008221034A515CC84000BD000008380240B5
:102740007848040800B5FFF7E7FF04490968C1F3BA
:102750004231034A515CC84000BD000008380240C5
:10276000784804082DE9F047002400250026A146FA
:102770002548006800F00C0020B1042805D0082886
:102780003AD105E0DFF8849039E0DFF8849036E054
:102790001D48001F006800F03F041B48001F006830
:1027A00000F4800078B11A481749091F0968C1F37D
:1027B0008811A0FB01700146224600233846FDF730
:1027C00061FD05460EE011480F49091F0968C1F374
:1027D0008811A0FB01700146224600233846FDF710
:1027E00051FD05460848001F0068C0F30140401C29
:1027F0004600B5FBF6F902E0DFF8109000BF00BF1D
:102800004846BDE8F0870000083802400024F40084
:1028100000C0A800F8B504460CB90120F8BD207826
:1028200000F00100002874D0F948006800F00C00A6
:1028300004280DD0F648006800F00C00082813D1D9
:10284000F348001F006800F48000B0F5800F0BD142
:10285000EF4808380068C0F34040002859D060684D
:10286000002856D10120D9E700BF6068B0F5803F4D
:1028700008D1E7480838006840F48030E449083956
:1028800008601EE06068B0F5A02F0DD1E048083860
:10289000006840F48020DE49083908600846006876
:1028A00040F4803008600CE0D9480838006820F413
:1028B0008030D749083908600846006820F4802035
:1028C000086000BF606890B1FFF766F9054606E052
:1028D000FFF762F9401B642801D903209EE7CC482A
:1028E00008380068C0F340400028F1D011E0FFF73D
:1028F00053F9054606E0FFF74FF9401B642801D95C
:1029000003208BE7C24808380068C0F34040002825
:10291000F1D1207800F0020002285FD1BC480068A5
:1029200000F00C0058B1BA48006800F00C0008280C
:102930001CD1B748001F006800F48000B0B9B4484B
:1029400008380068C0F3400020B1E068012801D0D9
:10295000012063E7AE480838006820F0F8002169DC
:1029600040EAC100AA490839086037E0E06800B3CE
:102970000120A8490860FFF70FF9054606E0FFF7B8
:102980000BF9401B022801D9032047E7A04808386B
:102990000068C0F340000028F1D09D480838006866
:1029A00020F0F800216940EAC1009949083908601F
:1029B00014E0002097490860FFF7EEF8054606E0AE
:1029C000FFF7EAF8401B022801D9032026E79048C8
:1029D00008380068C0F340000028F1D1207800F0EA
:1029E000080008282CD16069A8B101208A49086034
:1029F000FFF7D2F8054606E0FFF7CEF8401B0228A5
:102A000001D903200AE782486C300068C0F3400017
:102A10000028F1D014E000207F490860FFF7BCF8DF
:102A2000054606E0FFF7B8F8401B022801D903204D
:102A3000F4E677486C300068C0F340000028F1D11C
:102A4000207800F00400042870D100277048383046
:102A5000006800F0805090B900BF002000906C48E2
:102A60003830006840F080506949383108600846C5
:102A7000006800F08050009000BF00BF0127674849
:102A8000006800F48070B0B96448006840F4807059
:102A900062490860FFF780F8054606E0FFF77CF81A
:102AA000401B022801D90320B8E65C48006800F406
:102AB00080700028F2D000BFA068012808D15448D7
:102AC0006830006840F001005149683108601DE03D
:102AD000A06805280DD14E486830006840F0040019
:102AE0004B49683108600846006840F00100086002
:102AF0000CE047486830006820F001004449683124
:102B000008600846006820F00400086000BFA06864
:102B1000A8B1FFF741F8054609E0FFF73DF8401B73
:102B200041F28831884202D9032077E626E038480E
:102B300068300068C0F340000028EED013E0FFF7D3
:102B40002BF8054608E0FFF727F8401B41F28831D3
:102B5000884201D9032061E62D4868300068C0F33F
:102B600040000028EFD1012F07D1294838300068F4
:102B700020F0805026493831086000BFA069002845
:102B800045D02348006800F00C0008285DD0A069FB
:102B9000022845D100201F490866FEF7FDFF0546C3
:102BA00006E0FEF7F9FF401B022801D9032035E6B5
:102BB000174808380068C0F340600028F1D1D4E914
:102BC00007010843616A40EA81110122A06AC2EB51
:102BD000500041EA00412C20005D41EA00600C49B0
:102BE000091F086001200B490866FEF7D5FF05465E
:102BF00006E0FEF7D1FF401B022801D903200DE6B5
:102C0000034808380068C0F340600028F1D049E06C
:102C10000838024000004742800E474200700040E2
:102C2000002021490866FEF7B7FF054606E0FEF7DB
:102C3000B3FF401B022801D90320EFE51B480068C1
:102C4000C0F340600028F2D12CE0A069012800D137
:102C5000E4E51648001D0668A069012820D006F4A6
:102C60008001E06981421BD106F03F01206A814268
:102C700016D147F6C0703040616AB0EB811F0FD1AA
:102C800006F440310122A06AC2EB5000B1EB004FC4
:102C900006D106F070612C20005DB1EB006F01D011
:102CA0000120BBE50020B9E50000474200380240A2
:102CB00010B504460CB9012010BD606A38B96068CF
:102CC000B0F5827F00D105E00021E16102E0002142
:102CD000216161610021A16294F8510028B90020AE
:102CE00084F85000204600F047F8022084F8510094
:102CF0002068006820F0400021680860A08800F487
:102D00008270218901F404410843A18901F4006122
:102D10000843217C01F002010843217D01F00101FB
:102D20000843218B01F400710843217F01F0380131
:102D300008432021095D01F080010843218D01F441
:102D400000510843216808600421A06901EA10408D
:102D500094F8241001F010010843216848602068AD
:102D6000C06920F400602168C8610020606501200E
:102D700084F8510000209FE710B586B00446142166
:102D800001A8FDF7D7FA61492068884230D100BF19
:102D9000002000905E48006840F480505C49086064
:102DA0000846006800F48050009000BF00BF00BFDC
:102DB0000020009056481438006840F00100544943
:102DC000143908600846006800F00100009000BF58
:102DD00000BFE02001900220029000200390032019
:102DE00004900520059001A94A48FEF7CDFD8BE02F
:102DF00049492068884250D100BF002000904448D3
:102E0000001F006840F480404149091F08600846DF
:102E1000006800F48040009000BF00BF00BF0020A9
:102E200000903B481438006840F0040038491439D9
:102E300008600846006800F00400009000BF00BF72
:102E400000BF002000900846006840F002000860C3
:102E50000846006800F00200009000BF00BF0C2090
:102E6000019002200290002003900320049005208E
:102E7000059001A92948FEF787FD4FF40050019005
:102E8000022002900020039003200490052005906A
:102E900001A92348FEF778FD36E0224920688842E0
:102EA00032D100BF002000901948001F006840F494
:102EB00000401749091F08600846006800F40040F8
:102EC000009000BF00BF00BF0020009010481438E1
:102ED000006840F004000E49143908600846006894
:102EE00000F00400009000BF00BF4FF4E0500190DC
:102EF00002200290002003900320049006200590F9
:102F000001A90648FEF740FD06B010BD00300140A3
:102F100044380240000002400038004000080240EF
:102F200000040240003C00402DE9F8430446884676
:102F300016461D4694F85100012802D00220BDE833
:102F4000F8836068B0F5827F0CD1A06850B9042086
:102F500084F851003346424641462046009500F031
:102F600083F9ECE7FEF718FE0746B8F1000F00D032
:102F70000EB90120E3E700BF94F85000012801D109
:102F80000220DCE7012084F8500000BF042084F810
:102F9000510000206065C4F83880A687E68720636A
:102FA000A086E08620646064A068B0F5004F0BD175
:102FB0002068006820F040002168086020680068F0
:102FC00020F48040216808602068006800F040001C
:102FD000402805D02068006840F040002168086063
:102FE000E06830BB21E02068806800F0010050B14B
:102FF0002068007BA16B0870A06B401CA063E08F71
:10300000401EE08711E0FEF7C7FDC01BA84201D3B8
:10301000681C00B94DB9012084F8510000BF0020A0
:1030200084F8500000BF032089E7E08F0028DAD140
:1030300025E021E02068806800F0010050B12068A0
:10304000C068A16B0880A06B801CA063E08F401E4D
:10305000E08711E0FEF7A0FDC01BA84201D3681C69
:1030600000B94DB9012084F8510000BF002084F858
:10307000500000BF032062E7E08F0028DAD13A4613
:103080002946204603F0E0F908B1202060650120C0
:1030900084F8510000BF002084F8500000BF606D2C
:1030A00008B101204BE7002049E72DE9F843044629
:1030B0000F4616461D46FEF76FFD8046B14694F852
:1030C0005100012802D00220BDE8F88307B10EB9F3
:1030D0000120F9E700BF94F85000012801D1022037
:1030E000F2E7012084F8500000BF032084F851006B
:1030F000002060652763A686E686A063A087E08738
:1031000060642064A068B0F5004F0BD120680068AF
:1031100020F04000216808602068006840F480408A
:10312000216808602068006800F04000402805D051
:103130002068006840F0400021680860E068B0F551
:10314000006F37D1606810B1B9F1010F09D1206B60
:1031500000882168C860206B801C2063E08E401EC0
:10316000E08623E02068806800F0020002280AD18F
:10317000206B00882168C860206B801C2063E08E73
:10318000401EE08612E0FEF707FDA0EB0800A84213
:1031900001D3681C00B94DB9012084F8510000BF6B
:1031A000002084F8500000BF03208DE7E08E002847
:1031B000D8D136E0606810B1B9F1010F09D1206BA8
:1031C000007821680873206B401C2063E08E401E4D
:1031D000E08623E02068806800F0020002280AD11F
:1031E000206B007821680873206B401C2063E08E00
:1031F000401EE08612E0FEF7CFFCA0EB0800A842DC
:1032000001D3681C00B94DB9012084F8510000BFFA
:10321000002084F8500000BF032055E7E08E00280E
:10322000D8D142462946204603F058F908B120205B
:103230006065A06850B900BF002000902068C06899
:10324000009020688068009000BF00BF012084F8D3
:10325000510000BF002084F8500000BF606D08B12D
:10326000012031E700202FE72DE9FE4F04460F46ED
:1032700090461D460C9E01200190FEF78DFC814674
:1032800094F851B060680290AA46BBF1010F0BD0D0
:103290000298B0F5827F04D1A06810B9BBF1040F89
:1032A00002D00220BDE8FE8F1FB1B8F1000F00D0A0
:1032B0000DB90120F6E700BF94F85000012801D1B4
:1032C0000220EFE7012084F8500000BF94F851007D
:1032D000042802D0052084F8510000206065C4F85D
:1032E0003880E587A5872763E586A5862064606426
:1032F0002068006800F04000402805D02068006881
:1033000040F0400021680860E068B0F5006F52D1DD
:10331000606810B1BAF1010F09D1206B00882168F3
:10332000C860206B801C2063E08E401EE0863BE07E
:103330002068806800F00200022810D1E08E70B191
:10334000019801280BD1206B00882168C860206B90
:10335000801C2063E08E401EE086002001902068E3
:10336000806800F0010068B1E08F58B12068C06843
:10337000A16B0880A06B801CA063E08F401EE087DB
:1033800001200190FEF708FCA0EB0900B0420BD32E
:10339000701C48B1012084F8510000BF002084F85F
:1033A000500000BF03207DE7E08E0028C0D1E08FF1
:1033B0000028BDD152E0606810B1BAF1010F09D107
:1033C000206B007821680873206B401C2063E08E1E
:1033D000401EE0863CE02068806800F00200022881
:1033E00010D1E08E70B1019801280BD1206B0078CC
:1033F00021680873206B401C2063E08E401EE0862D
:10340000002001902068806800F0010068B1E08F22
:1034100058B12068C068A16B0870A06B401CA06305
:10342000E08F401EE08701200190FEF7B5FBA0EB86
:103430000900B04201D3701C00B94EB9012084F8D4
:10344000510000BF002084F8500000BF032029E78E
:10345000E08E0028BFD1E08F0028BCD14A4631461B
:10346000204603F03BF840B12020606500BF0020FB
:1034700084F8500000BF012014E7A06850B900BFD5
:10348000002000902068C06800902068806800904C
:1034900000BF00BF012084F8510000BF002084F865
:1034A000500000BF606D08B10120FBE60020F9E686
:1034B0007047704710B50346002200BF93F83C00E8
:1034C000012801D1022010BD012083F83C0000BF7B
:1034D00022F0FF00CC6840EA040222F440708C68BD
:1034E00040EA040222F480604C6840EA040222F4BC
:1034F00000600C6840EA040222F480500C6940EA43
:10350000040222F400504C6940EA040222F4804094
:10351000CC6940EA04021868426400BF002083F8C6
:103520003C0000BF00BFCEE730B502460B4600BFEF
:1035300092F83C00012801D1022030BD012082F820
:103540003C0000BF022082F83D001068446810680B
:10355000816824F070041868044310684460184DB2
:103560001068A8421BD01068B0F1804F17D0154DDD
:103570001068A84213D0144D1068A8420FD0134D04
:103580001068A8420BD0124D1068A84207D0114D08
:103590001068A84203D0104D1068A84205D121F050
:1035A00080015868014310688160012082F83D0065
:1035B00000BF002082F83C0000BF00BFBDE7000054
:1035C000000001400004004000080040000C0040E2
:1035D00000040140004001400018004070B504465E
:1035E0000D4615B994F842000BE0042D02D143209A
:1035F000005D06E0082D02D14420005D01E0452079
:10360000005D012801D0012070BD1DB9022084F8A1
:1036100042000EE0042D03D102214320015508E0B1
:10362000082D03D102214420015502E0022145204A
:10363000015504222946206803F01FFA2068406CD7
:1036400040F40040216848641A49206888421BD031
:103650002068B0F1804F17D017492068884213D0F6
:103660001649206888420FD01549206888420BD03F
:1036700014492068884207D013492068884203D043
:103680001249206888420CD12068806800F0070643
:10369000062E0CD02068006840F001002168086008
:1036A00005E02068006840F0010021680860002003
:1036B000AAE70000000001400004004000080040AC
:1036C000000C004000040140004001400018004090
:1036D00070B504460D4600222946206803F0CDF956
:1036E00000BF2068006A41F21111084050B92068FB
:1036F000006A8910084028B92068406C20F4004016
:103700002168486400BF00BF2068006A41F21111BF
:10371000084050B92068006A8910084028B920681C
:10372000006820F001002168086000BF1DB9012079
:1037300084F842000EE0042D03D1012143200155FD
:1037400008E0082D03D101214420015502E00121A8
:1037500045200155002070BD10B504460CB901206C
:1037600010BD94F83D0028B9002084F83C002046A4
:1037700000F026F8022084F83D00211D206803F0A7
:10378000F7F8012084F8460000BF84F83E000121CC
:103790003F200155402001554120015500BF00BF89
:1037A000012084F842004320015544200155452062
:1037B000015500BF012084F83D000020D0E7000043
:1037C00010B586B00446142101A8FCF7B3FD5A4990
:1037D0002068884218D100BF002000905748006838
:1037E00040F00100554908600846006800F00100FB
:1037F000009000BF00BF002205211920FEF756FEF1
:103800001920FEF73FFE94E02068B0F1804F1AD1F6
:1038100000BF002000904948001F006840F00100F0
:103820004649091F08600846006800F00100009042
:1038300000BF00BF002205211C20FEF737FE1C2020
:10384000FEF720FE75E03E492068884236D100BF71
:10385000002000903948001F006840F002003749FE
:10386000091F08600846006800F00200009000BFD1
:1038700000BF00BF0020009030481438006840F0BE
:1038800002002E49143908600846006800F0020062
:10389000009000BF00BF02200190029003900490AE
:1038A000059001A92748FEF76FF8002205211D2089
:1038B000FEF7FCFD1D20FEF7E5FD3AE022492068F9
:1038C00088421AD100BF002000901C48001F0068E9
:1038D00040F010001949091F08600846006800F010
:1038E0001000009000BF00BF002205213620FEF727
:1038F000DDFD3620FEF7C6FD1BE014492068884236
:1039000017D100BF002000900C48006840F0020072
:103910000A4908600846006800F00200009000BFF5
:1039200000BF002205212C20FEF7C0FD2C20FEF751
:10393000A9FD06B010BD000000000140443802405F
:103940000004004000040240001000400004014058
:10395000014691F83D00012801D001207047022066
:1039600081F83D001A4B086898421BD00868B0F1F6
:10397000804F17D0174B0868984213D0164B086831
:1039800098420FD0154B086898420BD0144B08682A
:10399000984207D0134B0868984203D0124B08682E
:1039A00098420CD10868806800F00702062A0CD003
:1039B0000868006840F001000B68186005E00868BE
:1039C000006840F001000B6818600020C6E70000A6
:1039D000000001400004004000080040000C0040CE
:1039E000000401400040014000180040014691F8E9
:1039F0003D00012801D001207047022081F83D00E0
:103A00000868C06840F001000B68D8601A4B08686D
:103A100098421BD00868B0F1804F17D0174B086848
:103A2000984213D0164B086898420FD0154B08687F
:103A300098420BD0144B0868984207D0134B086883
:103A4000984203D0124B086898420CD108688068ED
:103A500000F00702062A0CD00868006840F0010058
:103A60000B68186005E00868006840F001000B680A
:103A700018600020C0E70000000001400004004082
:103A800000080040000C00400004014000400140DC
:103A900000180040014600BF0868006A41F2111298
:103AA000104050B90868006A9210104028B90868A0
:103AB000006820F001000A68106000BF012081F852
:103AC0003D00002070472DE9F04104460D460027D7
:103AD00000BF94F83C00012802D10220BDE8F0812B
:103AE000012084F83C0000BF022084F83D002068DB
:103AF000866826F0770626F47F4620688660286868
:103B0000502833D00CDC202850D004DC00284BD0C7
:103B1000102851D149E0302849D040284CD139E013
:103B200060282DD0702807D0B0F5805F03D0B0F5A5
:103B3000005F41D10DE041E0D5E902136A682068D9
:103B400002F0ACFF2068866846F077062068866041
:103B500034E0D5E902136A68206802F09FFF20680C
:103B6000806840F480402168886027E0EA686968DE
:103B7000206803F083F85021206802F09AFF1DE0CE
:103B8000EA686968206803F0D5F86021206802F0CF
:103B900090FF13E0EA686968206803F06FF840213D
:103BA000206802F086FF09E000BF00BF00BF29685F
:103BB000206802F07EFF01E0012700BF00BF012066
:103BC00084F83D0000BF002084F83C0000BF384668
:103BD00084E7000010B504460F48A0421BD10F48EF
:103BE0000078012803DB0C210B4800F085F90C213B
:103BF000094800F0D3FC00EE100AB8EE400A07486E
:103C000001780078401C054A107002F1100000EBAA
:103C1000810080ED000A10BD2408002044DC012052
:103C20002DE9F04104460D461646002700BF94F8E2
:103C30003C00012802D10220BDE8F081012084F877
:103C40003C0000BF96B9EB68D5E90012206803F08C
:103C500029F82068806920F00C00216888612068BC
:103C60008069A96808432168886141E0042E13D166
:103C7000EB68D5E90012206803F070F820688069CD
:103C800020F440602168886120688069A96840EA62
:103C90000120216888612BE0082E12D1EB68D5E95C
:103CA0000012206803F077F82068C06920F00C004B
:103CB0002168C8612068C069A96808432168C86193
:103CC00016E00C2E13D1EB68D5E90012206803F042
:103CD0007EF82068C06920F440602168C8612068CF
:103CE000C069A96840EA01202168C86100E0012795
:103CF00000BF002084F83C0000BF38469CE710B5A8
:103D000004460CB9012010BD94F83D0028B90020EC
:103D100084F83C00204600F025F8022084F83D009D
:103D2000211D206802F024FE012084F8460000BF17
:103D300084F83E0001213F200155402001554120DB
:103D4000015500BF00BF012084F842004320015507
:103D5000442001554520015500BF012084F83D0055
:103D60000020D0E7704700002DE9F04304460D46DF
:103D7000002615B994F83E000BE0042D02D13F2037
:103D8000005D06E0082D02D14020005D01E04120E9
:103D9000005D804615B994F842000BE0042D02D175
:103DA0004320005D06E0082D02D14420005D01E0C3
:103DB0004520005D8146B8F1010F02D1B9F1010F34
:103DC00002D00120BDE8F0831DB9022084F83E0036
:103DD0000EE0042D03D102213F20015508E0082DFB
:103DE00003D102214020015502E00221412001556A
:103DF0001DB9022084F842000EE0042D03D10221F7
:103E00004320015508E0082D03D10221442001552B
:103E100002E002214520015535B1042D0BD0082DBB
:103E200010D00C2D1CD114E02068C06840F00200B6
:103E30002168C86016E02068C06840F0040021686E
:103E4000C8600FE02068C06840F008002168C860C2
:103E500008E02068C06840F010002168C86001E0F8
:103E6000012600BF00BF86BB01222946206802F060
:103E7000F3FD1A49206888421BD02068B0F1804FBA
:103E800017D017492068884213D016492068884205
:103E90000FD01549206888420BD014492068884209
:103EA00007D013492068884203D01249206888420D
:103EB0000CD12068806800F00707062F0CD020681E
:103EC000006840F001002168086005E02068006893
:103ED00040F0010021680860304673E700000140AF
:103EE0000004004000080040000C004000040140B5
:103EF000004001400018004070B504460D46002601
:103F000035B1042D0BD0082D10D00C2D1CD114E090
:103F10002068C06820F002002168C86016E02068B0
:103F2000C06820F004002168C8600FE02068C06805
:103F300020F008002168C86008E02068C06820F010
:103F400010002168C86001E0012600BF00BF002EFC
:103F50003FD100222946206802F07EFD00BF206884
:103F6000006A41F21111084050B92068006A8910B6
:103F7000084028B92068006820F001002168086026
:103F800000BF1DB9012084F83E000EE0042D03D1CE
:103F900001213F20015508E0082D03D101214020D7
:103FA000015502E00121412001551DB9012084F88D
:103FB00042000EE0042D03D101214320015508E009
:103FC000082D03D101214420015502E001214520A3
:103FD0000155304670BD70B504462068C56820683C
:103FE000066906F00200022819D105F00200022835
:103FF00015D1401F21680861012020772068806961
:1040000000F0030018B12046FFF7E4FD05E020466C
:1040100000F0F0F8204600F0A4F90020207706F028
:104020000400042819D105F00400042815D1C04368
:1040300021680861022020772068806900F44070C0
:1040400018B12046FFF7C6FD05E0204600F0D2F883
:10405000204600F086F90020207706F008000828A6
:1040600019D105F00800082815D1C043216808615E
:10407000042020772068C06900F0030018B12046B2
:10408000FFF7A8FD05E0204600F0B4F8204600F058
:1040900068F90020207706F01000102819D105F0EB
:1040A0001000102815D1C04321680861082020772E
:1040B0002068C06900F4407018B12046FFF78AFDFF
:1040C00005E0204600F096F8204600F04AF900206E
:1040D000207706F0010048B105F0010030B16FF023
:1040E000010021680861204600F016FA06F0800001
:1040F000802809D105F08000802805D1C0432168BF
:1041000008612046FFF7D4F906F04000402809D1A5
:1041100005F04000402805D1C043216808612046D1
:1041200000F055FA06F02000202809D105F0200003
:10413000202805D1C043216808612046FFF7B9F95E
:1041400070BD000010B586B00446142101A8FCF72C
:10415000F1F82349206888421FD100BF0020009059
:104160002048006840F010001E49086008460068BA
:1041700000F01000009000BF00BF4FF4005001900D
:10418000022002900120039000200490012005905D
:1041900001A91548FDF7F8FB20E014492068884282
:1041A0001CD100BF002000900E48006840F00200C3
:1041B0000C4908600846006800F00200009000BF4B
:1041C00000BF012001900220029000200390049083
:1041D0000320059001A90648FDF7D6FB06B010BDE7
:1041E000000001403038024000100240000401404D
:1041F0000004024070472DE9F04104460D46164682
:10420000002700BF94F83C00012802D10220BDE83D
:10421000F081012084F83C0000BF36B1042E1BD091
:10422000082E31D00C2E5ED145E02946206802F0E0
:1042300049FC2068806940F0080021688861206896
:10424000806920F0040021688861206880692969FC
:1042500008432168886148E02946206802F06AFC2A
:104260002068806940F40060216888612068806966
:1042700020F480602168886120688069296940EAAB
:1042800001202168886130E02946206802F090FC16
:104290002068C06940F008002168C8612068C069D2
:1042A00020F004002168C8612068C06929690843BA
:1042B0002168C86119E02946206802F0B5FC206831
:1042C000C06940F400602168C8612068C06920F4BA
:1042D00080602168C8612068C069296940EA0120BE
:1042E0002168C86101E0012700BF00BF00BF0020B6
:1042F00084F83C0000BF384689E710B504460CB985
:10430000012010BD94F83D0028B9002084F83C003D
:10431000204600F025F8022084F83D00211D206889
:1043200002F026FB012084F8460000BF84F83E001E
:1043300001213F200155402001554120015500BF7A
:1043400000BF012084F8420043200155442001555C
:104350004520015500BF012084F83D000020D0E732
:104360007047704770B504460D4615B994F83E0085
:104370000BE0042D02D13F20005D06E0082D02D1A4
:104380004020005D01E04120005D012801D00120B6
:1043900070BD1DB9022084F83E000EE0042D03D14B
:1043A00002213F20015508E0082D03D102214020C1
:1043B000015502E0022141200155012229462068D1
:1043C00002F04AFB23492068884203D02249206832
:1043D000884201D1012000E0002028B12068406C13
:1043E00040F40040216848641A49206888421BD084
:1043F0002068B0F1804F17D018492068884213D048
:104400001749206888420FD01649206888420BD08F
:1044100011492068884207D013492068884203D098
:104420001249206888420CD12068806800F0070695
:10443000062E0CD02068006840F00100216808605A
:1044400005E02068006840F0010021680860002055
:104450009EE700000000014000040140000400400D
:1044600000080040000C00400040014000180040DF
:1044700030B504460D4600222946206802F0ECFAC9
:1044800023492068884203D022492068884201D10C
:10449000012000E0002090B100BF2068006A41F2D6
:1044A0001111084050B92068006A8910084028B9E5
:1044B0002068406C20F400402168486400BF00BFC1
:1044C0002068006A41F21111084050B92068006A62
:1044D0008910084028B92068006820F00100216890
:1044E000086000BF1DB9012084F83E000EE0042DD5
:1044F00003D101213F20015508E0082D03D10121FE
:104500004020015502E0012141200155002030BD2D
:10451000000001400004014010B50446184920681D
:10452000884201D1FDF700FF16492068884201D179
:104530000FF084FD14492068884201D10FF086FDF8
:1045400012492068884204D111480068401C104973
:1045500008602068B0F1804F0FD10E48007800B994
:1045600010BD0D48FFF796FA3EF054FC00200A49B2
:10457000096848620848FFF7EBF900BFF0E7000060
:1045800000140040000400400010004000040140FE
:104590000000002062C10120DC070020024600204C
:1045A00031B1042907D0082908D00C290CD108E022
:1045B0001368586B09E01368986B06E01368D86BB2
:1045C00003E01368186C00E000BF00BF704770473D
:1045D000704770B50446002520684069C0F3C015D7
:1045E00094F84100212817D1B5B100BF00BF216860
:1045F000143151E8001F21F080002168143141E896
:104600000002002AF3D100BFA06B10B1A06BFCF731
:1046100047FF204602F010FD20684069C0F3801576
:1046200094F84200222817D1B5B100BF00BF21681D
:10463000143151E8001F21F040002168143141E895
:104640000002002AF3D100BFE06B10B1E06BFCF771
:1046500027FF204602F0AAFC002070BD7047000032
:104660002DE9F84F0446206805682068C668206870
:1046700047694FF00009CA4605F00F09B9F1000F6C
:104680000AD105F0200038B106F0200020B1204604
:1046900002F0E5FCBDE8F88FB9F1000F7CD007F01F
:1046A000010018B906F49070002875D005F00100DB
:1046B00030B106F4807018B1606C40F001006064A5
:1046C00005F0040030B107F0010018B1606C40F053
:1046D0000200606405F0020030B107F0010018B17B
:1046E000606C40F00400606405F0080048B106F01A
:1046F000200010B907F0010018B1606C40F008000C
:104700006064606C002846D005F0200028B106F0F7
:10471000200010B1204602F0A2FC20684069C0F3DE
:10472000801A606C00F0080010B9BAF1000F2DD0AB
:10473000204602F03BFC2068406900F04000402821
:1047400020D100BF00BF2168143151E8001F21F0C3
:1047500040002168143141E80002002AF3D100BF73
:10476000E06B50B17748E16B0865E06BFCF7EEFE5B
:1047700088B1E06B016D88470DE02046FFF76EFFC2
:1047800009E009E02046FFF769FF04E02046FFF753
:1047900065FF002060647DE7206B012878D105F07B
:1047A0001000002874D006F010000028FAD000BFD6
:1047B0000020009020680068009020684068009009
:1047C00000BF00BF2068406900F04000402860D171
:1047D000E06B006840681FFA80F8B8F1000F56D00F
:1047E000A08D404553DDA4F82E80E06BC069B0F584
:1047F000807F43D000BF00BF21680C3151E8001F0B
:1048000021F4807021680C3141E80002002AF3D1C4
:1048100000BF00BF00BF2168143151E8001F21F024
:1048200001002168143141E80002002AF3D100BFE1
:1048300000BF00BF2168143151E8001F21F0400083
:104840002168143141E80002002AF3D100BF202082
:1048500084F842000020206300BF00BF21680C31B3
:1048600051E8001F21F0100021680C3141E80002DE
:10487000002AF3D100BFE06BFCF712FE0220606358
:10488000A08DE28D801A81B22046FFF7A1FE01E7DC
:1048900042E0A08DE18D401A1FFA80F8E08DD0B380
:1048A000B8F1000F37D000BF00BF21680C3151E8CC
:1048B000001F21F4907021680C3141E80002002AA9
:1048C000F3D100BF00BF00BF2168143151E8001FC1
:1048D00021F001002168143141E80002002AF3D1DF
:1048E00000BF202084F842000020206300BF00BFEA
:1048F00021680C3151E8001F21F0100021680C31B3
:1049000041E80002002AF3D100BF02206063414663
:104910002046FFF75DFEBDE605F0800030B106F0F1
:10492000800018B1204602F093FDB3E605F0400088
:1049300030B106F0400018B1204602F06DFBA9E648
:1049400000BFA7E60B6E000810B504460CB90120A5
:1049500010BDA06900B100E000BF94F8410028B983
:10496000002084F84000204600F02AF8242084F833
:1049700041002068C06820F400502168C8602046CB
:1049800002F0ECFB2068006920F490402168086187
:104990002068406920F02A00216848612068C068CA
:1049A00040F400502168C86000206064202084F832
:1049B000410084F842000020606300BFC8E70000A7
:1049C00010B586B00446142101A8FBF7B3FCE149F9
:1049D000206888427CD100BF00200090DE4800683B
:1049E00040F01000DC4908600846006800F0100044
:1049F000009000BF00BF00BF00200090D6481438D0
:104A0000006840F00100D449143908600846006885
:104A100000F00100009000BF00BF4FF4C0600190A3
:104A200002200290002003900320049007200590AC
:104A300001A9CA48FCF7A8FFC948CA4908604FF055
:104A4000006048604021C74881600021C1604FF488
:104A500080610161002141618161C1614FF4403198
:104A6000016200214162FCF7A5FE08B1FCF761F983
:104A700000BFBC48A063846300BFB9487838BA4916
:104A800008604FF0006048600021B7488160C16055
:104A90004FF480610161002141618161C1614FF486
:104AA0004031016200214162FCF784FE08B1FCF74D
:104AB00040F900BFAC48E063846300BF00220521D9
:104AC0002520FDF7F3FC2520FDF7DCFC40E1FFE7A6
:104AD000A649206888427DD100BF002000909E48F2
:104AE000001F006840F400309B49091F0860084619
:104AF000006800F40030009000BF00BF00BF00203D
:104B0000009095481438006840F00100924914392B
:104B100008600846006800F00100009000BF00BF78
:104B20000C200190022002900020039003200490AA
:104B30000720059001A98948FCF726FF8C488D497C
:104B400008604FF00060486040218A488160002181
:104B5000C1604FF480610161002141618161C161E7
:104B60004FF44031016200214162FCF723FE08B19D
:104B7000FCF7DFF800BF7F48A063846300BF7C4878
:104B800018387D4908604FF00060486000217A487D
:104B90008160C1604FF480610161002141618161E8
:104BA000C1614FF44031016200214162FCF702FE15
:104BB00008B1FCF7BEF800BF6F48E063846300BF34
:104BC000002205212620FDF771FC2620FDF75AFC66
:104BD000BEE0FFE76949206888423BD100BF002062
:104BE00000905D48001F006840F480205A49091F6A
:104BF00008600846006800F48020009000BF00BFF5
:104C000000BF0020009054481438006840F00200B3
:104C10005149143908600846006800F0020000900D
:104C200000BF00BF4FF440600190022002900020BE
:104C30000390032004900720059001A95048FCF739
:104C4000A3FE002205212720FDF730FC2720FDF7D9
:104C500019FC7DE04B492068884279D100BF0020D3
:104C600000903D48006840F020003B49086008463D
:104C7000006800F02000009000BF00BF00BF0020CF
:104C8000009035481438006840F004003249143967
:104C900008600846006800F00400009000BF00BFF4
:104CA000C020019002200290002003900320049075
:104CB0000820059001A93448FCF766FE28481838FA
:104CC000324908604FF02060486040212F488160E1
:104CD0000021C1604FF48061016100214161816167
:104CE000C1614FF44031016200214162FCF762FD75
:104CF00008B1FCF71EF800BF2448A063846300BF1E
:104D000017489038224908608005486000212048F3
:104D10008160C1604FF48061016100214161816166
:104D2000C1614FF44031016200214162FCF742FD54
:104D300008B1FBF7FEFF00BF1548E063846300BFC6
:104D4000002205214720FDF7B1FB4720FDF79AFB24
:104D500006B010BD0010014044380240000002407F
:104D6000B8640240BCD901201CDA01200044004094
:104D7000A06002407CDA0120DCDA0120004800401B
:104D80000004024000140140000802403CDB012006
:104D90009CDB012070B504460D46164694F842008F
:104DA00020280BD105B10EB9012070BD0020206371
:104DB00032462946204602F0E7FAF6E70220F4E7F9
:104DC000704770472DE9F84F04460E46174699463E
:104DD0004FF0000A94F84100202850D106B117B9CD
:104DE0000120BDE8F88F00206064212084F8410094
:104DF000FCF7D2FE8246A784E784A068B0F5805F06
:104E000004D1206910B90025B04602E035464FF0C4
:104E100000081EE05346002280212046CDF8009075
:104E200002F046FB20B1202084F841000320D8E79F
:104E300045B9B8F80000C0F308002168486008F1DF
:104E4000020803E02878216848606D1CE08C401E51
:104E5000E084E08C0028DDD153460022402120462A
:104E6000CDF8009002F024FB20B1202084F841000E
:104E70000320B6E7202084F841000020B1E702209B
:104E8000AFE70000F7B50446154694F84100202826
:104E900036D1019800B10DB90120FEBD0198206204
:104EA000A584E58400206064212084F84100154831
:104EB000A16BC8631448A16B08641448A16BC86453
:104EC0000020A16B086501AE23681A1D31682B46CE
:104ED000A06BFCF7E5FC6FF040002168086000BFA4
:104EE00000BF2168143151E8001F41F080002168A3
:104EF000143141E80002002AF3D100BF0020CCE7C2
:104F00000220CAE7476F00089F6F00081F6E000865
:104F100010B504460320444908704448844216D121
:104F2000012211034248FCF731FE4248B0F8041157
:104F30008230FBF7FFF900203E49A1F804018022EE
:104F40003D493E48FFF726FF3D49087059E03B4880
:104F5000844240D13848801EB0F804118230FBF7FB
:104F6000E9F900203449891EA1F804013548007888
:104F7000012806D003280DD0052813D0062828D1F3
:104F800018E080222B49891C2848FFF703FF2C4991
:104F900088701FE080222C492C48FFF7FBFE28492F
:104FA000487017E0802224492448FFF7F3FE244983
:104FB00008700FE00220264981F8C10080221E49B6
:104FC0001E48FFF7E7FE1E490870002021490880AF
:104FD00000E000BF15E01D48844212D11A48801E2F
:104FE000B0F804118230FBF7A5F900201649891E9C
:104FF000A1F80401802210491048FFF7CBFE1049A8
:10500000087000200F4908701348007850B1134809
:1050100000683FF05BFB124800683FF057FB002040
:105020000D49087010BD00005C0000209CD80120D4
:105030000000024088D5012090D60120E4D801204C
:1050400063C1012062C1012096D7012074D90120DB
:105050005C090020A8C4012000C0012008C0012074
:105060001CC00120704700BFFEE701460868406988
:10507000C0F38020B0B16FF480600A6850610020F6
:105080000863202081F83D00002081F83E00086C74
:1050900040F00400086400BF002081F83C0000BF1D
:1050A000012070470020FCE72DE9F84304460D4637
:1050B00090461E46E76A2068006840F480602168D8
:1050C0000860082F04D0012F02D017F5803F06D1C9
:1050D0002068006840F480702168086008E0206B58
:1050E000112805D12068006840F4807021680860AC
:1050F000434600224FF001112046009600F003F9CC
:1051000060B12068006800F48070B0F5807F02D143
:105110004FF4007020640320BDE8F8832069B0F5E7
:10512000804F05D1E8B240F001002168086149E0F4
:1051300005F44070F02141EAE0102168086133462F
:1051400042462649204600F03DF908B10120E3E738
:10515000E8B221680861334642462049891F20464B
:1051600000F030F908B10120D6E700BF0020009020
:1051700020684069009020688069009000BF00BFEF
:105180002068006840F4807021680860434600226F
:105190004FF001112046009600F0B5F858B1206894
:1051A000006800F48070B0F5807F02D14FF4007089
:1051B00020640320B0E705F44070F12141EAE010DB
:1051C00021680861334642460449891F204600F0A1
:1051D000F9F808B101209FE700209DE708000100D1
:1051E0002DE9F84304460D4617469846E66A082E10
:1051F00004D0012E02D016F5803F06D12068006849
:1052000040F480702168086008E0206B122805D106
:105210002068006840F48070216808603B460022E6
:105220004FF001112046CDF8008000F06CF860B11D
:105230002068006800F48070B0F5807F02D14FF4E0
:10524000007020640320BDE8F8832069B0F5804F2A
:1052500004D105F0FE002168086112E005F44070F9
:10526000F02141EAE0102168086143463A460B49C3
:10527000204600F0A7F808B10120E4E7E8B2216871
:10528000086143463A460549891F204600F09AF8CE
:1052900008B10120D7E70020D5E700000800010091
:1052A00070B504460D46164625E02046FFF7DDFEA4
:1052B00008B1012070BD681CE8B1FCF76DFC801BD3
:1052C000A84200D8BDB920684069C0F3800090B9F9
:1052D00000202063202084F83D00002084F83E0058
:1052E000206C40F02000206400BF002084F83C00C7
:1052F00000BF0120DEE720684069C0F3800000287D
:10530000D3D00020D6E72DE9F04104460D461746DC
:105310001E46DDF8188038E0701CA8B3FCF73CFC92
:10532000A0EB0800B04200D876BBC5F307400128C7
:105330000AD120684069A9B20840A9B2884201D1C7
:1053400001200BE0002009E020688069A9B2084034
:10535000A9B2884201D1012000E00020B84214D156
:1053600000202063202084F83D00002084F83E00C7
:10537000206C40F02000206400BF002084F83C0036
:1053800000BF0120BDE8F081FFE7C5F30740012819
:105390000AD120684069A9B20840A9B2884201D167
:1053A00001200BE0002009E020688069A9B20840D4
:1053B000A9B2884201D1012000E00020B842ABD060
:1053C0000020DFE72DE9F04104460D4616461F4652
:1053D00058E020684069C0F38020E8B12068006888
:1053E00040F40070216808606FF4806021684861B3
:1053F00000202063202084F83D00002084F83E0037
:10540000206C40F00400206400BF002084F83C00C1
:1054100000BF0120BDE8F081701C90B3FCF7BCFB1D
:10542000C01BB04200D866BBC5F3074001280AD1B3
:1054300020684069A9B20840A9B2884201D1012080
:105440000BE0002009E020688069A9B20840A9B2F9
:10545000884201D1012000E0002090B900202063A3
:10546000202084F83D00002084F83E00206C40F0AD
:105470002000206400BF002084F83C0000BF012011
:10548000C8E7FFE7C5F3074001280AD12068406953
:10549000A9B20840A9B2884201D101200BE0002046
:1054A00009E020688069A9B20840A9B2884201D108
:1054B000012000E0002000288BD00020AAE770B572
:1054C00004460D46164637E020684069C0F30010D8
:1054D000A0B16FF0100021684861002020632020F7
:1054E00084F83D00002084F83E00206C206400BF5A
:1054F000002084F83C0000BF012070BDFCF74CFB8D
:10550000801BA84200D8BDB920684069C0F3801054
:1055100090B900202063202084F83D00002084F80A
:105520003E00206C40F02000206400BF002084F882
:105530003C0000BF0120E0E720684069C0F3801014
:105540000028C1D00020D8E770B504460D461646A5
:1055500025E02046FFF789FD08B1012070BD681CD9
:10556000E8B1FCF719FB801BA84200D8BDB9206840
:105570004069C0F3C01090B900202063202084F857
:105580003D00002084F83E00206C40F020002064A4
:1055900000BF002084F83C0000BF0120DEE7206847
:1055A0004069C0F3C0100028D3D00020D6E7000027
:1055B0001FB50020009001900290039014481549F7
:1055C0000860002048600021124881600161017676
:1055D00080F82010C162104981620021C160012160
:1055E000C161002180F8301001214161FBF7BAFC54
:1055F00008B1FBF79EFB0120009001900020029073
:1056000069460448FBF7E4FB08B1FBF792FB1FBDBA
:1056100000200140C4D301200100000F1CB5002070
:10562000009001900C480D4908600846FBF784FE85
:1056300008B1FBF77EFB00200090022001900022C1
:1056400069460648FBF7FFFD08B1FBF772FB002136
:105650000248FBF7E6FE1CBD007400406CD401203C
:1056600008B500BF002000902A48006840F4800080
:10567000284908600846006800F48000009000BFD8
:1056800000BF00BF002000900846006840F40010F2
:1056900008600846006800F40010009000BF00BFDA
:1056A000002205211020FCF701FF1020FCF7EAFE84
:1056B000002205211120FCF7F9FE1120FCF7E2FE83
:1056C000002205213820FCF7F1FE3820FCF7DAFE35
:1056D000002205213920FCF7E9FE3920FCF7D2FE33
:1056E000002205213A20FCF7E1FE3A20FCF7CAFE31
:1056F000002205214520FCF7D9FE4520FCF7C2FE1B
:10570000002205214620FCF7D1FE4620FCF7BAFE18
:1057100008BD00003038024000B5B9B01C22304945
:1057200032A8FAF7E0FD002132A828F03FFF2D490A
:1057300008601C222A491C312BA8FAF7D4FD00214D
:105740002BA828F033FF284908601C22244938314F
:1057500024A8FAF7C8FD002124A828F027FF234930
:1057600008601C221E4954311DA8FAF7BCFD002117
:105770001DA828F01BFF1E4908601C221849703123
:1057800016A8FAF7B0FD002116A828F00FFF194956
:1057900008601C2212498C310FA8FAF7A4FD0021E1
:1057A0000FA828F003FF144908601C220C49A831F7
:1057B00008A8FAF798FD002108A828F0F7FE0F497D
:1057C00008601C220649C43101A8FAF78CFD0021AB
:1057D00001A828F0EBFE0A49086039B000BD0000BE
:1057E0008047040804C0012008C001200CC001202B
:1057F00010C0012014C0012018C001201CC00120CD
:1058000020C0012000B587B0142102A8FAF792FD4C
:1058100000BF00200190AC48006840F01000AA4989
:1058200008600846006800F01000019000BF00BF4B
:1058300000BF002001900846006840F004000860A6
:105840000846006800F00400019000BF00BF00BFE0
:10585000002001900846006840F08000086008467B
:10586000006800F08000019000BF00BF00BF002072
:1058700001900846006840F0010008600846006892
:1058800000F00100019000BF00BF00BF00200190A8
:105890000846006840F0020008600846006800F012
:1058A0000200019000BF00BF00BF00200190084629
:1058B000006840F0080008600846006800F0080032
:1058C000019000BF00BF002249F6BC717F48FCF781
:1058D0005DF900224CF221017D48FCF757F90122C5
:1058E0004FF488717A48FCF751F900224DF22C21CF
:1058F0007848FCF74BF9012291037448FCF746F90C
:1059000000224FF2F3117448FCF740F90122910292
:105910007148FCF73BF900224FF418416F48FCF73F
:1059200035F93C200290012003900020049005905E
:1059300002A96648FCF728F84FF480400290012045
:105940000390022004900020059002A96048FCF713
:105950001BF848F2111002900120039000200490DF
:10596000059002A95A48FCF70FF8022002904FF464
:10597000041003900020049002A95548FCF704F895
:1059800001200290002003900120049002A95348B6
:10599000FBF7FAFF202002900120039000200490E2
:1059A0000120059002A94A48FBF7EEFF042002906F
:1059B00001200390002004900120059002A9454891
:1059C000FBF7E2FF4FF4F06002900120039000200B
:1059D00004900320059002A93C48FBF7D5FF4FF443
:1059E000584002900120039000200490012005906F
:1059F00002A93648FBF7C8FF4DF22820029001208B
:105A0000039000200490059002A93248FBF7BCFFE8
:105A10004FF4A060029001200390049000200590B4
:105A200002A92D48FBF7B0FF4FF400600290002060
:105A30000390049002A92848FBF7A6FF4FF2B30099
:105A4000029001200390002004900320059002A9F9
:105A50002148FBF799FF4FF4084002900120039082
:105A600000200490059002A91C48FBF78DFF4FF41D
:105A70008050029011200390012004900320059093
:105A800002A91648FBF780FF4020029001200390F6
:105A900000200490059002A90F48FBF775FF102025
:105AA0000290002003900120049002A90948FBF70E
:105AB0006BFF002205210720FCF7F8FC0720FCF70C
:105AC000E1FC07B000BD0000303802400010024089
:105AD0000008024000040240000C024000000240A6
:105AE00010B50C480C4908604CF250304860002159
:105AF00009488160C1604FF480410161002141612A
:105B00008161C1610162FCF74DF808B1FBF711F941
:105B100010BD000000540040EC06002010B50B48FA
:105B20000B4908600B484860002109488160C1604A
:105B30004FF480410161002141618161C1610162D5
:105B4000FCF730F808B1FBF7F4F810BD005C00403A
:105B500040070020A086010010B50E480E490860DD
:105B60004FF48270486000210B488160C160016180
:105B700001214161490281612821C1610021016245
:105B8000416281620A21C162FDF792F808B1FBF718
:105B9000D0F810BD0030014080D4012010B50E486F
:105BA0000E4908604FF48270486000210B48816004
:105BB000C160016101214161490281612021C1610E
:105BC00000210162416281620A21C162FDF770F821
:105BD00008B1FBF7AEF810BD00380040D8D4012062
:105BE00010B50F480F4908604FF4827048600021DB
:105BF0000C488160C16002210161002141614FF4C4
:105C0000007181612021C1610021016241628162D4
:105C10000A21C162FDF74CF808B1FBF78AF810BD04
:105C2000003C004030D5012000B595B00020119017
:105C30001290139014900F9010901C2108A8FAF75E
:105C400079FB20216846FAF775FB2D482D4908603D
:105C500040F2DB50486000212A4881603621C16053
:105C600000210161416180218161FDF775FD08B16D
:105C7000FBF75FF84FF48050119011A92148FDF710
:105C800022FF08B1FBF755F81E48FEF736FB08B1B6
:105C9000FBF74FF800200F9010900FA91948FDF75F
:105CA00043FC08B1FBF745F8602008901B200990E1
:105CB00000200A900B9004200C9000200D900E9074
:105CC000082208A90F48FEF796FA08B1FBF731F849
:105CD0000020009001900290039004904FF4005037
:105CE00005900020079069460648FDF7E3FB08B1E0
:105CF000FBF71FF80348FEF725FA15B000BD0000BA
:105D0000000001409407002000B587B000200390F8
:105D1000049005900690019002904FF08040144945
:105D20000860012048600021114881604AF2FF119B
:105D3000C160002101618161FDF70EFD08B1FAF734
:105D4000F8FF4FF48050039003A90948FDF7BBFE0C
:105D500008B1FAF7EEFF00200190029001A9044873
:105D6000FDF7E2FB08B1FAF7E4FF07B000BD000061
:105D7000DC07002000B58BB0002007900890099048
:105D80000A900590069001900290039004901F489D
:105D90001F4908600020486000211D4881604FF6BF
:105DA000FF71C1600021016180218161FDF7D4FC98
:105DB00008B1FAF7BEFF4FF48050079007A91448C6
:105DC000FDF781FE08B1FAF7B4FF1148FDF797FF20
:105DD00008B1FAF7AEFF00200590069005A90C481F
:105DE000FDF7A2FB08B1FAF7A4FF00200190012003
:105DF00002900020039004900C2201A90448FDF7B2
:105E00000FFF08B1FAF795FF0BB000BD000400408A
:105E1000240800201CB50020009001900E480F4976
:105E200008600120486000210C4881604AF2FF119F
:105E3000C16080218161FDF78FFC08B1FAF779FF1D
:105E400000200090019069460448FDF76DFB08B101
:105E5000FAF76FFF1CBD0000001000406C08002026
:105E600000B595B0002011901290139014900F90EF
:105E700010901C2108A8FAF75DFA20216846FAF76D
:105E800059FA2D482D49086040F2DB504860002146
:105E90002A4881603621C160002101614161802171
:105EA0008161FDF759FC08B1FAF743FF4FF48050C8
:105EB000119011A92148FDF706FE08B1FAF739FF44
:105EC0001E48FEF71AFA08B1FAF733FF00200F90C8
:105ED00010900FA91948FDF727FB08B1FAF729FF21
:105EE000602008901B20099000200A900B9004204D
:105EF0000C9000200D900E90042208A90F48FEF788
:105F00007AF908B1FAF715FF00200090019002908D
:105F1000039004904FF400500590002007906946CC
:105F20000648FDF7C7FA08B1FAF703FF0348FEF782
:105F300009F915B000BD000000040140B4080020BC
:105F400010B51548154908604FF4966048604FF445
:105F50008051124881600021C1604FF4C06101612D
:105F60000C21416100218161C161FEF7EDFC08B1A6
:105F7000FAF7DFFE09480068C06840F020000749D2
:105F80000968C86005480068C06840F0100003490F
:105F90000968C86010BD0000001001409CD80120B5
:105FA00010B51348134908604FF4E13048600021F0
:105FB00010488160C16001610C2141610021816153
:105FC000C161FEF7C1FC08B1FAF7B3FE09480068E9
:105FD000C06840F0200007490968C86005480068AB
:105FE000C06840F0100003490968C86010BD000097
:105FF00000440040E4D8012010B50B480B4908606C
:106000004FF4E1304860002108488160C1600161BF
:106010000C21416100218161C161FEF795FC08B14D
:10602000FAF787FE10BD0000004800402CD901207F
:1060300010B51348134908604FF4E130486000215F
:1060400010488160C16001610C21416100218161C2
:10605000C161FEF779FC08B1FAF76BFE09480068E8
:10606000C06840F0200007490968C860054800681A
:10607000C06840F0100003490968C86010BD000006
:106080000014014074D9012000BFFEE730B502467C
:106090004FF6FF7012B10446A14200D130BD11E0AD
:1060A00012F8014B604000230AE000F0010424B123
:1060B00040104AF20104604000E040105C1CE3B272
:1060C000082BF2DB0C1EA1F10105A9B2E8D100BF3B
:1060D000E4E700BFFEE70000F8B504460D460020E7
:1060E0000090002631490860012211033048FBF777
:1060F0004DFD022008F039F800224FF480512C4861
:10610000FBF744FD022008F030F814B1602000F0E5
:10611000EBF82849097804EA0100284308B1032074
:1061200000E0022002464FF47A7369462248FCF7E9
:10613000FBFE9DF800001D490968084300021B4949
:1061400008609DF80100096808431849086019496A
:10615000097804EA0100284398B19DF80200174924
:1061600008709DF800009DF8011008445B30C6B22D
:1061700046F0810611480078B04202D04FF0FF305F
:10618000F8BD012211030A48FBF700FD022007F0C9
:10619000ECFF00224FF480510548FBF7F7FC02208A
:1061A00007F0E3FF01480068EAE70000E80000208C
:1061B00000040240E0000020D8D40120E1000020CB
:1061C00010B56420FBF7B6FB00F06EF8642007F012
:1061D000CCFFDD2389222021022000F0EDF80220EF
:1061E00000F010F80549086000224FF4805104487F
:1061F000FBF7CCFC022007F0B8FF10BDDC0000204C
:106200000004024070B50446012211031948FBF74F
:10621000BDFC022007F0A9FF00224FF48051154871
:10622000FBF7B4FC022007F0A0FF44F0400000F0B0
:106230005BF800F027F81049087000F023F80F49C8
:10624000087000F01FF80E490870022007F08DFF5B
:10625000012211030748FBF799FC07480078000466
:106260000649097840EA01200549097840EA010514
:10627000284670BD00040240EC000020ED00002024
:10628000EE0000200EB50020029001904FF47A70CD
:10629000012301AA02A900900248FCF7E5FF9DF83E
:1062A00004000EBDD8D4012010B5012211030D4801
:1062B000FBF76CFC022007F058FF00224FF48051DE
:1062C0000848FBF763FC022007F04FFF022000F0B4
:1062D0000BF80A2007F049FF012211030148FBF7E0
:1062E00055FC10BD0004024001B582B000200190B1
:1062F0004FF47A70012301AA02A900900148FCF72B
:10630000B3FF0EBDD8D401202DE9F04104460D465F
:1063100016461F460120FFF775FF0C48007800F075
:10632000BF0040EAC71040EAC5003043C3B2084886
:10633000007800F0F80040EA04020648007800F017
:106340007F01012000F038F8BDE8F081EE00002068
:10635000ED000020EC00002070B504460D46022040
:10636000FFF750FF45EA0410C3B20448027804481E
:106370000178022000F020F870BD0000ED00002040
:10638000EC00002010B504460220FFF73BFF074851
:10639000007800F0CF0040EA0410C1B2044803784E
:1063A00004480278022000F007F810BDEC0000203D
:1063B000EE000020ED0000202DE9F04104460D46DE
:1063C00016461F46012211031C48FBF7DFFB022083
:1063D00007F0CBFE00224FF480511848FBF7D6FBA4
:1063E000022007F0C2FE44F02000FFF77DFF012CE1
:1063F00002D105F07F0100E029460846FFF774FF4F
:106400003046FFF771FF3846FFF76EFF022007F0B6
:10641000ACFE012211030948FBF7B8FB012C01D1A6
:10642000012000E0002006490978C1F380110840EE
:1064300010B1012003490870BDE8F081000402405A
:10644000EC000020E0000020F8B504460E4615469A
:106450006068B0F5827F0DD1A068B0F5004F03D021
:10646000A068B0F5806F05D12068006820F040007A
:10647000216808606068B0F5827F1FD1A068B0F520
:10648000806F0DD03346002280212046009500F019
:1064900069F808B3606D40F0200060650320F8BD26
:1064A0003346002201212046009500F05BF898B1A8
:1064B000606D40F0200060650320F0E73346002265
:1064C00001212046009500F04DF828B1606D40F0A4
:1064D000200060650320E2E70020E0E77CB5044689
:1064E0000E4615463346012202212046009500F053
:1064F00039F828B1606D40F02000606503207CBD54
:10650000164800681821B0FBF1F01549B0FBF1F016
:106510004FF47A71484301906068B0F5827F0DD1E5
:106520003346002280212046009500F01BF898B1E8
:10653000606D40F0200060650320E0E700BF019837
:1065400000B908E00198401E019020688068C0F3FF
:10655000C0100028F3D100BF0020D0E740C00120C8
:1065600040420F002DE9F84F04460D4690461E4666
:10657000DDF82890FBF710FBA0EB0900371AFBF7BA
:106580000BFB82462C480068C0F3CB307843009068
:1065900045E0701C002842D0FBF7FEFAA0EB0A0091
:1065A000B84200D2A7BB2068406820F0E000216814
:1065B00048606068B0F5827F0DD1A068B0F5004FEB
:1065C00003D0A068B0F5806F05D12068006820F086
:1065D000400021680860A06AB0F5005F0DD100BFDF
:1065E0002068006820F40050216808602068006876
:1065F00040F400502168086000BF012084F8510079
:1066000000BF002084F8500000BF0320BDE8F88FD1
:10661000FFE7009800B900270098401E009020680E
:1066200080682840A84201D1012000E000204045B8
:10663000AFD10020EAE7000040C00120002400BFE5
:1066400000203CF0A9FFC0F180000549888114B901
:1066500000203DF067F941F2883027F096FFEFE720
:10666000CC67012010B500BF502080F31188BFF324
:106670004F8FBFF36F8F00BF3DF002FF18B14FF097
:1066800080500449086000BF002080F3118800BFDB
:1066900010BD000004ED00E000B593B0302107A864
:1066A000F9F748FE142102A8F9F744FE00BF0020C4
:1066B00001902348006840F0805021490860084656
:1066C000006800F08050019000BF00BF00BF0020B4
:1066D00001901C48006840F480401A490860084650
:1066E000006800F48040019000BF00BF01200790C7
:1066F0000004089002200D9041050E910A210F918F
:106700004FF496711091022111910421129107A862
:10671000FCF780F808B1FAF70CFB0F20029002207A
:10672000039080200490400105900690022102A869
:10673000FBF70EFF08B1FAF7FCFA13B000BD00003A
:1067400040380240007000400348006840F4700088
:10675000014908607047000088ED00E004206849A6
:10676000087005204870674890ED000ABDEEC00A29
:1067700010EE100A00B28880624890ED0A0ABDEE61
:10678000C00A10EE100A00B2488004208871062169
:106790005B48C1715B4890ED0B0ABDEEC00A10EE7C
:1067A000100A01B256484181564890ED150ABDEED7
:1067B000C00A10EE100A01B251480181042050496C
:1067C000087307214E4841734E4890ED160ABDEEFE
:1067D000C00A10EE100A01B249480182494890ED02
:1067E000200ABDEEC00A10EE100A01B24448C18171
:1067F00004204349887408214148C174414890ED00
:10680000210ABDEEC00A10EE100A01B23C48C18256
:106810003C4890ED2B0ABDEEC00A10EE100A01B202
:106820003748818204203649087609213448417668
:10683000344890ED2C0ABDEEC00A10EE100A01B2E9
:106840002F4881832F4890ED360ABDEEC00A10EE26
:10685000100A01B22A4841830420294988770A2175
:106860002748C177274890ED370ABDEEC00A10EEE1
:10687000100A01B222484184224890ED410ABDEE3F
:10688000C00A10EE100A01B21D48018404201C4900
:1068900081F824000B211A4880F82510194890ED42
:1068A000420ABDEEC00A10EE100A01B2144801857A
:1068B000144890ED4C0ABDEEC00A10EE100A01B269
:1068C0000F48C18404200E4981F82A000C210C488D
:1068D00080F82B100B4890ED4D0ABDEEC00A10EE6B
:1068E000100A01B20648C185064890ED570ABDEE70
:1068F000C00A10EE100A01B20148818570470000FD
:106900009C670120C8C2012010B50248FDF763FB57
:1069100010BD00009407002010B50248FDF75BFB96
:1069200010BD0000DC07002010B50248FDF753FB46
:1069300010BD00002408002010B50348FAF7BBFC86
:106940000248FDF748FB10BD6CD401206C08002004
:1069500010B50248FDF73FFB10BD0000FCDB012035
:1069600010B50248FDF737FB10BD0000B408002049
:1069700010B502682D4B98420ED0B0F1804F0BD06D
:106980002B4B984208D02B4B984205D02A4B98426B
:1069900002D02A4B984203D122F070024B681A436E
:1069A000224B984220D0B0F1804F1DD0204B98420E
:1069B0001AD0204B984217D01F4B984214D01F4B2F
:1069C000984211D01E4B98420ED01E4B98420BD0CD
:1069D0001D4B984208D01D4B984205D01C4B984245
:1069E00002D01C4B984203D122F44072CB681A4368
:1069F00022F080034C6943EA040202608B68C362A0
:106A00000B688362094B984202D00C4B984201D12B
:106A10000B69036301234361036903F001031BB1A5
:106A2000036923F00103036110BD00000000014071
:106A30000004004000080040000C00400004014039
:106A4000004001400044014000480140001800405F
:106A5000001C00400020004030B501F01F0501245B
:106A600004FA05F3046A9C430462046A01F01F05FA
:106A700002FA05F52C43046230BD30B501F00F0574
:106A8000042404FA05F3046A9C430462046A01F0D6
:106A90000F0502FA05F52C43046230BD30B50C46F3
:106AA000816821F47F4142EA03252543294381601F
:106AB00030BD0A46816821F0700142F00703194396
:106AC0008160704730B5026A056A25F001050562EC
:106AD0004368846924F0700424F003040D682C4397
:106AE00022F002028D682A43104DA84200D103E033
:106AF0000F4DA84206D100BF22F00802CD682A43FC
:106B000022F00402094DA84202D0094DA84207D143
:106B100023F4807323F400734D692B438D692B4359
:106B2000436084614D684563026230BD00000140EE
:106B30000004014030B5026A056A25F010050562BF
:106B40004368846924F4E04424F440740D6844EA02
:106B5000052422F020028D6842EA0512124DA84257
:106B600000D103E0114DA84207D100BF22F08002FE
:106B7000CD6842EA051222F040020B4DA84202D035
:106B80000A4DA84209D123F4806323F400634D69C0
:106B900043EA85038D6943EA8503436084614D6858
:106BA0008563026230BD0000000001400004014026
:106BB00030B5026A056A25F4807505624368C469C8
:106BC00024F0700424F003040D682C4322F40072B6
:106BD0008D6842EA0522124DA84200D103E0114D12
:106BE000A84207D100BF22F40062CD6842EA052224
:106BF00022F480620A4DA84202D00A4DA84209D16F
:106C000023F4805323F400534D6943EA05138D693F
:106C100043EA05134360C4614D68C563026230BD39
:106C2000000001400004014030B5036A056A25F404
:106C3000805505624468C26922F4E04222F4407241
:106C40000D6842EA052223F400538D6843EA0533B8
:106C5000084DA84202D0084DA84204D124F4804433
:106C60004D6944EA85144460C2614D68056403625D
:106C700030BD0000000001400004014030B50B466B
:106C80001446026A056A25F001050562816921F052
:106C9000F00141EA041122F00A021A438161026202
:106CA00030BD000070B50C461546026A066A26F033
:106CB000010606628169184EB04214D0B0F1804FCF
:106CC00011D0164EB0420ED0154EB0420BD0154E1C
:106CD000B04208D0144EB04205D0144EB04202D09B
:106CE000134EB04201D1012600E000261EB121F072
:106CF0000301294301E041F0010121F0F001F026F8
:106D000006EA0316314322F00A0204F00A0632436F
:106D10008161026270BD000000000140000400407B
:106D200000080040000C0040000401400040014009
:106D30000018004030B50B461446026A056A25F07B
:106D400010050562816921F4704141EA043122F0A5
:106D5000A00242EA03128161026230BD70B50C46A6
:106D60001546026A066A26F010060662816921F459
:106D7000407141EA052121F470414FF4704606EA62
:106D80000336314322F0A002A02606EA041632435D
:106D90008161026270BD70B50C461546026A066AD2
:106DA00026F480760662C16921F00301294321F0AF
:106DB000F001F02606EA0316314322F420624FF474
:106DC000206606EA04263243C161026270BD70B5D6
:106DD0000C461546026A066A26F480560662C169A8
:106DE00021F4407141EA052121F470414FF47046CD
:106DF00006EA0336314322F420424FF4204606EAE5
:106E000004363243C161026270BD70B50546AC6B99
:106E10000020E085E0842046FDF720FC70BD70B5C1
:106E200006460025B46B20684069C0F3C01594F88D
:106E30004100212805D125B10020E084204600F042
:106E4000FBF820684069C0F3801594F842002228BE
:106E500005D125B10020E085204600F0A7F8606C40
:106E600040F0100060642046FDF7F8FB70BD70B57F
:106E70000546AC6B2868006800F48070002842D199
:106E8000E08500BF00BF21680C3151E8001F21F4EC
:106E9000807021680C3141E80002002AF3D100BF64
:106EA00000BF00BF2168143151E8001F21F001002C
:106EB0002168143141E80002002AF3D100BF00BF6D
:106EC00000BF2168143151E8001F21F04000216803
:106ED000143141E80002002AF3D100BF202084F8D9
:106EE0004200206B01280ED100BF00BF21680C3189
:106EF00051E8001F21F0100021680C3141E8000228
:106F0000002AF3D100BF00206063206B012804D168
:106F1000A18D2046FDF75CFB02E02046FDF750FF07
:106F200070BD70B50546AC6B01206063206B012815
:106F300005D1A08D41082046FDF74AFB02E020461E
:106F4000FDF73FFF70BD70B50546AC6B2868006863
:106F500000F48070F8B90020E08400BF00BF216811
:106F6000143151E8001F21F080002168143141E8FC
:106F70000002002AF3D100BF00BF00BF21680C311E
:106F800051E8001F41F0400021680C3141E8000247
:106F9000002AF3D102E02046FDF7BAFF70BD70B5BC
:106FA0000446A56B2846FEF75DF870BD00BF00BF24
:106FB00002680C3252E8002F22F4907102680C3201
:106FC00042E80013002BF3D100BF00BF00BF0268EE
:106FD000143252E8002F22F001010268143242E814
:106FE0000013002BF3D100BF016B01290ED100BFAC
:106FF00000BF02680C3252E8002F22F01001026834
:107000000C3242E80013002BF3D100BF202180F89E
:10701000421000210163704710B504462068C06823
:1070200020F040002168C860202084F841002046FC
:10703000FDF76EFF002010BD00BF00BF02680C32DC
:1070400052E8002F22F0C00102680C3242E800131F
:10705000002BF3D100BF202180F841107047F8B514
:10706000044694F84200222875D1A068B0F5805FEC
:107070000CD1206950B90025A66A20684068C0F389
:1070800008003080A06A801CA06215E0A56A002676
:10709000A068B0F5805F03D0A06828B9206918B94E
:1070A00020684068287004E02068406800F07F0095
:1070B0002870A06A401CA062E08D401E80B2E0856E
:1070C000002846D12068C06820F020002168C860F0
:1070D0002068C06820F480702168C860206840691A
:1070E00020F0010021684861202084F8420000203F
:1070F0006063206B012826D10020206300BF00BF01
:1071000021680C3151E8001F21F0100021680C317A
:1071100041E80002002AF3D100BF2068006800F0B7
:10712000100010280AD100BF0020009020680068DD
:10713000009020684068009000BF00BFA18D2046ED
:10714000FDF746FA02E02046FDF73AFE0020F8BDC2
:1071500001E00020FBE70220F9E700002DE9F84FED
:1071600004462068006920F44050E1680843216823
:1071700008612169A068084361690843E16908431F
:1071800000902068C06849F20C6188430099084368
:107190002168C8602068406920F44070A1690843F4
:1071A0002168486176492068884203D07549206883
:1071B000884203D1FBF7C6FA814602E0FBF7B2FA38
:1071C0008146E069B0F5004F6CD102206168A0FBF8
:1071D000015003461920A9FB007001462A46384693
:1071E000F9F750F86421B0FBF1F04FEA001A0220E1
:1071F0006168A0FB01510B461920A9FB00712A46CA
:107200003846F9F73FF8834602206168A0FB015039
:1072100003461920A9FB00712A463846F9F732F8CF
:107220006421B0FBF1F000EBC00101EB0010ABEB0F
:107230008000322101EBC0006421B0FBF1F000F0CE
:10724000F8000AEB400A02206168A0FB01500346E7
:107250001920A9FB007001462A463846F9F712F8B2
:10726000834602206168A0FB015003461920A9FB58
:1072700000712A463846F9F705F86421B0FBF1F0B1
:1072800000EBC00101EB0010ABEB8000322101EB01
:10729000C0006421B0FBF1F000F007005044216809
:1072A00088606AE004206168A0FB01500346192051
:1072B000A9FB007001462A463846F8F7E3FF8246EC
:1072C00004206168A0FB015003461920A9FB00704F
:1072D00001462A463846F8F7D5FF6421B0FBF1F0A5
:1072E00000EBC00101EB0010AAEB8000322101EBA2
:1072F00000106421B0FBF1F000F0F00A0420616896
:10730000A0FB017003461920A9FB00513A4628460C
:10731000F8F7B8FF6421B0FBF1F00AEB001A042083
:107320006168A0FB01510B461920A9FB00712A4698
:107330003846F8F7A7FF834604206168A0FB015098
:1073400003461920A9FB007001462A463846F8F783
:1073500099FF6421B0FBF1F000EBC00101EB0010DC
:10736000ABEB8000322101EB00106421B0FBF1F0A7
:1073700000F00F00504421688860BDE8F88F0000DD
:10738000001001400014014077B581B00446154655
:107390000298A062A58500206064222084F8420043
:1073A0002848E16BC8632848E16B08642748E16B13
:1073B000C8640020E16B086502AE32682368191DBD
:1073C0002B46E06BFAF76CFA00BF002000902068B3
:1073D0000068009020684068009000BF00BF2069EE
:1073E00070B100BF00BF21680C3151E8001F41F4AB
:1073F000807021680C3141E80002002AF3D100BFFF
:1074000000BF00BF2168143151E8001F41F00100A6
:107410002168143141E80002002AF3D100BF00BF07
:1074200000BF2168143151E8001F41F0400021687D
:10743000143141E80002002AF3D100BF002004B05B
:1074400070BD00006F6E0008236F00081F6E0008FB
:10745000014691F84100212828D18868B0F5805F65
:107460000BD1086948B90A6A1088C0F308000B6894
:107470005860086A801C086205E00B6A581C0862A4
:1074800018780B685860C88C401E80B2C88458B900
:107490000868C06820F080000B68D8600868C06881
:1074A00040F040000B68D860002070470220FCE7E5
:1074B0002DE9F84304460D4617469846089E31E0EC
:1074C000701C70B3FAF768FBA0EB0800B04200D85C
:1074D00016B90320BDE8F8832068C06800F00400F6
:1074E000F8B1802D1ED0402D1CD020680068C0F35C
:1074F000C000B0B100BF002000902068006800907C
:1075000020684068009000BF00BF2046FFF74EFD96
:107510000820606400BF002084F8400000BF012004
:10752000D8E7FFE7206800682840A84201D1012081
:1075300000E00020B842C3D00020CBE710B50348DC
:10754000FDF78EF8014827F0C7FA10BD9CD801203E
:1075500010B50348FDF784F8014827F0BDFA10BDC7
:10756000E4D8012010B50248FDF77AF810BD0000FC
:107570002CD9012010B50348FDF772F8014827F017
:10758000ABFA10BD74D9012000BFFEE70246024BE2
:1075900023F81210704700001C09002070B50A463D
:1075A000B2F57F4F18D10146CC1701EB5474E410AB
:1075B000164D2C5D0346DD1703EB5575ED10A3EB5F
:1075C000C5060125B5402C430146CD1701EB557585
:1075D000ED100E4E745518E0BAB90146CC1701EB08
:1075E0005474E410094D2C5D0346DD1703EB55750B
:1075F000ED10A3EBC5060125B540AC430146CD1700
:1076000001EB5575ED10014E745570BD34C001206D
:107610000FB4084B10B504A902AA039801F098FD15
:10762000044602A9002002F016F9204610BC5DF8BD
:1076300014FB00005798000837B514460846064B5F
:107640006A46214601F084FD04466946002002F0A6
:1076500002F920463EBD0000579800080248006825
:10766000C0F30220704700000CED00E010B50028C8
:1076700004DB0A07130E054A135406E00A07140E2A
:10768000034A00F00F031B1FD45410BD00E400E0B8
:1076900018ED00E002E008C8121F08C1002AFAD164
:1076A00070477047002001E001C1121F002AFBD182
:1076B000704770B50446002508E02168481C20602A
:1076C0000878303805EB850100EB41052168087822
:1076D00000F0C6F80028F0D1284670BD2DE9FF5F04
:1076E00082B00021DDE90430020DDDF840B0034333
:1076F00018D044F61050A2F2FF32424315141198EC
:1077000001281FD0A5EB0B00401C5FEA000A4FF0D8
:1077100000064E4FDFF83891B046504615D5CAF1F5
:10772000000413E0119801244AA3012801D16FEA53
:107730000B010298119AC0E90031C0E9024206B07B
:10774000BDE8F09FCBF10000DFE704460021404A8E
:10775000491842EB0450CDE9001012E0E00707D0D1
:1077600032463B4640464946F8F7CCFE80468946BD
:1077700032463B4610461946F8F7C4FE06460F4609
:107780006410002CEAD1DDE90401DDE90023BAF13F
:10779000000F06DAF8F7B6FE42464B46F8F7B2FE9F
:1077A00005E0F9F721F842464B46F9F71DF8044683
:1077B0000E460022284BF9F79FF803D84FF0FF3010
:1077C000014607E00022254B20463146F8F7F3FD3D
:1077D000F9F779F8102409E0002C0ADB0A220023CB
:1077E000F8F750FD039B30321A55641E50EA01022F
:1077F000F2D1641C039AC4F111031444119A012AB2
:1078000003D0012208430DD10AE0084304D0002030
:107810004FF0110B119072E7A3EB0B056D1E0DE0FD
:107820005B4504DD4FF0000205F1010504E003DAD9
:107830004FF00002A5F10105002AECD00298119941
:10784000C0E90231C0E9004579E7000000001440BA
:107850000000F03F300000000000F0430000E03F77
:107860000146302903DB392901DC01207047002063
:10787000FCE7000010B54421074800F017FE002285
:107880000F21064824F0FEF90549086002F0AAFC21
:1078900000200449087010BD00E40120C5A20008C2
:1078A00074010020700100202DE9F04F87B00746D9
:1078B0000C4615462946204600F066F920B94FF0DF
:1078C000FF3007B0BDE8F08F00222946204600F0C7
:1078D000FDF808B10020F4E70026204615F077FAFD
:1078E000401E00B20490204615F0F7F9401E00B289
:1078F000039068886188401A0FFA80FABAF1000F85
:1079000016DD2088ADF814006088ADF81600A08858
:10791000ADF818006088504400B2ADF81A00304647
:10792000711C4EB207EBC0000599016006994160D9
:10793000E8886188411A0398401A0FFA80FBBBF16E
:10794000000F1CDDB5F90600B4F90610884216DAFE
:107950002088ADF81400E888ADF81600A088ADF8CE
:107960001800E888584400B2ADF81A003046711C7F
:107970004EB207EBC0000599016006994160B5F968
:107980000200B4F90210884202DDB5F9020001E0FC
:10799000B4F902008046B5F90600B4F90610884231
:1079A00002DAB5F9060001E0B4F906000290029887
:1079B000A0EB08000FFA80F928882188401A00B24D
:1079C0000190019800281BDDB9F1000F18DD208817
:1079D000ADF81400ADF8168021880198084400B273
:1079E000ADF8180008EB090000B2ADF81A003046F7
:1079F000711C4EB207EBC000059901600699416009
:107A0000A8882188411A0498401A00B20090009872
:107A1000002818DDA888ADF81400ADF81680A988F4
:107A20000098084400B2ADF8180008EB090000B255
:107A3000ADF81A003046711C4EB207EBC000059934
:107A400001600699416030463BE730B50346B1F925
:107A50000040B2F90050AC4202DDB1F9004001E053
:107A6000B2F900401C80B1F90240B2F90250AC42B8
:107A700002DDB1F9024001E0B2F902405C80B1F9E7
:107A80000440B2F90450AC4202DAB1F9044001E01A
:107A9000B2F904409C80B1F90640B2F90650AC42FC
:107AA00002DAB1F9064001E0B2F90640DC800120BB
:107AB000B3F90040B3F90450AC4205DCB3F902401D
:107AC000B3F90650AC4200DD002030BDF8B50446E5
:107AD0000D4616460027B4F90000B5F9001088429B
:107AE00012DBB4F90200B5F9021088420CDBB4F9DC
:107AF0000400B5F90410884206DCB4F90600B5F9B3
:107B00000610884200DC01270FB90020F8BD0EB92D
:107B10000120FBE72088ADF800006088ADF8020086
:107B200032466946284600F0A7F808B90020EDE77C
:107B3000A088ADF800006088ADF8020032466946C2
:107B4000284600F099F808B90020DFE72088ADF852
:107B50000000E088ADF8020032466946284600F091
:107B60008BF808B90020D1E7A088ADF80000E088C4
:107B7000ADF8020032466946284600F07DF808B9A3
:107B80000020C3E70120C1E70246B2F90000B1F9C5
:107B90000430984213DCB2F90400B1F90030984285
:107BA0000DDBB2F90200B1F90630984207DCB2F9F8
:107BB0000600B1F90230984201DB01207047002035
:107BC000FCE7F8B504460D461646B4F90400B5F9CD
:107BD0000010884211DBB4F90600B5F902108842A2
:107BE0000BDBB4F90000B5F90410884205DCB4F9E8
:107BF0000200B5F90610884201DD0120F8BD0EB97A
:107C00000020FBE72088ADF800006088ADF8020096
:107C100032466946284600F02FF808B10020EDE70B
:107C2000A088ADF800006088ADF8020032466946D1
:107C3000284600F021F808B10020DFE72088ADF8E1
:107C40000000E088ADF8020032466946284600F0A0
:107C500013F808B10020D1E7A088ADF80000E08853
:107C6000ADF8020032466946284600F005F808B132
:107C70000020C3E70120C1E72DE9FC5F05460E4661
:107C800014464FF0000AB6F90000B5F9001088421A
:107C900013DBB6F90000B5F9041088420DDCB6F923
:107CA0000200B5F90210884207DBB6F90200B5F907
:107CB0000610884201DC4FF0010ABAF1000F02D130
:107CC0000020BDE8FC9F002C01DC0120F9E72846DC
:107CD00015F07DF8834600EBDB704710284614F062
:107CE000FCFF834600EBDB704FEA6008474501DA92
:107CF000384600E0404681464C4500DD4C46288829
:107D0000ADF800002888204400B2ADF8040068886F
:107D1000ADF802006888204400B2ADF806000022E9
:107D200031466846FFF7A8FF80B1BDF80400204443
:107D300000B2ADF80400BDF80600204400B2ADF872
:107D400006003146684622F073FABAE7E888001B5D
:107D500000B2ADF80200E888ADF806000022314616
:107D60006846FFF789FF80B1BDF80400204400B2E7
:107D7000ADF80400BDF80200001B00B2ADF802002F
:107D80003146684622F054FA9BE7A888001B00B2EF
:107D9000ADF80000A888ADF804000022314668461E
:107DA000FFF76AFF80B1BDF80000001B00B2ADF81C
:107DB0000000BDF80200001B00B2ADF80200314621
:107DC000684622F035FA7CE76888ADF802006888DA
:107DD000204400B2ADF80600002231466846FFF7A5
:107DE0004BFF80B1BDF80000001B00B2ADF80000F1
:107DF000BDF80600204400B2ADF8060031466846E2
:107E000022F016FA5DE701205BE710B5B1F900300A
:107E1000B2F90040A34202DAB1F9003001E0B2F950
:107E200000300380B1F90230B2F90240A34202DA15
:107E3000B1F9023001E0B2F902304380B1F9043007
:107E4000B2F90440A34202DDB1F9043001E0B2F915
:107E500004308380B1F90630B2F90640A34202DD56
:107E6000B1F9063001E0B2F90630C38010BD000060
:107E7000F8B5054623F001FF07460020009035B114
:107E80004C49E8680860284624F01AF803E016F028
:107E9000CBFB4849086047490968086922F068F83F
:107EA00044480068406920B142490968486922F0A5
:107EB0005FF840490968C86922F05AF83D490968E5
:107EC000086A22F055F83B480068006938B900207C
:107ED00038490968A1F8500100BF00BFF8BD22F081
:107EE0003BFA28F073FD28F011FB32480068B0F827
:107EF0005001002856D02F4800680068007C00F030
:107F0000010040B32B4800680068C068406810B3A7
:107F1000002419E02748006800F59870005D00B162
:107F200010E02448006800F5AC7000F021FB064624
:107F300020480068303000EBC400016831604068C0
:107F4000706000BF601C84B21A480068B0F850012D
:107F5000A042DFDC00BF4FF480711648006830306B
:107F60001DF01BFB20211348006800F598701DF0E0
:107F700014FB00200F490968A1F85001384623F08E
:107F80006FFE00900B4800680068406A50B10949D4
:107F9000096808680749096809684B6A06490A6858
:107FA000009998471DF028F800F03EF800F006F818
:107FB00000BF93E7DCC00120D8C0012010B5002429
:107FC00016E0C4EBC4000C4951F8200030B1C4EBFA
:107FD000C401094A52F821001DF0C0F8C4EBC401E5
:107FE000054A02EB81001C211DF0D7FA601CC4B2C7
:107FF000042CE6DB10BD0000DCE401200146094A48
:1080000010680BE042688A4202D002688A4204D1BA
:10801000027E22F00102521C027640690028F1D152
:1080200070470000BCC001207047000010B504215B
:10803000014800F03BFA10BDF4E3012010B5202107
:10804000014800F033FA10BD0CE401202DE9FF4790
:1080500004460D4616461F46DDE90C896FB9B8F592
:10806000807F0AD1002020806080681E00B2A0803E
:10807000701E00B2E080BDE8FF87002000900190F4
:1080800002900390ADF80450ADF80A60ADF80C50C2
:10809000ADF80E604B4642463946684621F0FEFF79
:1080A0004B464246394601A821F0F8FF4B4642466E
:1080B000394602A821F0F2FF4B464246394603A852
:1080C00021F0ECFFBDF90000BDF90410884202DA8E
:1080D000BDF9000001E0BDF90400BDF90810BDF9CB
:1080E0000C20914202DABDF9081001E0BDF90C1034
:1080F00088420BDABDF90000BDF90410884202DAAB
:10810000BDF900000DE0BDF904000AE0BDF908006A
:10811000BDF90C10884202DABDF9080001E0BDF992
:108120000C00801E00B22080BDF90000BDF90410D3
:10813000884202DDBDF9000001E0BDF90400BDF98F
:108140000810BDF90C20914202DDBDF9081001E0D4
:10815000BDF90C1088420BDDBDF90000BDF904101B
:10816000884202DDBDF900000DE0BDF904000AE01F
:10817000BDF90800BDF90C10884202DDBDF9080008
:1081800001E0BDF90C00801C00B2A080BDF9021016
:10819000BDF90600814202DABDF9020001E0BDF935
:1081A0000600BDF90A20BDF90E108A4202DABDF9B7
:1081B0000A1001E0BDF90E1088420BDABDF9021079
:1081C000BDF90600814202DABDF902000DE0BDF9F9
:1081D00006000AE0BDF90A10BDF90E00814202DA7C
:1081E000BDF90A0001E0BDF90E00801E00B26080FA
:1081F000BDF90210BDF90600814202DDBDF90200A1
:1082000001E0BDF90600BDF90A20BDF90E108A4251
:1082100002DDBDF90A1001E0BDF90E1088420BDD48
:10822000BDF90210BDF90600814202DDBDF9020070
:108230000DE0BDF906000AE0BDF90A10BDF90E0017
:10824000814202DDBDF90A0001E0BDF90E00801C8B
:1082500000B2E08000BF0EE72DE9F7430546164661
:108260000024134C23F009FD80463346294620465E
:10827000019A1BF0A9F907465FB900BF00BF2C2186
:1082800020461DF08AF94FF00040A0620020BDE8B2
:10829000FE830020A062E06918B9404623F0E0FCAC
:1082A000E061E06908B90120E0612046EFE70000E5
:1082B00030E4012010B51421114800F0F7F81BF04C
:1082C00035F9044600BF1CB900BF00BF00BFFEE780
:1082D00000BF14B900BF00BF10BD0A4920461BF003
:1082E0000DFA094920461BF00BFA084920461BF0FD
:1082F00009FA074920461BF0FFF900BFECE7000030
:1083000018E40120DD2C0208B131020839340208DA
:10831000A52C02082DE9FF4104460F4614B916F0BA
:1083200083F904460CB9BDE8FF81204616F015FA22
:1083300000B9F8E794F82800C0F3800010B100BF3E
:1083400000BFF0E71FB90020A4F85001EBE70020C0
:10835000ADF80800ADF80A00204616F07DF9401E81
:1083600000B2ADF80C00204616F0DCF9401E00B259
:10837000ADF80E0002AA39466846FFF766FB0646CE
:1083800006B9D0E72068007CC0F3400060B10298D5
:108390002063039860630120A4F85001606810B165
:1083A000606823F099FDBEE72068806918B12068F5
:1083B00069468269904700250BE004F1300000EB2C
:1083C000C50100226846FFF781FB00B1ABE7681CDE
:1083D00085B2B4F85001A842EFDCB4F8500120286F
:1083E00009DAB4F8502104F1300101EBC20069460A
:1083F00014F003FC0BE00020A4F85001B4F8502165
:1084000004F1300101EBC20002A914F0F6FBB4F84C
:108410005001401CA4F85001606810B1606823F05E
:108420005BFD00BF7FE770B50546284600F013F8F6
:10843000044600260CE02146284600F024F80646B3
:108440002146284600F0C0F820461CF087FE34463E
:10845000002CF0D170BD014609B900207047486872
:10846000FCE770B5064600243046FFF7F4FF0546EA
:1084700005E0641C2946304600F005F80546002D4D
:10848000F7D1204670BD02460B461068001D03441C
:108490001868704702460B46106803441868704716
:1084A000014609B9002070478868FCE70022426055
:1084B0008260CA1C22F003010160704770B5044657
:1084C000216801F108001CF06BFD0546A5B10022F2
:1084D0002946204625F03AFF29462046626825F0C5
:1084E00027FF606820B12A462046616825F02EFFEC
:1084F0006560A06800B9A560284670BD2DE9F0410F
:1085000006460D4606B115B90020BDE8F08130469B
:10851000FFF7A1FFA84206D13046FFF7CFFF044680
:1085200024BB0020F1E7316801F108001CF038FDA0
:1085300004460CB90020E8E729463046FFF7AAFFB9
:10854000074622463946304625F0F2FE3A46214695
:10855000304625F0FBFE22462946304625F0F6FE41
:108560002A462146304625F0E3FE00BF2046CCE7F0
:1085700070B50446216801F108001CF011FD0546A4
:10858000A5B100222946204625F0D2FE29462046E4
:10859000A26825F0DBFEA06820B12A462046A1682B
:1085A00025F0C6FEA560606800B96560284670BD0C
:1085B000014609B901207047486818B9886808B9A8
:1085C0000120F8E70020F6E72DE9F04104460D46CA
:1085D0000CB9BDE8F0812046FFF73DFFA8420FD15E
:1085E00029462046FFF74FFF6060606810B9002001
:1085F000A0602FE000222046616825F0A7FE29E058
:108600002046FFF74DFFA8420FD129462046FFF72D
:1086100041FFA060A06810B9002060601AE000224D
:108620002046A16825F084FE14E029462046FFF785
:1086300031FF064629462046FFF725FF07463A4602
:108640003146204625F074FE32463946204625F054
:108650007DFE00BF00BFBCE710B5044620688068FF
:1086600018B120682146826890472068006828B1C8
:108670002068006820602046FFF7EEFF10BD01462D
:10868000886818B18868B0F9160070470020FCE7C8
:108690000146886818B18868807E8009704700208C
:1086A000FCE72DE9F04104460D4616461DB916B902
:1086B0000120BDE8F08120461DF0A4F8A068008AE2
:1086C000284400B2A1680882A068408A304401B200
:1086D000A0684182012332462946204620F018F83E
:1086E00000220B21204619F0E1FB0746012F01D0A3
:1086F0003846DEE720461FF05DFF0120D9E7F7B5D9
:1087000082B004460E4614B9049805B0F0BD00BF0F
:108710006222314620461FF0BBF90190019D00BF47
:10872000BDB12868A8B100BF6322314620461FF0C2
:10873000AFF901900198C0B207464FB13A462B6895
:108740002846049998470190BDF80400ADF8100040
:1087500000BF0498D9E700002DE9F04F95B004461A
:108760008B4691469A461E9D608C20F0080008308A
:108770006084A4F820902A89594620461FF088F981
:108780001490A4F820A02A89594620461FF080F9A9
:108790001390608C20F008006084DDE9131088429B
:1087A0000CD1DDE91310884208D1BDF85000BDF8A6
:1087B0004C10884202D115B0BDE8F08FA4F820908B
:1087C0002A89594620461FF063F91490A4F820A086
:1087D000594620460FF053FB12902989129A1068CF
:1087E000149A23F02DF828890B2833D147F6FF710E
:1087F0001498884202D0139888422BD120461FF04B
:10880000ABFB009000EBD070471020461EF072F8D2
:10881000009000EBD0704FEA600847F6FF711498A3
:10882000884208D1781C08F10101884200DA01E091
:1088300008F10100149047F6FF711398884208D19F
:10884000781C08F10101884200DA01E008F101001A
:10885000139000BF2348FFF731FE064600BF1EB944
:1088600000BF00BF00BFFEE700BF06B9A3E7149832
:10887000F0601398306134602889B080C6F808B081
:1088800001A814F049F8314601A814F0D3F81649AC
:1088900001A814F09FF81548039000BF144901A8DF
:1088A00014F0A0F8FF22002101A814F0B5F82988DF
:1088B00001A814F0A3F8698801A814F084F8E86806
:1088C000089000BF01A8002190F8422061F3000247
:1088D00080F8422000BF2869079001A814F0C0F872
:1088E00000BF68E724E40120C52204086D250408C0
:1088F0009D24040810B514210148FFF7D7FD10BDD1
:1089000024E401202DE9FE4F04460F4690464FF027
:10891000000900254CE1E06800EBC5004068C0F3A9
:10892000406000B143E1E16801EBC501496821F015
:108930007F4021F0E2FA064626EA070008B9012046
:1089400000E00020029026EA080008B9012000E0BB
:1089500000200190DDE90101814270D0E06850F80B
:1089600035A04FF0000B6A461021504622F0C4FBA0
:1089700010B14FF0010B98E06A461121504622F0E9
:10898000BBFB10B14FF0010B8FE06A46122150463D
:1089900022F0B2FB10B14FF0010B86E06A461321C2
:1089A000504622F0A9FB10B14FF0010B7DE06A4662
:1089B0001521504622F0A0FB10B14FF0010B74E0DE
:1089C0006A461421504622F097FB10B14FF0010B7C
:1089D0006BE06A460A21504622F08EFB10B14FF040
:1089E000010B62E06A466B21504622F085FB10B114
:1089F0004FF0010B59E06A466C21504622F07CFB97
:108A000010B14FF0010B50E06A460121504622F0B0
:108A100073FB10B14FF0010B47E06A46042150464A
:108A200022F06AFB10B14FF0010B3EE06A460221D2
:108A3000504622F061FB18B14FF0010B35E0B5E074
:108A40006A460321504622F057FB10B14FF0010B4C
:108A50002BE06A460521504622F04EFB10B14FF044
:108A6000010B22E06A460621504622F045FB10B178
:108A70004FF0010B19E06A463221504622F03CFBD0
:108A800010B14FF0010B10E06A466E21504622F003
:108A900033FB10B14FF0010B07E06A466D215046E1
:108AA00022F02AFB08B14FF0010BBBF1000F02D0FE
:108AB0000320BDE8FE8F6A466921504622F01CFB68
:108AC00010B14FF0020970E06A466A21504622F068
:108AD00013FB10B14FF0020967E06A466E21504661
:108AE00022F00AFB10B14FF002095EE06A466D21E8
:108AF000504622F001FB10B14FF0020955E06A46E2
:108B00003721504622F0F8FA10B14FF002094CE03C
:108B10006A463821504622F0EFFA10B14FF00209B0
:108B200043E06A463521504622F0E6FA10B14FF094
:108B300002093AE06A464021504622F0DDFA10B1BF
:108B40004FF0020931E06A464521504622F0D4FA3E
:108B500010B14FF0020928E06A464121504622F048
:108B6000CBFA10B14FF002091FE06A46422150468D
:108B700022F0C2FA10B14FF0020916E06A46432112
:108B8000504622F0B9FA10B14FF002090DE06A46E2
:108B90004921504622F0B0FA10B14FF0020904E02A
:108BA000B9F1000F01D14FF0010900BF00BF6D1CEA
:108BB000608CC0F30510A8423FF6ADAE484678E79A
:108BC0000148006870470000DCC001207047014682
:108BD000C1F30412072A00DD0722D0B2704700005B
:108BE00001464FF6FF70814201D11F20704709B93D
:108BF0000020FBE7712902DA0948405CF6E7A1F1A1
:108C0000710081B20748006838B1074800688142A6
:108C100003D204480068405CE8E70020E6E7000073
:108C2000D08104088C0100209001002010B518218B
:108C30000348FFF73BFC012023F060F810BD000063
:108C4000D0E301202DE9F04106460C4617461D46AB
:108C500029463046084A126890472060206830B1A3
:108C6000296888190021044A1268904700E0002012
:108C70003860BDE8F081000034C101202DE9F04FDB
:108C800087B004460F4692469846DDE910560DB16E
:108C9000002028801CB9002007B0BDE8F08F2078A4
:108CA00008B90020F8E70FB90020F5E74FF00009F8
:108CB00006F0020010B906F0040098B1002000E0B0
:108CC000401C215C0A2905D0215C0D2902D0215CC1
:108CD0000029F5D1215C01B1401C15B14FF0FF31E5
:108CE0002980D9E706F0020008B141F6FF7800209C
:108CF0000690059038E000200490059808B90120FE
:108D000000E0002006A904AACDE90062CDE9021026
:108D10000599601843465246394623F089FA83463E
:108D20000498A8EB00000FFA80F8049848440FFA62
:108D300080F9BBF1000F00D11CE005985844059064
:108D400020780A2802D020780D2800D112E005985A
:108D5000205C0A2803D00598205C0D2803D10598D3
:108D6000401C059006E000BF0598205C10B1B8F1EA
:108D7000000FC0DC00BF059870B905A92046094A5C
:108D800012689047834635B100225946384619F09B
:108D900011FA0FFA80F900BF0DB1A5F800900598FF
:108DA0007AE7000034C1012001460023B1F59C4F51
:108DB00005D349F6A570814201D8012070470022F1
:108DC00007E007A0805C884201D1012305E0501C28
:108DD000C2B203A0805C0028F3D100BF1846EDE7C3
:108DE000202C2E3B3A2D5F00024600200FA31B785B
:108DF0008B4211D113781BB90123137001200BE0B2
:108E00001378012B02D10023137005E01378022B95
:108E100002D10023137001201378012B04D12029E3
:108E200001D10223137001207047000023000000CD
:108E30002DE9F04781460E4614461F46DDF820A076
:108E400035461BE0600800FB075529464846D047D9
:108E5000B0F1000809DD04F0010080F00100C0EB72
:108E60005404E8190546064608E0B8F1000F02DA96
:108E70006408354602E02846BDE8F087002CE1D1C1
:108E80000020F9E72DE9FF4F85B08346DDE9158A1B
:108E9000DDE91349DDE91775129E05F00200F8B906
:108EA0004FB105F0010030B1B9F1000F02D105F06A
:108EB0000C0000B17F1E03E030222046641C3254B7
:108EC000544501D2202CF7D303E030222046641C05
:108ED000325405F0010018B1BC4201D2202CF4D369
:108EE00005F01000B0B305F4806050B94CB15445A2
:108EF00001D0BC4205D1641E1CB1B8F1100F00D1E5
:108F0000641EB8F1100F09D105F0200030B9202CF3
:108F100004D278222046641C325415E0B8F1100FB8
:108F200009D105F0200030B1202C04D2582220466F
:108F3000641C325408E0B8F1020F05D1202C03D292
:108F400062222046641C3254202C03D23022204658
:108F5000641C3254202C16D2B9F1000F04D02D22FB
:108F60002046641C32540EE005F0040020B12B2290
:108F70002046641C325406E005F0080018B1202297
:108F80002046641C3254CDE90275CDE90064584690
:108F900006A90EC900F0A2F809B0BDE8F08F2DE9CE
:108FA000FF4F8FB08046DDE91FABDDE91D96219DA7
:108FB0001C9C00270CB925F0100505F4806000B159
:108FC000E4B100BFB4FBF6F106FB1141C8B20A28B8
:108FD00002DA00F1300107E005F0200109B141217A
:108FE00000E0612101440A39CBB239467F1C07AA4F
:108FF0005354B4FBF6F40CB1202FE3D307A8CDE90A
:1090000004AB8DE8810203960695404610A90EC96F
:10901000FFF738FF13B0BDE8F08F2DE9FF4F8FB099
:10902000DDE9217BDDF89080209EDDE91C454FF0D5
:109030000009002184EA01006940084301D128F0B9
:10904000100808F4806028B1002184EA010069401A
:1090500008432DD000BF32463B4620462946F7F74D
:1090600011F902F0FF0ABAF10A0F02DA0AF1300030
:1090700007E008F0200008B1412000E061205044E2
:109080000A38C2B2484609F1010907A90A54324612
:109090003B4620462946F7F7F5F804460D460021E1
:1090A00084EA01006940084302D0B9F1200FD2D30D
:1090B0002398CDE9036BCDE9050807A91E98CDE9F2
:1090C000001902900FA80FC8FFF7DCFE13B0BDE82F
:1090D000F08F9A4200D28854704770472DE9FF5FA5
:1090E00005461446DDE90EA6DDE91087A34607F024
:1090F000020078B907F0010060B9B14607E02246E6
:10910000641C2020039B0199A84709F10109C1456E
:10911000F5D300BF08E02246641C711E0E461AF803
:109120000100039B0199A847002EF4D107F002002B
:1091300050B105E02246641C2020039B0199A847FA
:10914000A4EB0B004045F5D3204604B0BDE8F09FEA
:109150002DE9FF4F95B09A46884606460025EEE178
:10916000252877D100242746F94A0121039400E0FD
:10917000044316F8013F203B01FA03F01042F7D1F7
:1091800030782A2811D06FF02F033078A0F1300208
:10919000092A16D8039A44F0020402EB820203EB78
:1091A00042021044761C0390EFE758F8042B039218
:1091B000002A03DA504244F40054039044F00204BD
:1091C000761C30782E2816D116F8010F44F00404CE
:1091D0002A280DD06FF02F023078A0F13003092B30
:1091E00009D807EB870302EB4303C718761CF3E7A4
:1091F00058F8047B761C30786C280FD006DC4C289D
:1092000017D068280DD06A2814D104E0742810D033
:109210007A280FD10DE044F400140AE044F48014DD
:1092200001E044F440147278824202D104F58014C3
:10923000761C761C307866280BD013DC582877D043
:1092400009DC002875D04528F6D04628F4D04728F8
:109250001AD193E118E0632835D0642879D06528C5
:1092600012D18BE1702873D008DC6728F1D069280F
:109270006FD06E280DD06F2806D1ACE073282CD0AB
:10928000752874D0782853D05246179990476D1C92
:1092900054E1C4F30250022809D003280DD0D8F8B5
:1092A000001004280DD00D6008F1040846E1D8F83C
:1092B0000010EA17C1E90052F6E7D8F800100D8057
:1092C000F2E70D70F0E718F8041B8DF8001000208D
:1092D0008DF80100EB46012003E058F804BB4FF085
:1092E000FF3061074FF0000102D40DE009F10101E8
:1092F0008946B9420FDA8145F8DB1BF809100029CD
:10930000F4D108E009F1010189468142FADB1BF83A
:1093100009100029F6D103985346A0EB090721460E
:109320003846179A00F080FA284400EB090507E058
:1093300044E008E10DE01BF8010B524617999047F5
:10934000B9F10109F7D2534621463846179AF2E09F
:1093500039E00A21C4F302524FF0000B0091022AB7
:1093600006D058F8040BC117032A09D00AE023E0FD
:1093700008F1070020F00702F2E80201904605E03C
:1093800000B2C117042A01D140B2C117002906DA80
:109390000A460021404261EB02012D2202E0220533
:1093A00004D52B228DF80420012203E0E20701D02E
:1093B0002022F7E7914657E00A2100E010214FF004
:1093C000000B00910BE010214FF0000B44F004045F
:1093D0000827009103E008204FF0000B0090C4F331
:1093E0000252022A05D058F8040B0021032A08D0A3
:1093F00008E008F1070020F00702F2E802019046B9
:1094000003E080B2042A00D1C0B24FF00009220765
:109410002AD53278702A07D0DDF800C08CF0100C05
:109420005CEA0B0C05D00EE040228DF804200122EE
:1094300008E050EA010306D030238DF804308DF89F
:10944000052002229146009B83F0080353EA0B0398
:109450000AD150EA010201D1620705D530228DF808
:1094600004204FF001097F1E3278582A04D039A217
:109470000C920CAA02920BE03BA2F9E75B46009A21
:10948000F6F700FF0C9B9B5C029A521E029213702F
:1094900050EA0102F2D1029804A9081A00F1200B47
:1094A000600702D524F4803400E001275F4502DD27
:1094B000A7EB0B0000E0002000EB0B0100900398ED
:1094C0004944401A0390E00306D453462146179AB4
:1094D000039800F0A9F90544002706E001A85246C8
:1094E000C05D179990476D1C7F1C4F45F6DBE0036C
:1094F0000CD553462146179A039800F095F9054478
:1095000004E030205246179990476D1C0099481E80
:1095100000900029F5DC08E0029802995246007894
:10952000491C0291179990476D1CBBF10001ABF1EA
:10953000010BF1DC5BE100F065F90544761C307845
:1095400000287FF40DAE19B02846BDE8F08F00006A
:109550000928010030313233343536373839616209
:1095600063646566000000003031323334353637CD
:10957000383941424344454600000000600700D4AA
:10958000062708F1070020F00700F0E802238046D4
:1095900003F0004C5FEA0C0001D097A009E0200521
:1095A00001D596A005E0E00701D095A001E0AFF25B
:1095B0004C001390307823F0004365280CD006DC73
:1095C000452809D046281DD047287FD13BE0662892
:1095D00018D067287AD136E00021112F01DB112045
:1095E00000E0781CCDE9000104A90CA8FEF776F88C
:1095F000DDE90D010C9A4FF0000B07F10109109203
:1096000000914EE04FF000400097CDE9011004A911
:109610000CA8FEF763F8DDE90D020C9B0F994FF0E3
:10962000000B91461093009211B9791C00EB0109CF
:10963000B7EB090003D4C0F1FF3B07F10109A9EB27
:109640000700019042E0012F00DA01270021112FCD
:1096500001DD112000E03846CDE9000104A90CA885
:10966000FEF73CF8DDE90D010C9A00914FF0000B7C
:10967000B946109221070FD4009A4A4503DA914661
:1096800001E0A9F10109B9F1010F05DD109AA9F175
:109690000101515C3029F4D0B84202DA10F1040F14
:1096A00003DA0121CDE9011010E0002803DC834436
:1096B000A9EB000102E0411C494500DD8946A0EB11
:1096C0000B00401C01904FF000400290200705D491
:1096D0000198484502DB4FF0FF30019000208DF8E3
:1096E0004B0002980DF14B07B0F1004F25D002203E
:1096F0000C902B200D90029800280CDA404202902A
:109700002D200D9007E00A210298F6F7C9FF3031AD
:10971000029007F8011D0C99481E0C900029F2DCFC
:1097200002980028EFD1791E0D980870307800F06B
:10973000200040F0450007F8020D11A8C01BC01D15
:1097400002901398007800B1012000EB0901019804
:1097500001EBE071029801440398401A401E039007
:10976000E00306D453462146179A039800F05CF8AC
:1097700005441398007818B15246179990476D1C0C
:10978000E00323D553462146179A039800F04CF87E
:1097900005441BE0BBF1000F07DB0098584504DDD2
:1097A0001098179910F80B0001E0179930205246D5
:1097B000904701980BF1010B401E05F10105019046
:1097C00004D12E205246179990476D1CB9F1000123
:1097D000A9F10109DEDC05E017F8010B52461799E3
:1097E00090476D1C0299481E02900029F4DC5346F4
:1097F0002146179A03989EE62D0000002B000000DA
:10980000200000002DE9F041044600251E461746C1
:10981000880404D405E039462020B0476D1C641E3E
:10982000F9D52846BDE8F0812DE9F0410446002530
:109830001E469046C80301D5302700E02027880443
:1098400004D505E041463846B0476D1C641EF9D585
:109850002846BDE8F0810A68531C0B601070704701
:109860002DE9FF4F8BB0074600250C9800B9FA4F41
:10987000EAE20E98007825280AD02A466D1C0E9937
:109880000878DDE90C13B8470E98401C0E90DBE217
:109890000E98401C0E90002400BF0E9800782B28D4
:1098A00019D004DC20281ED023282CD123E02D2819
:1098B00009D0302827D144F001040E98401C0E90A6
:1098C00001200A9022E044F002040E98401C0E9001
:1098D00001200A901AE044F004040E98401C0E90F7
:1098E00001200A9012E044F008040E98401C0E90EB
:1098F00001200A900AE044F010040E98401C0E90DB
:1099000001200A9002E000200A9000BF00BF0A98E0
:109910000028C2D180460E990878FDF7A1FF20B13A
:109920000EA8FDF7C6FE804612E00E9800782A28A1
:109930000ED1189901C91891002804DA44F00204E4
:10994000C0F1000800E080460E99491C0E9100BF4E
:109950004FF000090E9800782E281FD144F480643F
:109960000E98401C0E900E990878FDF779FF20B1F3
:109970000EA8FDF79EFE814610E00E9800782A287A
:109980000CD1189901C91891002801DD014600E0A9
:10999000002189460E99491C0E9100BF0E9800784F
:1099A0006C280AD004DC682816D06A2835D128E053
:1099B000742820D07A2830D129E044F480740E989D
:1099C000401C0E900E9800786C2804D144F400746A
:1099D0000E98401C0E9021E044F080040E98401C2C
:1099E0000E900E980078682804D144F040040E9838
:1099F000401C0E9012E044F480740E98401C0E90AF
:109A00000CE044F400740E98401C0E9006E044F400
:109A100080740E98401C0E9000E000BF00BF0E98AE
:109A2000007869281DD00EDC622821D006DC2528AC
:109A30007ED050281AD058287BD115E0632879D0E1
:109A40006428F9D10CE0732875D004DC6F280ED09F
:109A50007028F1D109E0752804D07828ECD102E013
:109A600000BF00BF00BF00BF00BF00BF00BF00BFFE
:109A70000E980078782803D00E980078582801D1E5
:109A8000102623E00E980078702803D00E980078F6
:109A900050280CD1102644F0100444F480740E9821
:109AA0004078562812D10E98401C0E900EE00E9869
:109AB00000786F2801D1082608E00E980078622807
:109AC00001D1022602E00A2624F010040E98007844
:109AD000582803D00E980078502801D144F0200473
:109AE0000E980078692805D00E980078642801D077
:109AF00024F00C0404F4806008B124F001040E98F2
:109B00000078692803D00E98007864287CD104F48A
:109B10000070B8B31898C01D20F007001890D0E965
:109B200000AB189A083218920020CDE9069803E09D
:109B300073E17CE1F2E01CE1CDE904600894BAEB4A
:109B400000017BEB000001DA012000E00020002191
:109B500002900846B1EB0A0170EB0B0002DA5046A6
:109B6000594605E000200146B0EB0A0061EB0B010D
:109B7000CDE900012A463846DDE90C13FFF74DFA1E
:109B80000546C7E0FFE704F48070D0B1189850F89C
:109B900004AB18904FEADA70CDE903980296059469
:109BA000BAF1000F01DD514601E0CAF10001CDE933
:109BB00000102A463846DDE90C13FFF7F0F9054698
:109BC000A8E004F0400028B1189810F8041B189081
:109BD000C8B20DE004F0800028B1189830F8041BDA
:109BE000189008B204E0189800681899091D189197
:109BF00082464FEADA70CDE9039802960594BAF1ED
:109C0000000F02DD514602E00BE0CAF10001CDE990
:109C100000102A463846DDE90C13FFF7C0F9054667
:109C200078E00E980078562818D1189850F804ABB0
:109C30001890DAF804000068099009980090DAF8A2
:109C400000300D98421B0C9841193846FFF708FE6A
:109C50000544002009905DE0DB90000804F40070EA
:109C6000D0B11898C01D20F00700CDE906980894DF
:109C700018900020CDE904600290189903C9189A41
:109C800008321892CDE900012A463846DDE90C1366
:109C9000FFF7C3F905463DE004F4807098B1002257
:109CA000CDE9039802960594189800681899091D43
:109CB000CDE9000218912A463846DDE90C13FFF77A
:109CC0006EF9054626E004F0400028B1189810F817
:109CD000041B1890C8B20DE004F0800028B1189859
:109CE00030F8041B189088B204E01898006818999E
:109CF000091D189182460020CDE900A0CDE9039806
:109D0000029605942A463846DDE90C13FFF747F919
:109D1000054600BF0E98401C0E9093E0012604F00B
:109D2000020050B905E02A466D1C2020DDE90C1325
:109D3000B8473046761C4045F5D3189911F8043BD6
:109D4000D8B22A466D1C1891DDE90C13B84704F00F
:109D5000020050B105E02A466D1C2020DDE90C13FD
:109D6000B8473046761C4045F5D30E98401C0E90FF
:109D700068E0189850F804AB18905046B9F1000FFD
:109D800001D0494601E04FF0FF310A46014600E0AC
:109D9000491C0B781BB1131EA2F10102F8D10E1A57
:109DA00004F4806028B14E4501D2304600E04846B8
:109DB000064604F0020050B905E02A466D1C20203A
:109DC000DDE90C13B8473046761C4045F5D306E074
:109DD0001AF8010B2A466D1CDDE90C13B8479AF8F6
:109DE000000040B104F480600028F1D0B9F1000017
:109DF000A9F10109ECD104F0020050B105E02A46B6
:109E00006D1C2020DDE90C13B8473046761C404518
:109E1000F5D30E98401C0E9014E02A466D1C2520A8
:109E2000DDE90C13B8470E98401C0E900AE02A4654
:109E30006D1C0E990878DDE90C13B8470E98401C8C
:109E40000E9000BF00BF00BF0E98007800287FF47E
:109E500010AD0D98854201D2284601E00D98401EB4
:109E600002460020DDE90C13B84728460FB0BDE8D4
:109E7000F08F2DE9F04104460E46002774B13146BB
:109E8000204600F006F90546B5F5803F05D20C2DB9
:109E900001D9284600E00C20074600BF3846BDE83F
:109EA000F081000010B504462CB9002210210548AD
:109EB000F7F76CFE04E0012210210248F7F766FE76
:109EC00010BD00000008024038B504461FA000681D
:109ED000009003221E49684636F042FB1D48006888
:109EE0001D4908601A48007800041949497800EBB8
:109EF0000120174989780844164908600846006817
:109F000000F4000070B1084600686FF07F414840DF
:109F10001049086008460068401C08600846006850
:109F2000404208600B4890ED000AB8EEC00ADFED31
:109F30000B0A20EE200AF0EE040A20EE200ADFEDE4
:109F4000080A80EE201A84ED001A38BDFFFFFF00DA
:109F5000CA000020D4000020D000002000007A4475
:109F60000000004B30B587B005460C461B48007812
:109F700038B90120194908700020194908700DF0FE
:109F80003BF80020FFF78EFF0A2039F045FC00F077
:109F900029F8052039F040FC002040210390CDE94C
:109FA000040101210690CDE900012023024601466B
:109FB00002902AF0A3FF052039F02EFC00F01EF8D5
:109FC0001E2039F029FC2046FFF77EFF0120FFF715
:109FD00069FF052039F020FC07B030BDC800002023
:109FE0003BC0012008B506200090012202496846C6
:109FF00036F0B6FA08BD0000B800002008B5082009
:10A00000009001220249684636F0AAFA08BD000015
:10A01000B80000202DE9FC4106460F4614464020BA
:10A0200000EB8701601E0844C0B28DF800000025D7
:10A0300004E0715D681C0DF80010C5B2A542F8DBA4
:10A04000621C0349684636F08BFABDE8FC810000CB
:10A05000B8000020024600BF481E084018B100BFEB
:10A0600000BF00BFFEE700BF481E1040101A704737
:10A0700010B502464B1E13444C1E23EA040000BFD9
:10A080004B1E0B401BB100BF00BF00BFFEE700BF6F
:10A0900010BD024600BF481E084018B100BF00BFF7
:10A0A00000BFFEE700BF481E10444B1E9843704798
:10A0B0002DE9F84F81460E46924699F8090000F0C6
:10A0C0000700022801D1304600E05046834656453D
:10A0D00001DD304600E050460746032000EB470014
:10A0E00020F0030000F1100539480068394909687B
:10A0F000A0EB0108002405EB0800374909688842F5
:10A1000006D233480468606820F0004060603AE09E
:10A1100031480068854221D813E04FF0FF300090AD
:10A12000002269462D480FF035FB002269462C4875
:10A130000FF030FB2648006826490968A0EB0108AB
:10A1400000BF08EB0500244909688842E5D820488B
:10A150000468606820F00040606014E028461AF04F
:10A160001FFF044600BF1CB900BF00BF00BFFEE7D1
:10A1700000BF14B90020BDE8F88F606820F00040EF
:10A1800000F10040606032465946484602F07EFECB
:10A190002060606800F04040401C6060606820F013
:10A1A00080406060A781A4F80EB06068C00F20B145
:10A1B000204600F11001A16008E005480068103059
:10A1C000A060034800682844014908602046D2E79F
:10A1D0002C010020880100202801002027660108AA
:10A1E000C9BF010810B50120074908700748FEF7EC
:10A1F00032F920B90648006821F062FE03E0044805
:10A20000006821F069FE10BD7001002000E401200B
:10A210007401002010B5044694F84200C0F34000D9
:10A2200070B9B4F8400000280ADDB4F840004FF6D9
:10A23000FF71884204D0B4F84000401EA4F84000EA
:10A24000B4F84000D0B9A06B20B194F84200C0F33C
:10A25000400098B121461A48FEF7B6F9FFF7C2FF51
:10A26000E06810B12046E1688847206910B12046B7
:10A270002169884720461AF071FF1FE0E06B4042D9
:10A280002063A06BD0B194F84210C1F3400111B922
:10A29000616B4942216394F842104908C94394F81C
:10A2A000422061F3410284F84220206AA16A2162BF
:10A2B000A062E06AA16BE162A06300BF10BD000074
:10A2C00000E401202DE9F04180464248006821F079
:10A2D000C7FC06464048007880F001003E490870FF
:10A2E0003E48FEF7B8F804466BE000203C49087091
:10A2F00094F84200C0F3800037490978884253D06F
:10A30000354801783034A07C61F38200A074206865
:10A310008719A07C303CC0F3C00010BB206B002824
:10A320001FDC002F1DDB94F8420000F0010060B933
:10A33000606950B12046616988470546206A284413
:10A340002062A06A2844A06200BFA06810B1204625
:10A35000A168884794F8420020F00800083084F88B
:10A360004200206B30442063206B00281BDBD4E9C3
:10A370000B10884201DDE06A20632046E1698847CE
:10A380000546606AA84206D06562606818B1294631
:10A39000D4E900029047D4E90B10884202DB204642
:10A3A000FFF738FF00BF00BF0D48007820B10B4811
:10A3B000FEF751F8044604E021460848FEF763F82A
:10A3C0000446002C91D121F058FC02490860BDE8F8
:10A3D000F08100006C0100207101002000E40120E8
:10A3E0007001002070B504460D46606818B129461A
:10A3F0006068FFF7F7FF206818B1294620462268F9
:10A40000904770BD2DE9FF4F8FB01F46DDF8888063
:10A410001C980E901D980D9000200B9023980428F6
:10A4200006D0052809D006280CD014281AD114E02B
:10A4300000200C904FF0020917E001200C904FF023
:10A44000030912E001200C904FF00209FEF7B8FB5F
:10A4500005462868008F0B9007E001200C904FF014
:10A46000020902E013B0BDE8F08F00BF002489E1CB
:10A470001E9860430E9901EB20201C901F986043AA
:10A480000D9901EB20201D901C9805121D980612B5
:10A49000002D07DB1098854204DA002E02DB1198AC
:10A4A000864203DB002008F8040069E11C98C0B272
:10A4B0000A901D9800F0FF0A0A98802807DA4FF0EA
:10A4C000FF3B0A98C0F17F0040000A9005E04FF082
:10A4D000010B0A98803840000A90BAF1800F07DA21
:10A4E0004FF0FF300990CAF17F004FEA400A05E0C3
:10A4F00001200990AAF180004FEA400A0F980890C5
:10A5000006FB07F000FB09F005FB09010898084469
:10A51000089005EB0B0000287EDB05EB0B01109883
:10A52000401E814278DC099830440028F4DB099809
:10A5300031181198401E8142F4DC08980790089861
:10A540000BFB09000690099800FB07F1089801FB36
:10A55000090005900C9800287FD0239B052B06D17D
:10A56000079B9878059B9978069B9A783BE0239BFC
:10A57000142B18D1DDF844C007FB0CFCDDF83CE0DF
:10A580000EEB4C0306FB073C1CF8050006FB073CE2
:10A59000AC441CF80B20DDF824C0B4440CFB073C91
:10A5A0001CF805101FE0239B062B19D1079B1B8865
:10A5B000BDF82CC063450BD0059B1B88BDF82CC093
:10A5C000634505D0069B1B88BDF82CC0634503D1AD
:10A5D000002308F80430D3E0FF20FF21FF2202E02F
:10A5E000FF20FF21FF22814207D001FB0AF3CAF5B9
:10A5F000807C00FB0C33C3F30721824209D00A9B05
:10A600005343DDF828C0CCF5807C00FB0C33C3F34A
:10A6100007228B185B1000E059E008F8043018F8A6
:10A62000043003B9ACE0079B93F800C05B780CEBF7
:10A6300003239BB20493059B93F800C05B780CEB5B
:10A6400003239BB20393069B93F800C05B780CEB4B
:10A6500003239BB202930CE0FFE707980088049065
:10A66000069800880290059800880390FF2008F85B
:10A670000400BDF81000BDF80C1088420CD1BDF8E4
:10A680001000BDF80810884206D1219800EB440064
:10A69000BDF81010018019E00AF0FF02DDE90301A6
:10A6A00013F036FD03900A98C2B20499029813F091
:10A6B0002FFD02907F22DDE9020113F029FD0190B8
:10A6C000219800EB4400BDF80410018057E0089980
:10A6D0000A78497802EB01218AB2219921F81420E5
:10A6E0002399052904D0062905D0142919D10EE093
:10A6F0000899887817E0219931F81410BDF82C20BA
:10A70000914201D1002100E0FF2108460BE0119A9F
:10A7100007FB02F10F9A02EB410106FB0711485DAE
:10A7200001E0FF2000BF00BF15B9BBF1000F06DB41
:10A730001099491EA9420BD1BBF1000F08DD0A99FF
:10A74000C1F1FF014143C1F3072108F8041015E0EE
:10A7500016B90999002906DB1199491EB1420AD19F
:10A760000999002907DDCAF1FF014143C1F307211F
:10A7700008F8041002E0002108F8041000BF00BF30
:10A78000601C04B220988442FFF672AE00BF69E6F6
:10A790002DE9F84F04468C4690469946109FDDE916
:10A7A0000A56AA460096002032E00C9941430AEB73
:10A7B00021250D994143DDF800B00BEB21262A122B
:10A7C0003312002A05DB624503DA002B01DB434527
:10A7D00002DB0021395419E0214603FB09FB0BEB96
:10A7E0004B0B02EB420EF344594491F800B091F840
:10A7F00001E00BEB0E2B1FFA8BFEDDF83CB02BF8C3
:10A8000010E091F802B007F800B000BF411C08B298
:10A810000E998842C9DBBDE8F88F000010B53048BA
:10A82000006800285BD000202D49086025F070F9F1
:10A830002C48007801281AD12B480078B8B92B4849
:10A84000C07E052801DB002002E02848C07E401CB5
:10A850002649C8760A46D27E254B53F82210254A4F
:10A86000D06A19F0C2F914202349088033E0234844
:10A8700000782149088021480078032811D003DCA2
:10A8800038B1012819D108E007280ED00F2814D1BB
:10A890000FE001201549C87613E002201349C8765D
:10A8A0000FE003201149C8760BE004200F49C87659
:10A8B00007E005200D49C87603E000200B49C87663
:10A8C00000BF00BF094AD27E094B53F82210094A43
:10A8D000D06A19F08AF909F075FC38F0F9F810BD62
:10A8E00088C401201301002014010020CCE50120C0
:10A8F00004020020AC040020FC080020120100200B
:10A9000010B586B000246F480078072879D2DFE8B8
:10A9100000F0042E53799EC3D2006B48007868B9CA
:10A9200014226AA101A8F5F71CFD01A839F068FA04
:10A9300065480078401C6449087017E06248007858
:10A94000401C614908700846007800EBC00101EB2B
:10A9500000104FF4FA71B1EB800F07DA00205A496A
:10A96000087058480078401C56490870A6E05648C0
:10A97000007840B959A039F037FA53480078401CA4
:10A980005149087017E050480078401C4E49087043
:10A990000846007800EBC00101EB00104FF4FA719B
:10A9A000B1EB800F07DA002047490870454800786E
:10A9B000401C4449087081E04348007840B94BA0EE
:10A9C00039F012FA40480078401C3F49087017E0FF
:10A9D0003D480078401C3C4908700846007800EB70
:10A9E000C00101EB00104FF4FA71B1EB800F07DAF0
:10A9F00000203549087033480078401C3149087000
:10AA00005CE05AE03048007840B93CA039F0ECF9FD
:10AA10002D480078401C2C49087017E02A4800781F
:10AA2000401C294908700846007800EBC00101EB82
:10AA300000104FF4FA71B1EB800F07DA00202249C1
:10AA4000087020480078401C1E49087036E01E48F7
:10AA5000007840B92DA039F0C7F91B480078401C98
:10AA60001949087017E018480078401C164908700A
:10AA70000846007800EBC00101EB00104FF47A713A
:10AA8000B1EB800F07DA00200F4908700D480078FD
:10AA9000401C0C49087011E080212048F5F74AFC61
:10AAA00000201E49891EA1F8020106480078401CBA
:10AAB0000449087002E0012400E000BF00BF204606
:10AAC00006B010BD490000204A00002047534454FE
:10AAD0005F534747545F56312E30000041542B5589
:10AAE000554944533D464646300D0A0041542B55C6
:10AAF0005549444E3D464646310D0A0041542B55BA
:10AB0000554944573D464646320D0A0041542B52A2
:10AB100045424F4F543D310D0A00000096D70120A9
:10AB200070B504460D462946204638F005FD70BD37
:10AB300070B504460D4600BF204600F03BF818B142
:10AB400000BF00BF00BFFEE700BF284600F050F97D
:10AB5000001D616808446060204600F03AF8204615
:10AB600070BD70B505460C46284600F041F904F169
:10AB70001001884201D3012070BD0020FCE701468E
:10AB8000A1F1080070477CB505460C46204600F050
:10AB90002FF906466A4601A922F01EFA21462846E8
:10ABA000DDE900320EF0DEF97CBD0146087900F0E7
:10ABB0000100704710B50446204600F019F908B9A5
:10ABC000012010BD0020FCE70146087900F00200DA
:10ABD000704770B50446204600F097F805462C6093
:10ABE000284670BD7CB506460C46002001900090BA
:10ABF00000256CB16A4601A9204622F00AFA0198A4
:10AC00000A2805DA6A4601A9304626F0C7FF05463C
:10AC100085B100BF284600F0EBF8A04203D200BF88
:10AC200000BF00BFFEE700BF29463046DDE9003225
:10AC300025F0C3FF28467CBD70B504462046FFF7CB
:10AC4000C8FF0546284600F0BEF8204600F0B6F8DA
:10AC500070BD70B50446204600F057F805462846FA
:10AC600000F0B6F8204600F0BEF870BD70B506469C
:10AC70000D46284600F049F8044600BF1CB900BF45
:10AC800000BF00BFFEE700BF2046FFF78EFF90B178
:10AC900000BF2846FFF78EFF18B100BF00BF00BFFE
:10ACA000FEE700BF2146304600F076F821462846F0
:10ACB000FFF73EFF0546284670BD70B506460D46B7
:10ACC0002846FFF781FFF0B1284600F057F8044608
:10ACD00000BF1CB900BF00BF00BFFEE700BF00BF40
:10ACE0002046FFF762FF18B900BF00BF00BFFEE7B4
:10ACF00000BF2146304600F04FF829462046FFF7B6
:10AD000017FF054600BF284670BD2DE9F0410446F7
:10AD1000204600F06DF8061F204600F0B8F8074600
:10AD2000314623F0CDFB054600BF2046FFF742FF2A
:10AD300018B100BF00BF00BFFEE700BF2846BDE856
:10AD4000F0812DE9F04106460C461546002794B1E6
:10AD500000BF1DB900BF00BF00BFFEE700BF2A460D
:10AD60002146304600F097F82046FFF772FF204654
:10AD700000F08DF807463846BDE8F08110B504466E
:10AD800000BF2046FFF720FF18B900BF00BF00BF7B
:10AD9000FEE700BF206810BD7CB505460C46204686
:10ADA00000F026F806466A4601A922F015F9214668
:10ADB0002846DDE9003225F000FF7CBD416841F006
:10ADC000010141607047416841F0020141607047F4
:10ADD000416821F0020141607047426802F00303BC
:10ADE0000B4343607047416821F0010141607047A7
:10ADF0000146486820F0030070472DE9F0470646F9
:10AE00000C46304600F043F88046211F23F058FBE3
:10AE100007463046FFF7ECFF211D451A00BF3846B4
:10AE200000F035F88146384600F031F880460421BC
:10AE3000FFF71EF9814503D000BF00BF00BFFEE74A
:10AE400000BF00BF3046FFF7D3FF2919091D884214
:10AE500003D000BF00BF00BFFEE700BF2946384651
:10AE6000FFF7BBFF00BF3846FFF7C2FF0C2803D235
:10AE700000BF00BF00BFFEE700BF21463046FFF71E
:10AE8000ACFF3846FFF7D8FE3846BDE8F0870146EC
:10AE900001F1080070472DE9F04106460C461546C1
:10AEA00000BF2046FFF781FE18B900BF00BF00BFFA
:10AEB000FEE700BF29462046FFF753FE78B129463A
:10AEC0002046FFF79AFF07462046FFF782FE3846E6
:10AED000FFF779FF39463046FFF755FE00BFBDE862
:10AEE000F0812DE9F04106460C46154600BF20468C
:10AEF000FFF75BFE18B100BF00BF00BFFEE700BF59
:10AF000029462046FFF72DFE88B129462046FFF747
:10AF100074FF07463846FFF75BFF39463046FFF7B8
:10AF2000A5FE074639463046FFF72DFE00BFBDE8B7
:10AF3000F08100002DE9F04F89B004460D46002154
:10AF400020461BF0C0FB30B91C2128461AF025FB17
:10AF500009B0BDE8F08F2946204600F00BFB2946DA
:10AF6000204600F07DF8002120461CF0D1FC08901E
:10AF7000002120461CF050FD0790002120461CF0C7
:10AF800045FB012800D100E0002081460021204639
:10AF90001CF09DFE0746002120461CF0D7FB06460C
:10AFA00042F2D170874205D1608CC0F3C02008B94D
:10AFB000012000E00020824620461BF024FC069081
:10AFC00000BF4FF0000824480288414620461CF08C
:10AFD0005FFD03900398C0B200BF8346AA68296949
:10AFE0002868CDE90209CDE900125A465146089B6E
:10AFF00006980CF0D1FF288342F2D170864205D129
:10B00000608CC0F3802008B9012000E0002005908A
:10B0100020461BF0D9FB049000BF4FF000080F48FA
:10B020000288414620461CF033FD03900398C0B2CD
:10B0300000BF83460023EA6869686869CDE90213A6
:10B04000CDE900025A46079BDDE904010CF0A4FF9C
:10B05000688300BF7CE70000F0C00120F4C001203D
:10B060002DE9F34F87B00C4607980CF079FA80462B
:10B0700007981BF0C8FB0690404602F08EFB20614B
:10B080002169480019F0D6FF20602169480019F0B5
:10B09000D1FFA060002548E05848029038F915001B
:10B0A00041F69A7188423FD10020019029E0019930
:10B0B00007981BF008FB0090514900981CF060FFB6
:10B0C00000B11BE000980CF069FA8246BAF1010F5A
:10B0D00000D013E000980CF051FA8346AB4500D045
:10B0E0000CE000981CF038FF0299884201DA0298BF
:10B0F00002E000981CF030FF029000BF0198401C55
:10B10000019007981BF0FDFA01998842CFD8029868
:10B11000002804DB0298A16821F8150003E0002153
:10B12000A06820F8151000BF6D1C2069A842B3D894
:10B130000026B14600251BE038F9150041F69B7149
:10B14000884202DB411A0E4411E041F69A718842AE
:10B1500006D1A16831F8151049440FFA81F906E0CB
:10B16000A16821F8150009EB00010FFA81F96D1CA7
:10B170002069A842E0D8002107981CF0C9FB05907F
:10B180002169491EDDE9050200FB112000B206908D
:10B190000698A0EB090007B2002F00DA00274FF055
:10B1A000FF30049000200390002513E038F91500CB
:10B1B00041F69B7188420CDB421A11B207FB01F287
:10B1C000B2FBF6F212B2A36823F81520049503919E
:10B1D00000BF6D1C2069A842E8D8049800280ADB4B
:10B1E0000398301A7843B0FBF6F0381A01B2A2681F
:10B1F000049822F8101009B0BDE8F08F01E0FFFFBD
:10B20000010006002DE9FC5F054600221146284694
:10B210001EF0D4FA002128461CF03CFA8146002199
:10B2200028461CF005FC484407B2002128461CF0C3
:10B2300033FB48440FFA80FA28461CF07BF9384467
:10B2400050440FFA80FB3B4E28461BF05AFA0190FF
:10B250004FF000085CE0A868006850F828403649C4
:10B2600020461CF08DFE00B150E020461DF01AFA79
:10B27000002839D1002120461CF08DF9009000985B
:10B2800030B1012807D0022804D0032815D100E0EE
:10B2900000BF00BF00BFB4F91A10B5F91600081AB4
:10B2A000401CB04201DA304605E0B4F91A10B5F995
:10B2B0001600081A401C06B214E0002120461CF0BB
:10B2C00042FD70B904F1140011F0D6FC3844B042CC
:10B2D00001DA304604E004F1140011F0CDFC3844EA
:10B2E00006B200BF00BF10E0B4F91A10B5F916009D
:10B2F000081A401CB04201DA304605E0B4F91A10D1
:10B30000B5F91600081A401C06B200BF08F1010882
:10B31000019880459FD30748864209D006EB0A0072
:10B3200006B25E4502DD3046BDE8FC9F5846FBE7AD
:10B330005846F9E701E0FFFF010004002DE9FC5F3A
:10B3400005460022114628461EF01CFA0021284618
:10B350001CF0A0F98246002128461CF021FB504435
:10B360000FFA80F8002128461CF0EAFA50440FFA40
:10B3700080F928461CF0EEF84844404400B20190A1
:10B38000724C28461BF0BDF98346002128461CF06C
:10B3900019F9012866D100265BE0A868006850F81A
:10B3A00026706B4938461CF0EBFD00B150E0384682
:10B3B0001DF078F9002839D1002138461CF0EBF84F
:10B3C0000090009830B1032805D0062804D0082842
:10B3D00015D102E000BF00BF00BFB5F91800B7F9F2
:10B3E0001410401A401CA04201DA204605E0B5F9CD
:10B3F0001800B7F91410401A401C04B214E00021E0
:10B4000038461CF094FC70B907F1140011F092FC5E
:10B410004044A04201DA204604E007F1140011F094
:10B4200089FC404404B200BF00BF10E0B5F9180029
:10B43000B7F91410401A401CA04201DA204605E07A
:10B44000B5F91800B7F91410401A401C04B200BF37
:10B45000761C5E45A1D33D48844269D004EB0900C7
:10B4600004B265E000265BE0A868006850F826702A
:10B47000374938461CF084FD00B150E038461DF0D5
:10B4800011F980BB002138461CF085F80090009827
:10B4900030B1012805D0042804D0072815D102E0D6
:10B4A00000BF00BF00BFB7F91800B5F91410401A6B
:10B4B000401CA04201DA204605E0B7F91800B5F9B2
:10B4C0001410401A401C04B215E0002138461CF04C
:10B4D0003AFC78B907F1140011F02CFC4844A04262
:10B4E00002DA204605E008E007F1140011F022FC22
:10B4F000484404B200BF00BF10E0B7F91800B5F926
:10B500001410401A401CA04201DA204605E0B7F9A9
:10B510001800B5F91410401A401C04B200BF761C84
:10B520005E45A1D30948844202D004EB080004B26E
:10B530000648844202D10198BDE8FC9F01988442EC
:10B5400001DD2046F8E70198F6E7000001E0FFFF83
:10B550000100040010B50446206819F0E7FD60689A
:10B5600019F0E4FDA06819F0E1FDE06819F0DEFDD6
:10B5700010BD00002DE9F34F87B00C4607980CF082
:10B5800037FC8046404602F008F960616169480076
:10B5900019F050FD60606169480019F04BFDE060F2
:10B5A000002547E05948029038F9150041F69A7194
:10B5B00088423ED14FF0000A29E0514607981BF01F
:10B5C00082F80190524901981CF0DAFC00B11CE0AD
:10B5D00001980CF02BFC8346BBF1010F00D014E066
:10B5E00001980CF013FC00900098A84200D00CE0E9
:10B5F00001981BF07FF90299884201DA029802E073
:10B6000001981BF077F9029000BF0AF1010A079830
:10B610001BF077F85045D0D80298002804DB029838
:10B62000E16821F8150003E00020E16821F8150029
:10B6300000BF6D1C6069A842B4D80026B146002541
:10B640001BE038F9150041F69B71884202DB411A74
:10B650000E4411E041F69A71884206D1E16831F852
:10B66000151049440FFA81F906E0E16821F8150048
:10B6700009EB00010FFA81F96D1C6069A842E0D85E
:10B68000002107981CF0C8F9069007981BF09CF859
:10B6900001466269521E069800FB121000B2059026
:10B6A0000598A0EB090007B2002F00DA00274FF041
:10B6B000FF30049000200390002513E038F91500B6
:10B6C00041F69B7188420CDB421A11B207FB01F272
:10B6D000B2FBF6F212B2E36823F815200495039149
:10B6E00000BF6D1C6069A842E8D8049800280ADBF6
:10B6F0000398301A7843B0FBF6F0381A01B2E268CA
:10B70000049822F8101009B0BDE8F08F01E0FFFFA7
:10B710000100060038B5044600256E222946204661
:10B720001CF0B6F90090009800B208B1022038BDB4
:10B7300000256D22294620461CF0AAF900900098A9
:10B7400000B2B0F5807F01D00220F0E70025612231
:10B75000294620461CF09CF900900098C0B2FF28B2
:10B7600001D00120E3E700256822294620461CF08D
:10B770008FF900900098C0B208B10120D7E70020EF
:10B78000D5E7000010B52DED028BB0EE408A9FED9D
:10B790003B0AF0EE408A3A48007820B101281CD0DC
:10B7A000022864D160E000244FF4FC600AF038FA0B
:10B7B00004024FF4FD600AF033FA04434AF6AA206B
:10B7C000844203D002202E49087005E001202C4954
:10B7D0000870162009F05EF84AE0F0EE040AB0EEB8
:10B7E000600A00203CE0274901EB8001D1ED000A0E
:10B7F000F4EEC80AF1EE10FA30D82249421C01EBEF
:10B800008201D1ED000AF4EEC80AF1EE10FA25DB50
:10B8100000EE900AB8EE601ADFED180A41EE000A59
:10B82000F0EE608A174901EB8201D1ED000A15495B
:10B8300001EB800191ED001A70EEC10A114901EB94
:10B84000800191ED001A38EE411A61EE001A81EE86
:10B85000A01A71EE280AF0EE608A03E0411CC8B21B
:10B860000A28C0DB00BF03E0F0EE488A00E000BF1A
:10B8700000BFB0EE680ABDEC028B10BD00000000F6
:10B88000F000002068DD012010B52DED028BB0EE38
:10B89000408A9FED3B0AF0EE408A3A48007820B19A
:10B8A00001281CD0022864D160E000244FF4047009
:10B8B0000AF0B6F904024FF406700AF0B1F9044335
:10B8C0004AF6AA20844203D002202E49087005E0DF
:10B8D00001202C490870122008F0DCFF4AE0F0EE4D
:10B8E000040AB0EE600A00203CE0274901EB800129
:10B8F000D1ED000AF4EEC80AF1EE10FA30D8224970
:10B90000421C01EB8201D1ED000AF4EEC80AF1EE0F
:10B9100010FA25DB00EE900AB8EE601ADFED180A87
:10B9200041EE000AF0EE608A174901EB8201D1ED89
:10B93000000A154901EB800191ED001A70EEC10A71
:10B94000114901EB800191ED001A38EE411A61EEC8
:10B95000001A81EEA01A71EE280AF0EE608A03E068
:10B96000411CC8B20A28C0DB00BF03E0F0EE488AE1
:10B9700000E000BF00BFB0EE680ABDEC028B10BD56
:10B980000000000039C00120B8DC012010B52DED09
:10B99000028BB0EE408A9FED3B0AF0EE408A3A48B7
:10B9A000007820B101281CD0022864D160E0002476
:10B9B0004FF446600AF034F9040240F668400AF099
:10B9C0002FF904434AF6AA20844203D002202E49CC
:10B9D000087005E001202C490870192008F05AFF72
:10B9E0004AE0DFED2A0AB0EE600A00203CE0284978
:10B9F00001EB8001D1ED000AF4EEC80AF1EE10FA75
:10BA000030D82349421C01EB8201D1ED000AF4EE4B
:10BA1000C80AF1EE10FA25DB00EE900AB8EE601AC3
:10BA2000DFED1C0A41EE000AF0EE608A184901EBD6
:10BA30008201D1ED000A164901EB800191ED001A57
:10BA400070EEC10A124901EB800191ED001A38EE47
:10BA5000411A61EE001A81EEA01A71EE280AF0EE8A
:10BA6000608A03E0411CC8B20A28C0DB00BF03E0C3
:10BA7000F0EE488A00E000BF00BFB0EE680ABDECFF
:10BA8000028B10BD00000000F3000020806AFB4123
:10BA900094DD0120F628944110B52DED028BB0EE17
:10BAA000408A9FED3B0AF0EE408A3A48007820B188
:10BAB00001281CD0022864D160E000244FF4CC603F
:10BAC0000AF0AEF804024FF4CD600AF0A9F804437E
:10BAD0004AF6AA20844203D002202E49087005E0CD
:10BAE00001202C490870152008F0D4FE4AE0DFED53
:10BAF0002A0AB0EE600A00203CE0284901EB8001F0
:10BB0000D1ED000AF4EEC80AF1EE10FA30D823495C
:10BB1000421C01EB8201D1ED000AF4EEC80AF1EEFD
:10BB200010FA25DB00EE900AB8EE601ADFED180A75
:10BB300041EE000AF0EE608A184901EB8201D1ED76
:10BB4000000A164901EB800191ED001A70EEC10A5E
:10BB5000124901EB800191ED001A38EE411A61EEB5
:10BB6000001A81EEA01A71EE280AF0EE608A03E056
:10BB7000411CC8B20A28C0DB00BF03E0F0EE488ACF
:10BB800000E000BF00BFB0EE680ABDEC028B10BD44
:10BB9000000000003CC001200000C843E4DC01209C
:10BBA00010B52DED028BB0EE408A9FED3B0AF0EE12
:10BBB000408A3A48007820B101281CD0022864D17C
:10BBC00060E000244FF42E600AF02AF8040240F6E8
:10BBD000E8200AF025F804434AF6AA20844203D05C
:10BBE00002202E49087005E001202C490870182019
:10BBF00008F050FE4AE0F6EE000AB0EE600A0020BF
:10BC00003CE0274901EB8001D1ED000AF4EEC80ABF
:10BC1000F1EE10FA30D82249421C01EB8201D1ED3D
:10BC2000000AF4EEC80AF1EE10FA25DB00EE900AE5
:10BC3000B8EE601AF8EE040A41EE000AF0EE608AEF
:10BC4000174901EB8201D1ED000A154901EB800192
:10BC500091ED001A70EEC10A114901EB800191EDDE
:10BC6000001A38EE411A61EE001A81EEA01A71EE48
:10BC7000280AF0EE608A03E0411CC8B20A28C0DB43
:10BC800000BF03E0F0EE488A00E000BF00BFB0EE66
:10BC9000680ABDEC028B10BD00000000F20000201D
:10BCA0003CDD012010B52DED028BB0EE408A9FEDFA
:10BCB0003B0AF0EE408A3A48007820B101281CD0B7
:10BCC000022864D160E000244FF49E6009F0A8FFD0
:10BCD00004024FF49F6009F0A3FF04434AF6AA2030
:10BCE000844203D002202E49087005E001202C492F
:10BCF0000870142008F0CEFD4AE0F6EE000AB0EE1F
:10BD0000600A00203CE0274901EB8001D1ED000AE8
:10BD1000F4EEC80AF1EE10FA30D82249421C01EBC9
:10BD20008201D1ED000AF4EEC80AF1EE10FA25DB2B
:10BD300000EE900AB8EE601AF8EE040A41EE000A2E
:10BD4000F0EE608A174901EB8201D1ED000A154936
:10BD500001EB800191ED001A70EEC10A114901EB6F
:10BD6000800191ED001A38EE411A61EE001A81EE61
:10BD7000A01A71EE280AF0EE608A03E0411CC8B2F6
:10BD80000A28C0DB00BF03E0F0EE488A00E000BFF5
:10BD900000BFB0EE680ABDEC028B10BD00000000D1
:10BDA0003AC001208CDC012010B52DED028BB0EEE5
:10BDB000408A9FED3B0AF0EE408A3A48007820B175
:10BDC00001281CD0022864D160E000244FF41660E2
:10BDD00009F026FF040240F6681009F021FF044331
:10BDE0004AF6AA20844203D002202E49087005E0BA
:10BDF00001202C490870172008F04CFD4AE0F0EEB5
:10BE0000080AB0EE600A00203CE0274901EB8001FF
:10BE1000D1ED000AF4EEC80AF1EE10FA30D822494A
:10BE2000421C01EB8201D1ED000AF4EEC80AF1EEEA
:10BE300010FA25DB00EE900AB8EE601ADFED180A62
:10BE400041EE000AF0EE608A174901EB8201D1ED64
:10BE5000000A154901EB800191ED001A70EEC10A4C
:10BE6000114901EB800191ED001A38EE411A61EEA3
:10BE7000001A81EEA01A71EE280AF0EE608A03E043
:10BE8000411CC8B20A28C0DB00BF03E0F0EE488ABC
:10BE900000E000BF00BFB0EE680ABDEC028B10BD31
:10BEA00000000000F100002010DD012010B52DED94
:10BEB000028BB0EE408A9FED3B0AF0EE408A3A4892
:10BEC000007820B101281CD0022864D160E0002451
:10BED0004FF4607009F0A4FE04024FF4627009F0A0
:10BEE0009FFE04434AF6AA20844203D002202E4932
:10BEF000087005E001202C490870132008F0CAFCE6
:10BF00004AE0F0EE080AB0EE600A00203CE0274963
:10BF100001EB8001D1ED000AF4EEC80AF1EE10FA4F
:10BF200030D8224A411C02EB8101D1ED000AF4EE27
:10BF3000C80AF1EE10FA25DB00EE900AB8EE601A9E
:10BF4000DFED180A41EE000AF0EE608A411C02EBB8
:10BF50008101D1ED000A114601EB800191ED001A3B
:10BF600070EEC10A114601EB800191ED001A38EE26
:10BF7000411A61EE001A81EEA01A71EE280AF0EE65
:10BF8000608A03E0411CC8B20A28C0DB00BF03E09E
:10BF9000F0EE488A00E000BF00BFB0EE680ABDECDA
:10BFA000028B10BD000000000400002060DC0120B6
:10BFB0007CB504460D46164628882189084400B2FF
:10BFC000ADF8000068886189084400B2ADF802004D
:10BFD000A8882189084400B2ADF80400E888618986
:10BFE000084400B2ADF8060032466946204663694F
:10BFF00098477CBD2DE9FF4F8FB00F46209DF87804
:10C0000000F0010008B1F94800E0F9480E90F87816
:10C0100000F0010008B1F74800E0F7480D90F8780B
:10C0200000F0010008B9F34800E0F3480C9001204B
:10C030000B90BEE000210B9100206988B5F804C088
:10C04000A1EB0C010AB200261AE006EB860CE968A7
:10C0500001EB8C01097C01F0010141B906EB860C72
:10C06000E96801EB8C018989014408B207E006EB1D
:10C07000860CE96801EB8C010989511A0AB2761C19
:10C080002969B142E1D800268EE006EB860CE9680A
:10C0900001EB8C01097C01F0010100297DD100BF79
:10C0A00018B900BF00BF00BFFEE700BF92FBF0F869
:10C0B0000FFA88F306EB8609D5F80C8008EB89089F
:10C0C000B8F80C8008FB03F80FFA88F106EB860934
:10C0D000D5F80C8008EB8908B8F9049006EB860ABD
:10C0E000D5F80C8008EB8A08B8F90680884501DD90
:10C0F000884607E006EB860AD5F80C8008EB8A082C
:10C10000B8F90680C14508DD06EB8609D5F80C8034
:10C1100008EB8908B8F9048013E006EB8609D5F826
:10C120000C8008EB8908B8F90680884501DD88464F
:10C1300007E006EB8609D5F80C8008EB8908B8F90A
:10C140000680C4468C450BD04FF0010806EB860AEA
:10C15000D5F80C9009EB8A09C9F81080CDF82C802D
:10C1600006EB8609D5F80C8008EB8908A8F808C00A
:10C1700006EB8609D5F80C8008EB8908B8F80C8026
:10C18000A0EB08080FFA88F006EB8609D5F80C80BA
:10C1900008EB8908B8F8088000E004E0A2EB080882
:10C1A0000FFA88F200BF761C2969B1423FF66DAFE5
:10C1B00000BF0B9800287FF43DAF00210F981BF0C3
:10C1C00019FA012800D100E000200A90002009900F
:10C1D000089008A809A9CDE9001029890BB2B5F982
:10C1E000022038781E9922F0A5FAF87800F00100B4
:10C1F00048B10A9838B10F981AF005FBBDF8241021
:10C20000084400B2099011990F981AF05CFA04469C
:10C210008FE17A4920461BF0B3FE40B1F878C0F3B5
:10C22000800111AA0F980BF04FFC044681E1002118
:10C2300020461BF063FA07900798002860D0002082
:10C240000390002610E006EB8601E86850F8210014
:10C25000A04208D106EB8600E96801EB8000B0F946
:10C260000800039003E0761C2869B042EBD800BFB9
:10C27000F87800F0010050B1608C20F4006000F507
:10C2800000606084608C20F48060608409E0608CD1
:10C2900020F4806000F580606084608C20F4006091
:10C2A000608404F114000D9988470399884226D0D0
:10C2B00020461CF07FF900BFA08AADF80400E08A98
:10C2C000ADF80600208BADF80800608BADF80A00D1
:10C2D00000BF04F114000E9A0399904701AA292186
:10C2E000204615F0E3FD20461AF054FB2246222199
:10C2F000009015F0DBFD20461CF05CF900BF07E064
:10C30000608C20F400606084608C20F48060608425
:10C31000002006907878012812D0022819D104F163
:10C3200014000C998847B5F90010491C21F001014F
:10C33000081A039000EBD070401000B2069009E09C
:10C3400004F114000C9988472988081A00B2069055
:10C3500000E000BF00BFF87800F0010050B10A987B
:10C3600040B104F114000D998847BDF82410081A53
:10C3700000B20990002003906B22204603991BF025
:10C3800087FB029002980FFA80F800BF002003900C
:10C390006C22204603991BF07BFB029002980FFA57
:10C3A00080F900BF20461BF0D7FD059020461AF00B
:10C3B000A1FA049008F4C040B0F5005F01D101205B
:10C3C00000E0002030B128F4C040B0F5FA6F01DC85
:10C3D000012000E00020E0B128F4C040B0F57A7FF1
:10C3E0000EDD28F4C040C0F57A700BE065CE010880
:10C3F00059CE0108C1CD0108CDCC010801000600CD
:10C4000028F4C04005994843642190FBF1F00FFAED
:10C4100080F809F4C040B0F5005F01D1012000E0D0
:10C42000002030B129F4C040B0F5FA6F01DC0120E2
:10C4300000E0002090B129F4C040B0F57A7F04DD1F
:10C4400029F4C040C0F57A7001E029F4C040049995
:10C450004843642190FBF1F00FFA80F9A18A1C98FF
:10C46000401A40440FFA80FAE18A1D98401A484465
:10C470000FFA80FBF87800F0010010B1BDF924003C
:10C4800000E0069850440FFA80FAF87800F00100B6
:10C4900008B1069801E0BDF9240058440FFA80FB6A
:10C4A000BAF1000F02D1BBF1000F1BD020461CF0E7
:10C4B00081F8A08A504400B2A082208B504401B27F
:10C4C0002183E08A584401B2E182608B584401B272
:10C4D000618320461CF06EF800235A4651462046E0
:10C4E0001CF016F9F87800F0010008B10A9870B94C
:10C4F00004F114000D9988471F990844BDF82010D5
:10C500000844BDF82410084400B2099008E0BDF8C2
:10C5100020101F980844BDF82410081A00B2099092
:10C52000F878C0F3800111AA0F980BF0CDFA0446F9
:10C5300000BF24B1DDE9111081427FF46AAE13B06F
:10C54000BDE8F08F2DE9F04F8DB005468946B9F171
:10C55000000F02D10DB0BDE8F08FA5F81890286843
:10C5600010B1286818F0FAFD09EB4901062202EB28
:10C57000410018F015FD286000BF286818B900BFF9
:10C5800000BF00BFFEE700BF28686860022128687E
:10C5900001FB0900801CE8600421286801FB0900F8
:10C5A000001DA860B9F1010F0CD1B42069680870B2
:10C5B0000020E96808800120E96848800020A96817
:10C5C0000880C7E709F10101C80018F033FD0746EC
:10C5D00009F1010007EB80084FF0000A4FEA8900DB
:10C5E00002B20BA90CA800F067F90024BDF93000D5
:10C5F0008010079000200390CCE0002616E00BA9E5
:10C600000CA800F061F90CA800F04BF900B90FE09C
:10C61000BDF93000801007A941F82600BDF83000B0
:10C6200000F0030003A941F82600761C042EE6DB87
:10C6300000BF042E00D0B3E00A990798884219D1B0
:10C64000079800B227F814000FFA8AF028F81400AF
:10C65000DDE903010844059908440699084469681E
:10C6600008556868005D0007000E69680855601C81
:10C6700004B28DE0DDE9070188422CD0079800B2B2
:10C6800027F814000FFA8AF028F814000398696854
:10C6900008556868005D0007000E69680855601C51
:10C6A00004B20798401E00B227F814000FFA8AF06F
:10C6B00028F814000498001D0599084406990844B8
:10C6C000696808556868005D0007000E69680855CC
:10C6D000601C04B25CE00999079888422CD0079846
:10C6E00000B227F814000FFA8AF028F81400DDE9E8
:10C6F00003010844696808556868005D0007000E7A
:10C7000069680855601C04B20798401E00B227F8FB
:10C7100014000FFA8AF028F81400059808300699DA
:10C720000844696808556868005D0007000E69687C
:10C730000855601C04B22BE0079800B227F81400DB
:10C740000FFA8AF028F81400DDE90301084405997E
:10C750000844696808556868005D0007000E69684C
:10C760000855601C04B20798401E00B227F8140058
:10C770000FFA8AF028F8140006980C3069680855FA
:10C780006868005D0007000E69680855601C04B207
:10C790000AF1010A0CA800F084F800287FF42DAFFC
:10C7A00000BF40F2D32109FB01F0029002988012F1
:10C7B0000190601E37F910100198814205D1601E6A
:10C7C00038F910100198814226D0DDE90121A1EB52
:10C7D0008220B0F5007F04DC00FB00F1480000146B
:10C7E00007E0C0F5806000FB00F148000014C0F1D4
:10C7F0000F00019909B227F81410019909B228F81D
:10C8000014106A6810556968095D0907090E6A689D
:10C810001155611C0CB200BFA61E0EE038F81600C0
:10C8200027F8140037F8160028F814006868805DAF
:10C8300069680855761E601C04B2002EEEDA4FF0CF
:10C84000000B00260020E968088023E0E96821F851
:10C850001B6037F81600A96821F81B0010E0A868D3
:10C8600030F81B0037F91610884203DAA86830F850
:10C870001B0001E037F91600A96821F81B00761C9F
:10C8800038F91600584501D1A642E8DB0BF101004A
:10C890000FFA80FBA642D9DB384618F047FC00BFF0
:10C8A00058E60146B1F90200B1F90020904201DCDE
:10C8B000012070470020FCE7028000234380C2F182
:10C8C00001031BB20B807047B1F90020002A07DC7E
:10C8D0000B8842885200D21C1A4412B20A800CE023
:10C8E00042880388D21A5200521D0B881A4412B291
:10C8F0000A800288521E12B202804288521C12B272
:10C900004280704710B500200AF006FE0D4991F8EC
:10C910002C10884215D00B48007801280BD10A480A
:10C92000007840B100200AF0F7FD064981F82C009C
:10C930000CF064FC05E0034890F82C10002025F072
:10C940006FF910BDCCE501205D00002010B501207D
:10C950000AF0E2FD184991F8FD1488422AD01748E0
:10C96000007808B301200AF0D7FD134981F8FD04CF
:10C97000084690F8FD0428B1012291031048F5F70C
:10C9800005F905E000224FF480410D48F5F7FEF867
:10C990000C48007802280DD107480078032809D1F7
:10C9A000192026F021FB05E0034890F8FD14012032
:10C9B00025F036F910BD0000E46701205D0000207D
:10C9C00000080240CCE5012000B503200AF0A4FDD8
:10C9D000114991F8001588421CD010480078A8B180
:10C9E0000D4890F8FF04012810D00B4890F800057E
:10C9F00060B903200AF090FD40B109480078022890
:10CA000004D10120044981F8000503E0002103203E
:10CA100025F006F900BD0000E46701205D0000205C
:10CA2000CCE5012000B502200AF076FD114991F80D
:10CA3000FF1488421CD010480078A8B10D4890F827
:10CA40000005012810D00B4890F8FF0460B90220BF
:10CA50000AF062FD40B109480078022804D10120A3
:10CA6000044981F8FF0403E00021022025F0D8F8F2
:10CA700000BD0000E46701205D000020CCE501203E
:10CA800010B504200AF048FD2B490978491E884258
:10CA900051D02948007820B1012807D0022844D17C
:10CAA0001EE00021042025F0BBF843E024F060FDE7
:10CAB0002249D1F8B8001DF0C0FC2049D1F8B800D7
:10CAC000012119F0D0F81D490869012118F0D5FDA0
:10CAD0000220194908700121042025F0A1F829E05D
:10CAE0001748007840B9012015490870134828F00C
:10CAF000EBFAC82001F033FB24F01CFC0F49086955
:10CB00001DF09BFC0D490869012119F0ACF80B4997
:10CB1000D1F8B800012118F0B0FD012006490870D5
:10CB20000021042025F07CF804E00121042025F0F8
:10CB300077F800BF00BF10BDCCE50120AC04002099
:10CB4000AD01002037B582B01546022D04DCBDF8DA
:10CB50000C10084605B030BDBDF80C00C00ABDF889
:10CB6000081000EBD1241F2C01D2204600E01F202A
:10CB7000BDF8081060F3CF210291BDF80C00C0F39E
:10CB80004510BDF80810C1F3451144183F2C01D2DF
:10CB9000204600E03F20BDF8081060F34A110291E2
:10CBA000BDF80C0000F01F00BDF8081001F01F01D7
:10CBB00044181F2C01D2204600E01F20BDF80810A9
:10CBC00060F304010291FF2D03D1BDF8081008465F
:10CBD000C0E72A46DDE9020111F078FA0190BDF8BC
:10CBE00004100846B6E717B581B01446022C04DCE1
:10CBF000BDF80810084604B010BDBDF80400C00A16
:10CC0000BDF80810C90A10FB01F04109BDF8040085
:10CC100061F3CF200190BDF8040000F01F00BDF8C3
:10CC2000081001F01F0110FB01F04109BDF80400DC
:10CC300061F304000190BDF80400C0F34510BDF895
:10CC40000810C1F3451110FB01F08109BDF8040083
:10CC500061F34A100190FF2C03D1BDF8041008467F
:10CC6000C9E72246DDE9010111F030FA0090BDF874
:10CC700000100846BFE737B582B01546022D04DC28
:10CC8000BDF80C10084605B030BDBDF80C00C00A58
:10CC9000BDF80810A0EBD124002C01DD204600E0F7
:10CCA0000020BDF8081060F3CF210291BDF80C0000
:10CCB000C0F34510BDF80810C1F34511441A002C0B
:10CCC00001DD204600E00020BDF8081060F34A11A5
:10CCD0000291BDF80C0000F01F00BDF8081001F033
:10CCE0001F01441A002C01DD204600E00020BDF8A1
:10CCF000081060F304010291FF2D03D1BDF8081064
:10CD00000846C0E72A46DDE9020111F0DFF901908B
:10CD1000BDF804100846B6E710B55849D1F8C4006C
:10CD200001211BF022F928B15449D1F8C400012196
:10CD300018F099FF5149D1F8C00001211BF015F9F5
:10CD400028B14E49D1F8C000012118F08CFF4B49A1
:10CD5000D1F8C80001211BF008F928B14749D1F8E2
:10CD6000C800012118F07FFF4449D1F8CC0001210F
:10CD70001BF0FBF828B14149D1F8CC00012118F093
:10CD800072FF3E49D1F8D00001211BF0EEF828B126
:10CD90003A49D1F8D000012118F065FF3749D1F8A0
:10CDA000D40001211BF0E1F828B13449D1F8D400B6
:10CDB000012118F058FF3149D1F8D80001211BF0AA
:10CDC000D4F828B12D49D1F8D800012118F04BFF33
:10CDD0002A49D1F8DC0001211BF0C7F828B1274906
:10CDE000D1F8DC00012118F03EFF2449D1F8E00021
:10CDF000012118F042FC2149D1F8E400012118F08A
:10CE00003CFC1E49D1F8E800012118F036FC1B4912
:10CE1000D1F8EC00012118F030FC1849D1F8C40019
:10CE2000174917F0F5FE1549D1F8C8001449143117
:10CE300017F0EEFE1149D1F8D0001149283117F052
:10CE4000E7FE0E49D1F8D8000D493C3117F0E0FE5D
:10CE5000002024F0B7FF012024F0B4FF022024F0CA
:10CE6000B1FF002007490870632007490870084691
:10CE700001780448007826F0DBFE10BDAC040020E9
:10CE800047E80120C8C40120C9C4012008B50346F1
:10CE900000930098484080EA620008BD70B50546DE
:10CEA0000C46002608480078012802D14FF64E763D
:10CEB00000E0064E3146284600F00AF86FF07F4148
:10CEC000204600F005F870BDBC010020FFEECA004E
:10CED00038B504460D46082C65D2DFE804F004108E
:10CEE0001C2834404C58284610F0E8FF2F49009089
:10CEF0000022D1F84C0100991CF02FFE54E0284686
:10CF000010F0DCFF294900900022D1F8440100997B
:10CF10001CF023FE48E0284610F0D0FF2349009083
:10CF20000022D1F83C0100991CF017FE3CE0284695
:10CF300010F0C4FF1D4900900022D1F8340100997F
:10CF40001CF00BFE30E0284610F0B8FF17490090A7
:10CF50000022D1F8480100991CF0FFFD24E028468A
:10CF600010F0ACFF114900900022D1F84001009967
:10CF70001CF0F3FD18E0284610F0A0FF0B490090CC
:10CF80000022D1F8380100991CF0E7FD0CE028469A
:10CF900010F094FF054900900022D1F82C0100996F
:10CFA0001CF0DBFD00E000BF00BF38BDAC0400207A
:10CFB0001FB55848007830B1012825D0042869D021
:10CFC00005287CD185E05448807800F00F00534953
:10CFD0000870084600780007000E087008460078C0
:10CFE0004D49C97801F00F0108444C4908700846C2
:10CFF00002784BA16846FAF70BFB4B49D1F84C017C
:10D00000694617F005FE82E04348007800F00F0003
:10D0100042494880084640884FF6FF7101EA0010F7
:10D020003E494880084640883B49497801F00F0155
:10D0300008443A494880084640884FF6FF7101EAA3
:10D04000001036494880084640883349897801F005
:10D050000F01084431494880084640884FF6FF7167
:10D0600001EA00102D494880084640882A49C978BD
:10D0700001F00F01084429494880084642882BA145
:10D080006846FAF7C5FA2849D1F84401694617F00D
:10D09000BFFD3CE020488078204948700846407831
:10D0A0000007000E4870084640781B49C9780844BC
:10D0B0001A4948700846427819A1684600E025E000
:10D0C000FAF7A6FA1849D1F84801694617F0A0FD09
:10D0D0001DE011484078642110FB01F00E49897869
:10D0E00001EB810100EB41000B49C97808440B4971
:10D0F0008880084682880FA16846FAF789FA0A49AB
:10D10000D1F84001694617F083FD00E000BF00BF81
:10D110001FBD0000BA010020C40100205C090020EE
:10D120003078253032780000AC040020307825308B
:10D13000347800002564000038B504460D4634B14B
:10D14000012C10D0022C1AD0032C30D123E0384807
:10D1500010F0B4FE374900900022D1F88001009908
:10D160001CF0FBFC24E0324810F0A8FE314900908E
:10D170000022D1F87C0100991CF0EFFC18E02C484B
:10D1800010F09CFE2B4900900022D1F87801009904
:10D190001CF0E3FC0CE0264810F090FE25490090BE
:10D1A0000022D1F8740100991CF0D7FC00E000BF08
:10D1B00000BF35B1012D11D0022D1CD0032D34D16B
:10D1C00026E06FF07F4010F079FE1A4900900022AF
:10D1D000D1F8800100991CF0C0FC27E06FF07F407F
:10D1E00010F06CFE134900900022D1F87C010099E8
:10D1F0001CF0B3FC1AE06FF07F4010F05FFE0D49A9
:10D2000000900022D1F8780100991CF0A6FC0DE0F6
:10D210006FF07F4010F052FE064900900022D1F8D6
:10D22000740100991CF099FC00E000BF00BF38BDFC
:10D23000FFEECA00AC0400207CB505460C46002079
:10D2400000900190102C05DA22461FA16846FAF7DB
:10D25000DFF911E0142C04D11CA00088ADF8000007
:10D260000AE0152C04D11AA00088ADF8000003E0F4
:10D2700018A00088ADF8000035B1012D0BD0022DAB
:10D2800010D0032D1CD114E01349D1F88001694658
:10D2900017F0BEFC15E01049D1F87C01694617F083
:10D2A000B7FC0EE00C49D1F87801694617F0B0FCE4
:10D2B00007E00949D1F87401694617F0A9FC00E0BC
:10D2C00000BF00BF7CBD00002578000030000000DA
:10D2D000780000002D000000AC04002010B56D485F
:10D2E000007830B1012830D0042866D0052874D1E8
:10D2F00090E014206849087015204870674800784D
:10D30000001188706548007800F00F00C870002494
:10D3100006E06148015D2046FFF78EFF601CC4B245
:10D32000042CF6DB03205E49087063205D49087019
:10D33000084601785A480078FFF7FEFE5A49D1F8AE
:10D340007001012118F08FFCA1E0544840880F21A2
:10D3500001EA203050490870504840880F2101EA06
:10D3600020204D4948704D4840880F2101EA201087
:10D37000494988704948807800F00F00C87000243F
:10D3800006E04548015D2046FFF756FF601CC4B229
:10D39000042CF6DB032042490870632041490870E1
:10D3A000084601783E480078FFF7C6FE3E49D1F8AE
:10D3B0007001012118F057FC69E01420364908700B
:10D3C00015204870354840780011887033484078FF
:10D3D00000F00F00C870002407E057E02E48015D00
:10D3E0002046FFF729FF601CC4B2042CF6DB0320A3
:10D3F0002B49087063202B4908700846017828489B
:10D400000078FFF799FE2849D1F87001012118F042
:10D410002AFC3CE0002020490870204880886421D4
:10D4200090FBF1F01C4948701C4880880A2190FB51
:10D43000F1F090FBF1F201FB1200174988701748D8
:10D4400080880A2190FBF1F201FB12001249C8709A
:10D45000002406E01048015D2046FFF7EDFE601C49
:10D46000C4B2042CF6DB03200D49087063200D497B
:10D470000870084601780A480078FFF75DFE0A49FF
:10D48000D1F87001012118F0EEFB00E000BF00BFF1
:10D4900010BD0000BA010020C40100205C0900207A
:10D4A000C2010020C3010020AC04002010B50246D8
:10D4B0000B461E200021124CA478641E04EB440489
:10D4C00003EB4404E1B232B1012A06D0022A09D0AA
:10D4D000032A11D10BE008460FE001F10F04E1B27D
:10D4E00008460AE001F11404E1B2084605E001F142
:10D4F0001904E1B2084600E000BF00BF10BD000003
:10D50000E467012010B58060C06000230361002142
:10D5100010E0002400F1140343F82140002206E04B
:10D5200000F13C0303EBC11343F82200521C202AF4
:10D53000F6DB491C0A29ECDB10BD2DE9FF4F87B053
:10D540000546DDE9178ADDF85890149F089CB9F16B
:10D55000040F02D0B9F1060F58D128460FF0D9FBBD
:10D5600083465946504618F04FF8B5F90200784303
:10D570004100B5F9000001EB4000044428460FF0DB
:10D5800003FC0590059840000490780000B20390D9
:10D59000CDF80880B5F902600DE02146049A0298A2
:10D5A00017F079FE039804440599029800EB4100B6
:10D5B0000290701C06B2B5F90600B042EDDAB9F17E
:10D5C000060F22D14FF47F414FF0000C01F47C4E46
:10D5D0004CEA5E1CC1F3C40E4CEA0E0CCDF800C040
:10D5E000BDF800E0F446CDF804C04246BDF8043072
:10D5F000002007E032F81010994202D100210AF809
:10D600000010401C5845F5D300BF88E0B9F1050F64
:10D6100041D1B5F90200784300EB4000B5F90010A4
:10D6200001EB41010844044428460FF0ADFB381AD1
:10D6300000B20590059800EB400000B20490284627
:10D640000FF036FB039028460FF09EFB8346002622
:10D650001DE00020069010E0A17806980AF800105E
:10D660002078617800EB012081B2069828F810102C
:10D67000E41C0698401C00B2069006985845EBDB67
:10D6800008EB4B08DA4404980444701C06B2039873
:10D690008642DEDB43E0B9F1140F40D1B5F9020058
:10D6A00078434100B5F9000001EB400004447800E4
:10D6B00000B2059028460FF0FBFA049028460FF0C0
:10D6C00063FB834600260BE04FEA4B0221464046AF
:10D6D00017F0E1FD08EB4B0805980444701C06B2F6
:10D6E00004988642F0DB089C099841000A9801FBE7
:10D6F0000044B5F90000B5F9021007FB010004442D
:10D70000002608E05A462146504617F0C4FDDA4488
:10D710003C44701C06B204988642F3DB00BF0BB099
:10D72000BDE8F08F30B502460B461146B1F928002E
:10D730000C8D04F4C044B4F5005F01D1012400E075
:10D74000002444B1B1F9284024F4C044B4F5FA6F80
:10D7500001DC012400E00024F4B191F83C4004F025
:10D760000304012C01D1002016E0B1F9284024F473
:10D77000C044B4F57A7F06DDB1F9284024F4C044F2
:10D78000C4F57A7403E0B1F9284024F4C0445C4342
:10D79000642594FBF5F420B230BD0146002000E082
:10D7A000401C31F9102041F6FF739A42F8D17047BE
:10D7B00010B504463B48007830B101281ED004283B
:10D7C00034D0052864D14BE03748007837490870D9
:10D7D00035480078022801D1012000E0002000EB4C
:10D7E000400031490978032901D1012100E00021DD
:10D7F000022202FB01002C4908704AE02A48007806
:10D800002A490870284800782044274908700846AB
:10D810000078C82802DD0320087006E0224800785E
:10D82000032802DD00202049087032E01E480078FD
:10D830001E4908701C480078022801D1012000E030
:10D84000002000EB400018490978032901D101218B
:10D8500000E00021022202FB01001349087018E0D9
:10D8600011480078114908700F48007820440E498B
:10D87000087008460078012802DA0320087006E0E4
:10D8800009480078032802DD01200749087000E0FC
:10D8900000BF00BF0548017803480078FFF74CFC43
:10D8A00010BD0000BA010020C2010020C301002009
:10D8B00010B5044634B900224FF480710448F4F7DF
:10D8C00065F904E0012211020148F4F75FF910BD87
:10D8D000000C024008B101B102B97047416082609A
:10D8E00000BFFAE770B52DED028B82B004460D46FD
:10D8F000604A61496148FFF7EDFF0026ECB394ED03
:10D90000000AF3EE090AB4EEE00AF1EE10FA04DDC3
:10D91000B3EE090A84ED000A0AE094ED000AB5EEC0
:10D92000C00AF1EE10FA03D29FED550A84ED000A09
:10D9300094ED000AB0EE408AB0EE480AFDF7A4FF6D
:10D94000B0EE408AB3EE090AB4EEC08AF1EE10FAE6
:10D9500004DDB3EE090AB0EE408A08E0B5EEC08AF5
:10D96000F1EE10FA03D29FED460AB0EE408A454828
:10D9700080ED048A9FED440A00E018E028EE000ADA
:10D98000B0EE408A9FED410A28EE000ADFED400A22
:10D9900080EE201ABCEEC10A10EE100A86B20023F7
:10D9A000012202213548009624F09EFB00BF85B37A
:10D9B00095ED000AF0EE040AB4EEE00AF1EE10FA7A
:10D9C00004DDB0EE040A85ED000A0CE095ED000AD6
:10D9D000F8EE040AB4EEE00AF1EE10FA03D2B8EE63
:10D9E000040A85ED000A95ED000AB0EE408AB0EE1B
:10D9F000480AFEF757F9B0EE408AB0EE040AB4EEDA
:10DA0000C08AF1EE10FA05DDB0EE040AB0EE408AED
:10DA10000BE02AE0B8EE040AB4EEC08AF1EE10FA88
:10DA200003D2B8EE040AB0EE408A164880ED048AAC
:10DA3000F6EE000AB7EE040A08EE200AB0EE408ABD
:10DA40009FED120A28EE000AF0EE040A80EE201A7A
:10DA5000BCEEC10A10EE100A86B200231A4601215C
:10DA60000648009624F040FB00BF02B0BDEC028BDC
:10DA700070BD0000B1D8000895DA0008C0DD0120B3
:10DA800000000000900000200000C84200FF7F4717
:10DA900000401C4570B504460D464FF47A732A4683
:10DAA00021460248F5F701FB70BD000030D501208A
:10DAB00010B52DED028B044614B9BDEC028B10BDE0
:10DAC00094ED000AF3EE0E0AB4EEE00AF1EE10FA5D
:10DAD00004DDB3EE0E0A84ED000A0AE094ED000ABC
:10DAE000B5EEC00AF1EE10FA03D29FED260A84EDDE
:10DAF000000A94ED000AB0EE408AB0EE480AFEF744
:10DB0000D5F9B0EE408AB3EE0E0AB4EEC08AF1EE5B
:10DB100010FA04DDB3EE0E0AB0EE408A08E0B5EE6E
:10DB2000C08AF1EE10FA03D29FED160AB0EE408AD9
:10DB3000154880ED048AB2EE040AC8EE000AB0EE81
:10DB4000608A9FED120A28EE000AF0EE080A80EEC5
:10DB5000201AB0EE418A9FED0D0AB4EEC08AF1EEB4
:10DB600010FA03DB9FED0A0AB0EE408ABCEEC80A49
:10DB700010EE103A002211460648F3F739FC00BFB8
:10DB80009BE700000000000090000020000080459E
:10DB900000F07F456CD4012037B582B005461446AD
:10DBA0002146039810F006F90190BDF804100846CC
:10DBB00005B030BD10B543480078082800D110BD2D
:10DBC00040480078082876D2DFE800F00412202EC2
:10DBD0003C4A5866122007F09FFAAA214FF40470BD
:10DBE00008F006F9AA214FF4067008F001F963E085
:10DBF000132007F091FAAA214FF4607008F0F8F8AA
:10DC0000AA214FF4627008F0F3F855E0142007F0F1
:10DC100083FAAA214FF49E6008F0EAF8AA214FF493
:10DC20009F6008F0E5F847E0152007F075FAAA2193
:10DC30004FF4CC6008F0DCF8AA214FF4CD6008F076
:10DC4000D7F839E0162007F067FAAA214FF4FC60F4
:10DC500008F0CEF8AA214FF4FD6008F0C9F82BE0D7
:10DC6000172007F059FAAA214FF4166008F0C0F8FF
:10DC7000AA2140F6681008F0BBF81DE0182007F054
:10DC80004BFAAA214FF42E6008F0B2F8AA2140F610
:10DC9000E82008F0ADF80FE0192007F03DFAAA21BE
:10DCA0004FF4466008F0A4F8AA2140F6684008F056
:10DCB0009FF801E0FFE700BF00BF0820014908709E
:10DCC00000BF7CE7A800002010B5414890F800058F
:10DCD000012877D10121032023F0A2FF3D480078DD
:10DCE000C0B901203B49087007F0DAFE002038492E
:10DCF00081F8FD0400224FF480413748F3F746FFD6
:10DD00000120334908720520887600210C200BF091
:10DD10002FFE5BE031480088401C00B22F4908808C
:10DD200006F050FA2D48B0F9000005284EDD2C48C9
:10DD3000807D00F00100002848D128490880022099
:10DD4000234981F80005002081F8FF040846007887
:10DD5000032825D008460178042025F0E7FF1C4859
:10DD60000179632025F064FF032019490870002021
:10DD700088710878042125F0D9FF0320144908711F
:10DD800048710879632125F053FF114991F8FE0489
:10DD900026F08AFC34F02CFA04201249087008E0BE
:10DDA00000200B4988711C2025F01EF91B2025F04E
:10DDB0001BF90C4800780BF0EBFD002005490870BA
:10DDC00004E0FFE70021032023F02AFF10BD00003C
:10DDD000E4670120D0C4012000080240D4C401201F
:10DDE000CC67012048C1012010B5364890F8FF04E7
:10DDF000012862D10121022023F012FF324800786D
:10DE000048B901203049087007F054F800210C206F
:10DE10000BF0AEFD55E02D480088401C00B22B49A8
:10DE2000088006F0CFF92948B0F90000052848DD40
:10DE30002748807D00F00100002842D12349088056
:10DE40002348407D20B902201E4981F8FF0403E0E9
:10DE500000201C4981F8FF041A48007803281ED0CE
:10DE600018480178042025F061FF164801796320E5
:10DE700025F0DEFE03201349087000208871087821
:10DE8000042125F053FF02200E49087148710879DA
:10DE9000632125F0CDFE04200E49087005E0002026
:10DEA000084988711B2025F09FF80A4800780BF07C
:10DEB0006FFD00200449087003E00021022023F0D8
:10DEC000AFFE10BDE4670120CFC40120D2C4012001
:10DED000CC67012048C101202DE9FF4F8DB00746D6
:10DEE0000D461646E87A022803DC012011B0BDE891
:10DEF000F08F28892A6901460C901098FAF7ACF93E
:10DF000004460CB90020F1E7217D01F01F0014F058
:10DF100077FE10B14FF0060818E0207D00F01F00DA
:10DF20000E2801D1804611E0207D00F01F0014284A
:10DF300001D180460AE0217D01F01F0014F043FE6C
:10DF400010B14FF0050801E04FF00408B8F10E0FD2
:10DF500009D1288818B96888B0F5807F03D04FF0C0
:10DF600005080020A061206A38B100BF00BF31461B
:10DF70003846226A32F0CEF8DEE0A069002859D097
:10DF800031460BA80EF042FE288818B96888B0F513
:10DF9000807F32D030460EF0DBFE834600BFF08833
:10DFA0007188401A401C00B20890281D6988CDE98C
:10DFB0000010B5F9003059460BA8089AFAF746F850
:10DFC000BDF82C003188084400B2ADF82C00BDF833
:10DFD0002E007188084400B2ADF82E00BDF8300064
:10DFE0003188084400B2ADF83000BDF832007188C5
:10DFF000084400B2ADF8320000BF0BAA09A8B96806
:10E00000F9F723FD8146B9F1000F04D1204601F054
:10E01000B8FA01206AE7D7F808A009A8B860CDF8D7
:10E020000080324629463846A36910F0EFFBC7F856
:10E0300008A081E032460BA8B968F9F706FD0A90FE
:10E040000A9820B9204601F09CFA01204EE70BA85F
:10E050000EF07EFE09900BA80EF07AFE00EB400059
:10E06000039016F0E7FF8146D7F808A00BA907A890
:10E070000EF0CCFD012107A80EF0EEFEBDF92C003C
:10E08000B6F90010401A0690BDF92E00B6F902103C
:10E09000A0EB010BBDF92E00059042E007AA514606
:10E0A00002A8F9F7D2FC0A900A9800B936E0CDF838
:10E0B0000090099803B20FFA8BF2069801B220463D
:10E0C00015F000FB0490049801280ED0204615F0AE
:10E0D00019FA00BF00BF484617F028F8204601F0A3
:10E0E00050FAC7F808A0002000E702A8B8604B4625
:10E0F00007AA29463846CDF8008010F087FBBDF806
:10E100001E00401C00B2ADF81E00BDF82200401CED
:10E1100000B2ADF822000BF1010B00BF0598401CC6
:10E120000590BDF9321005988142B7DAC7F808A00A
:10E13000484616F0FBFF00BF204601F022FA0120FE
:10E14000D4E600BF00BF7047002105E0002200E0D8
:10E15000521C6E2AFCDB491C8142F7DB704701E050
:10E16000411E88B20028FBDC70470CB500210191EC
:10E170000BE00021009102E00099491C00910099F8
:10E180000429F9DB0199491C019101998142F0D1DF
:10E190000CBD00002DE9F04780460C461546294885
:10E1A0000078002848D0B4F90400B4F90010401AEF
:10E1B000401CB4F90610B4F90220891A491C4843DE
:10E1C00021490860B4F9000020490860B4F9020050
:10E1D0001F490860B4F904001E490860B4F906003C
:10E1E0001D490860B4F906C0B4F90290ACEB090C03
:10E1F0000CF10103B4F904C0B4F90090ACEB090CC4
:10E200000CF10102B4F9021048460DF0D1FFB4F947
:10E2100002700CE0B4F9006004E0288834F0E4FCFB
:10E22000AD1C761CB4F90400B042F6DA7F1CB4F9D8
:10E230000600B842EEDA00BF404610F0EEF9BDE845
:10E24000F0870000A4C00120B8C00120A8C00120B0
:10E25000ACC00120B0C00120B4C0012010B50DF049
:10E26000F5FF10BD70B504460D4600222946204634
:10E2700005F04EFD01222946204605F049FD022207
:10E280002946204605F05EFB04222946204605F07B
:10E2900059FB70BD2DE9F74F9EB00C46E07802287F
:10E2A00002DC21B0BDE8F08F1CA820990EF0C9FC5B
:10E2B000B4F9200001282EDD94F82200FD282ADB85
:10E2C000208840B3BDF8700014F8231F4908C1F33B
:10E2D0008001084400B2ADF87000BDF872002178EA
:10E2E0004908C1F34001084400B2ADF87200BDF81E
:10E2F000740021784908C1F3C001401A00B2ADF89A
:10E300007400BDF8760014F82319C1F34001401AD7
:10E3100000B2ADF876001E981CA982681AA8F9F719
:10E3200094FB00B9BDE7E07B00F0070616B9A088B2
:10E33000199001E0E0881990BDF86410608981426D
:10E3400000D100261CA811F03BFA18901C2111A83E
:10E35000F1F7F0FFA0788DF85D00BDF86400ADF82E
:10E360004C00189860B9208850B94EB91CA811907B
:10E37000E0788DF85C0011A91E9812F0FEFB90E782
:10E38000E078FD2801DBFF2000E0E07810901CA879
:10E390000EF00FFD0F901CA80EF091FC0E90DDE921
:10E3A0000E01814201DA0F9800E00E980D90B4F949
:10E3B00000100D98B1EB600F02DAB4F9000001E033
:10E3C0000D98401007461AA80EF0F3FC81464FF056
:10E3D000FF300C9000200B90002F01DC189870B1DA
:10E3E000484616F027FE0B9000233AB21CA905A858
:10E3F00011F05EFD002105A810F0E4FE0C90BDF8C0
:10E400006800ADF80C00BDF86C00ADF810000B987A
:10E41000149003A811901690FF208DF85C00A01DA9
:10E42000DDE90E2114F0C0F98046B8F1000F0CD0E0
:10E43000022E0AD1BDF96810D8F8080000EB41009F
:10E44000BDF97010A0EB4100129001A811F0B8F9CD
:10E4500000901898A0B3BDF96A502CE028B2ADF82E
:10E460000E0028B2ADF812004A4610990B9817F02A
:10E470005AF8BDF968100FFA89F32AB20B9811F017
:10E480004FF98DF854009DF85400012802D1022064
:10E490008DF85400012E09D1BDF97210691AD8F80F
:10E4A000080000EB41000088ADF84C0011A91E984F
:10E4B00012F063FB6D1CBDF96E00A842CEDAC8E015
:10E4C000FFE700255CE0BDF8720028440FFA80FAEF
:10E4D000BDF87600401B0FFA80FBBDF96A0050457D
:10E4E00004DDBDF96E00584500DA48E04A4610994F
:10E4F0000B9817F018F8BDF90C100FFA89F3524673
:10E500000B9811F00DF98DF854009DF85400012876
:10E5100002D102208DF85400BDF96A00504514DC88
:10E52000ADF80EA0ADF812A0012E0AD1BDF97210FF
:10E53000AAEB0101D8F8080000EB41000088ADF813
:10E540004C0011A91E9812F018FBBDF96E00584539
:10E5500014DBADF80EB0ADF812B0012E0AD1BDF942
:10E560007210ABEB0101D8F8080000EB4100008805
:10E57000ADF84C0011A91E9812F0FFFA00BF6D1CF7
:10E58000BD42A0DBBDF87000ADF80400BDF874001A
:10E59000ADF80800BDF87200384400B2ADF80600CE
:10E5A000BDF87600C01B00B2ADF80A000098B0B903
:10E5B000AEB9BDF87200384400B2ADF80E00BDF837
:10E5C0007600C01B00B2ADF8120010988DF85C0008
:10E5D0000020149011A91E9812F0CFFA38E010987C
:10E5E0008DF85C0001208DF85400BDF97600A0EB99
:10E5F000070ABDF97200C51927E0009870B14A46B4
:10E6000010990B9816F08FFFBDF968100FFA89F377
:10E610002AB20B9811F084F88DF8540028B2ADF8A6
:10E620000E0028B2ADF81200012E09D1BDF972100A
:10E63000691AD8F8080000EB41000088ADF84C00DA
:10E6400011A91E9812F099FA6D1C5545D5DD00BF31
:10E6500000BF0B9810B10B9816F068FD0C98401C89
:10E6600028B10C9811F00CFD05A811F085F8B8F14F
:10E67000000F02D0404614F08EF800BF11E62DE9DD
:10E68000F04F91B006460C461546206910B911B0FE
:10E69000BDE8F08FA07E022800DCF8E729460FA82D
:10E6A000B268F9F7D2F900B9F1E7D6F808800FA8F7
:10E6B000B060206915F07BFB0746022F55D1002082
:10E6C00041F6FF71CDE90001029003460EA8D4E99E
:10E6D00004121DF063FE28460EF06BFB824600EB31
:10E6E000DA70298801EB6000BDF9389009EBD97127
:10E6F000A0EB610000B2ADF83000BDF83000BDF80D
:10E7000038100844401E00B2ADF8340028460EF020
:10E71000D6FA824600EBDA70698801EB6000BDF939
:10E720003A9009EBD971A0EB610000B2ADF832006C
:10E73000BDF83200BDF83A100844401E00B2ADF8F2
:10E74000360004A810F04EFC60690490208BADF8F0
:10E750001C00A07E8DF82A00002000900CAA04A9BD
:10E760003046236910F086F8B0E00EA9206914F055
:10E77000F5FE8146B9F1010F7DD108A810F05DF8D2
:10E78000A0788DF82C00208BADF82800E07E8DF865
:10E790002A00A07E8DF82B00207FE8BB28460EF0D3
:10E7A00008FB834600EBDB70298801EB60000E99C3
:10E7B000C1F38A2A0AEBDA71A0EB610000B2ADF86E
:10E7C000180028460EF07BFA834600EBDB70698860
:10E7D00001EB60000E994FEA515A0AEBDA71A0EB97
:10E7E000610000B2ADF81A00BDF818000E99C1F32F
:10E7F0008A210844401E00B2ADF81C00BDF81A0082
:10E800000E9900EB5150401E00B2ADF81E0006AA52
:10E8100008A93046236900E002E00FF0BDFF51E097
:10E820006888ADF81A00BDF81A000E9900EB515037
:10E83000401E00B2ADF81E003DE02888ADF818007B
:10E84000BDF818000E99C1F38A210844401E00B299
:10E85000ADF81C0019E006AA08A9304623690FF09C
:10E860009BFFBDF818000E99C1F38A21084400B23D
:10E87000ADF8180000E026E0BDF81C000E99C1F3C9
:10E880008A21084400B2ADF81C00BDF91800B5F9A2
:10E8900004108842DFDDBDF81A000E9900EB5150DC
:10E8A00000B2ADF81A00BDF81E000E9900EB5150F1
:10E8B00000B2ADF81E00BDF91A00B5F90610884285
:10E8C000BBDD00BF01E000BF00BF00BFC6F808808D
:10E8D00000BFDCE62DE9F04F87B083460C461646B4
:10E8E00094F82200022802DC07B0BDE8F08F208CEB
:10E8F00000B9F9E794F82300C0F3440000B9F3E746
:10E9000094F8230000F0010000B1EDE730460EF06E
:10E9100050FA814630460EF0D2F90746B4F900505D
:10E92000B94501DA484600E038468246B5EB6A0F41
:10E9300001DD4FEA6A05314605A80EF082F9BDF9FE
:10E94000141094F82300400800F0040010B1B4F94A
:10E95000200003E0B4F9200028444042084400B2FB
:10E96000ADF81400BDF9181094F82300400800F029
:10E97000080010B1B4F9200003E0B4F920002844E5
:10E980004042081A00B2ADF81800BDF9161094F80C
:10E990002300400800F0020010B1B4F9200003E0A9
:10E9A000B4F9200028444042084400B2ADF81600F3
:10E9B000BDF91A1094F82300C0F3400010B1B4F967
:10E9C000200003E0B4F9200028444042081A00B2B5
:10E9D000ADF81A00208C281A0FFA80F8B8F1000F51
:10E9E00001DA4FF00008A07894F82210CDE9021067
:10E9F000E08BADF804002BB205AA31465846CDF89D
:10EA0000008000F002F800BF6EE72DE9FF4FA3B0D1
:10EA10000D4616461F463298FF2801DBFF2000E016
:10EA200032983290284610F0CBFE2290229868B996
:10EA300067B9309850B93298009032462946319BD8
:10EA4000239800F0A9FA27B0BDE8F08F2398294653
:10EA5000826820A8F8F7F9FF00B9F4E720A80EF0C3
:10EA6000A8F981461C2119A816F097FD484616F012
:10EA7000E1FA1C904FF0FF301890002F0ADD0023C0
:10EA80003A46294612A811F013FA002112A810F0F4
:10EA900099FB1890012331460CA8309A11F008FA1E
:10EAA00000210CA810F08EFB0B9009A819901E9065
:10EAB000BDF8C400ADF86C0032988DF87C00339836
:10EAC0008DF87D00B5F900003844B6F90010884291
:10EAD00003DDB5F90000384401E0B6F9000000B2EA
:10EAE000ADF81C00B5F90400C01BB6F9041088424B
:10EAF00003DAB5F90400C01B01E0B6F9040000B266
:10EB0000ADF82000B5F902003844B6F90210884289
:10EB100003DDB5F90200384401E0B6F9020000B2A5
:10EB2000ADF81E00B5F90600C01BB6F90610884204
:10EB300003DAB5F90600C01B01E0B6F9060000B221
:10EB4000ADF8220007A80EF034F90690B5F90200DE
:10EB5000B6F90210884201DC012000E00020824664
:10EB6000B5F90600B6F90610884201DB012000E085
:10EB700000208346229800284CD0BDF88000ADF8D4
:10EB80002400BDF88400ADF82800BDF9824029E0DA
:10EB9000BAF1000F04D1BDF91E00A04200DD20E053
:10EBA000BBF1000F04D1BDF92200A04200DA1DE044
:10EBB00020B2ADF8260020B2ADF82A0049461C98D4
:10EBC00016F022FDBDF980100FFA89F322B21C98CD
:10EBD00010F0A6FD8DF8740019A9239811F0CDFF4F
:10EBE00000BF641CBDF98600A042D1DA00BF0CA8AA
:10EBF00010F0C2FD0B9811F043FA1898401C28B190
:10EC000012A810F0B9FD189811F03AFA1C9816F0F5
:10EC10008DFA18E7B5F90000B6F90010884201DC5A
:10EC2000012000E000200590B5F90400B6F90410B9
:10EC3000884201DB012000E00020049001200390C5
:10EC4000059860B1049850B1BAF1000F07D0BBF13C
:10EC5000000F04D00698322801DA0020039001202A
:10EC60008DF87400BAF1000F15D0039898B1BDF873
:10EC70001C00ADF82400BDF82000ADF8280068881D
:10EC8000ADF826007088401E00B2ADF82A0019A920
:10EC9000239811F072FFBBF1000F15D0039898B1C3
:10ECA000BDF81C00ADF82400BDF82000ADF8280028
:10ECB000F088401C00B2ADF82600E888ADF82A00C4
:10ECC00019A9239811F059FF059898B12888ADF833
:10ECD00024003088401E00B2ADF82800BDF81E00A8
:10ECE000ADF82600BDF82200ADF82A0019A9239836
:10ECF00011F043FF049898B1B088401C00B2ADF801
:10ED00002400A888ADF82800BDF81E00ADF8260044
:10ED1000BDF82200ADF82A0019A9239811F02DFFA3
:10ED20000398F0BBBDF88000ADF82400BDF8840066
:10ED3000ADF82800B6F90200B5F90210401AB84241
:10ED400001DA384604E0B6F90200B5F90210401ABB
:10ED500000B20290002442E06888204400B2019092
:10ED6000E888001B00B20090BDF982100198814232
:10ED700005DDBDF986100098814200DA2EE0494693
:10ED80001C9816F041FCBDF924100FFA89F3019A82
:10ED90001C9810F0C5FC8DF87400BDF98210019824
:10EDA00000E020E0814209DC0198ADF826000198DE
:10EDB000ADF82A0019A9239811F0DFFEBDF98610DD
:10EDC0000098814209DB0098ADF826000098ADF864
:10EDD0002A0019A9239811F0D0FE00BF641C0298E4
:10EDE0008442B9DBC7E0BDF88000ADF82400BDF96E
:10EDF0008410BDF91C00401E814202DABDF9840076
:10EE000002E0BDF91C00401E00B2ADF8280009A8C0
:10EE10000DF0CFFF8046B8F1000F48DD059810B91E
:10EE2000BAF1000F1ED0BDF9824017E020B2ADF854
:10EE3000260020B2ADF82A0041461C9816F0E4FBEB
:10EE4000BDF92410434622B21C9810F069FC8DF8DD
:10EE5000740019A9239811F090FE641CBDF91E00DE
:10EE6000A042E3DC059810B9BBF1000F1FD0BDF93B
:10EE70002200441C17E020B2ADF8260020B2ADF805
:10EE80002A0041461C9816F0BFFBBDF924104346EA
:10EE900022B21C9810F044FC8DF8740019A9239834
:10EEA00011F06BFE641CBDF98600A042E3DABDF9E7
:10EEB0008010BDF92000401C814202DDBDF98000B8
:10EEC00002E0BDF92000401C00B2ADF82400BDF8FE
:10EED0008400ADF8280009A80DF06BFF8046B8F15A
:10EEE000000F48DD049810B9BAF1000F1ED0BDF92B
:10EEF000824017E020B2ADF8260020B2ADF82A001B
:10EF000041461C9816F080FBBDF92410434622B2FE
:10EF10001C9810F005FC8DF8740019A9239811F0C5
:10EF20002CFE641CBDF91E00A042E3DC049810B95D
:10EF3000BBF1000F1FD0BDF92200441C17E020B226
:10EF4000ADF8260020B2ADF82A0041461C9816F014
:10EF50005BFBBDF92410434622B21C9810F0E0FB85
:10EF60008DF8740019A9239811F007FE641CBDF9EF
:10EF70008600A042E3DA0CA810F0FEFB0B9811F01B
:10EF80007FF812A810F0F8FB189811F079F81C9887
:10EF900016F0CCF800BF56E52DE9FF4F89B080464A
:10EFA0000C461546DDF858901C21684616F0F5FA17
:10EFB00007A80090BDF83000ADF808008DF8189053
:10EFC000B4F90200B5F90210884201DC012000E02A
:10EFD00000200646B4F90600B5F90610884201DBA8
:10EFE000012000E000200746B4F90000B5F9001048
:10EFF000884201DC012000E000208246B4F90400D0
:10F00000B5F90410884201DB012000E000208346AE
:10F010002088ADF81C00A088ADF820006088ADF80D
:10F020001E006888401E00B2ADF822001EB169467D
:10F03000404611F0A2FDE888401C00B2ADF81E0069
:10F04000E088ADF822001FB16946404611F095FDF9
:10F050002088ADF81C002888401E00B2ADF82000C2
:10F0600016B1B5F9020001E0B4F90200ADF81E00D6
:10F0700017B1B5F9060001E0B4F90600ADF82200B9
:10F08000BAF1000F03D06946404611F076FDA8881A
:10F09000401C00B2ADF81C00A088ADF82000BBF108
:10F0A000000F03D06946404611F067FD0DB0BDE882
:10F0B000F08F00002DE9F04105463F4800680FF051
:10F0C000C7FA04462868C66B706B10B13046716B86
:10F0D0008847394800680068008837490968096826
:10F0E000498810FB01F0E168884201D1012000E06D
:10F0F00000200746206898B1606888B187B90CE0A5
:10F100002D4800680068806A38B12B4A1268106880
:10F11000294A12681268916A884720690028EFD14D
:10F1200001202061244800680068C068806900F000
:10F13000010050B1204800680068C0688069C0F3D1
:10F14000400010B10120606101E000206061606951
:10F1500008B1012000E0002080462868406998B18D
:10F160002868007CC0F3011048B12868007CC0F317
:10F17000800020B1D6E9001000F020F804E0D6E9C4
:10F1800000212868FCF714FF206890B1606880B106
:10F190002868007C00F0010010B1B8F1000F08D021
:10F1A0002168A068884202D16068A06001E0206800
:10F1B000A060BDE8F0810000DCC001202DE9F34F24
:10F1C00083B004468848006805688748006800687E
:10F1D000007CC0F3400040B1287CC0F3800020B127
:10F1E00000BF00BF05B0BDE8F08F287CC0F3011060
:10F1F00002280AD121462846049A00F004F9214643
:10F200002846049AFCF7D4FEEBE0287CC0F30110FA
:10F21000012804D0287CC0F301100328F4D1002079
:10F220000290714800680FF013FA824620460DF0F4
:10F2300088FD064620460DF026FD83464FF4A0507B
:10F24000B0FBF6F000B2584505DA4FF4A050B0FB21
:10F25000F6F000B200E058460190B4F90280287C34
:10F26000C0F3011001280BD168882188401A401E84
:10F2700000B2E080E088801B401C00B2608006E0A5
:10F280002088608060883044401E00B2E080002703
:10F290009EE0ABEB07010198814201DD019801E09E
:10F2A000ABEB07000FFA80F90120CAF8100047BB4A
:10F2B000B34526DBB146297CC1F30111032901D1F5
:10F2C000012100E0002108463146049A00F00FF9C0
:10F2D000287CC0F30110012807D1A4F8008008EBB6
:10F2E0000600401E00B2A0803FE02888401EA0EB30
:10F2F000080000B2A080A088801B401C00B22080C3
:10F3000033E0029820B94FF4205015F093FE02909C
:10F3100002980090297CC1F30111032901D1012138
:10F3200000E0002108464A463146049B00F0B2F84E
:10F33000287CC0F3011001280AD108EB070000B2B5
:10F34000208008EB07004844401E00B2A0800CE07B
:10F350002888401EA0EB0800C01B00B2A080A08837
:10F36000A0EB0900401C00B2208007EB09005845C3
:10F370000DDBDAF8180000F0010040B1DAF81800EF
:10F38000C0F3400018B10120CAF8140002E00020C8
:10F39000CAF81400029808B9049800E002980246DE
:10F3A00021462846FCF704FE04E0A86A10B128466E
:10F3B000A96A8847DAF810000028F6D106FB09F19F
:10F3C000049800EB4100049007EB090007B200BF6E
:10F3D0005F45FFF65EAF029810B1029815F0A6FEE9
:10F3E00000BF00BFFEE60000DCC0012018B50488A5
:10F3F00000940C88048014880C801C881480BDF84C
:10F4000000401C8018BD2DE9FC5F05460C461646E1
:10F4100020460DF096FC824620460DF034FC8346D3
:10F420001AFB0BF001900198471E4FF0000811E005
:10F4300006EB47000088009006EB470006EB48010A
:10F440000988018006EB4800BDF8001001807F1E8E
:10F4500008F101084745EBD8B4F90690688861883F
:10F46000401A401E00B2E0806888A0EB0900401EF0
:10F4700000B26080B4F9049028882188401A401EA8
:10F4800000B2A0802888A0EB0900401E00B22080B6
:10F49000BDE8FC9F2DE9F04704461D46089F01FB8F
:10F4A00002F0A0F1010C481E00FB02F800231AE054
:10F4B00008EB03000CB1ACEB000000260FE0A946FE
:10F4C000AD1C07EB400AB9F80090AAF800900CB107
:10F4D000104400E0801A06F101090FFA89F68E4205
:10F4E000EDDB581C03B29342E2DBBDE8F0872DE967
:10F4F000F04782460C46154600263BE0002731E0E7
:10F50000601E801B0FFA80F8601EC01B0FFA80F986
:10F51000BAF1000F12D007FB048C05EB4C0308FB7B
:10F52000049C05EB4C0209FB046C05EB4C0106FB4B
:10F53000047C05EB4C00FFF759FF11E009FB046C5C
:10F5400005EB4C0308FB049C05EB4C0207FB048C09
:10F5500005EB4C0106FB047C05EB4C00FFF746FF76
:10F56000781C07B2601C00EBD071B7EB610FC7DBF2
:10F57000701C06B204EBD471B6EB610FBEDBBDE8C4
:10F58000F08710B50446204613F0BCFF10BD000004
:10F590002DE9F04FBDB005460E4600BF00BFAB469B
:10F5A0000BF13000F9F704F810B13DB0BDE8F08F71
:10F5B00005F114023BA8B168F8F747FA00B9F4E77F
:10F5C000B0683A903BA8B06035A80FF0CEFD35AAE0
:10F5D0004FF4E021284618F0B7FD27A810F07EFD73
:10F5E0009DF8DC008DF89F0047F6FF70ADF89C0099
:10F5F0004FF4E021284618F076FB074600EBD77061
:10F600004FEA60094FF4E021284618F06CFB0746EA
:10F6100000EBD7704FEA600A314604A816F008FEE6
:10F6200024A80A9016A808904FF4E02011906F4883
:10F630000590052006900BF13000F8F731FF0446E5
:10F64000CCE00A2235A924A815F025FE382227A9E6
:10F6500016A815F020FEE088ADF89000E088ADF81F
:10F660005C0039A80D9038A80E90607B00F0010076
:10F6700020B1B4F90070B4F9028012E0B4F90400CA
:10F6800047F6FF71884200D1A2E0A08882B26B46A3
:10F690002846A1680DF0F6FFBDF90070BDF90280A3
:10F6A00000BFA88A384407B2E88A40440FFA80F8BD
:10F6B000B9F1000F04D0BAF1000F01D0012000E031
:10F6C000002001900198B0B1A7EB090000B2ADF89D
:10F6D000080007EB090000B2ADF80C00A8EB0A0027
:10F6E00000B2ADF80A0008EB0A0000B2ADF80E0057
:10F6F00002A8079001E000200790207B00F00300A3
:10F7000080B3207B00F0010010B1B5F9140000E0D7
:10F710003846ADF8E400ADF8E680207B00F002004A
:10F7200010B1B5F9180000E03846ADF8E000BDF8BA
:10F73000E600ADF8E20004AA1A21284612F0B6FB52
:10F7400038AB39AA24A930460FF0F8FC019820B153
:10F7500002AA16A9304610F0A5FC04AA1B212846CF
:10F7600012F0A4FB207B00F00C0080B3ADF8E47035
:10F77000207B00F0040010B1B5F9160000E040460F
:10F78000ADF8E600BDF8E400ADF8E000207B00F045
:10F79000080010B1B5F91A0000E04046ADF8E200EB
:10F7A00004AA1A21284612F081FB38AB39AA24A9F1
:10F7B00030460FF0C3FC019820B102AA16A93046CA
:10F7C00010F070FC04AA1B21284612F06FFB00BF4A
:10F7D00021460BF13000F8F75DFE0446002C7FF463
:10F7E00030AF3A98B06000BFDFE60000204A04085E
:10F7F0002DE9F04FA5B004460F46254604F114014B
:10F8000023A8BA68F8F721F92290229810B925B0F8
:10F81000BDE8F08FB868219023A8B8600021204689
:10F8200017F050FF1E900021204618F0A1F8014665
:10F830001E98084400B21D900021204618F010F9CF
:10F8400001461E98084400B21C90204616F0DBFFCB
:10F850007E35E9884843001200B21B90204616F01E
:10F86000B3FF29894843001200B21A9017A80FF07D
:10F870007CFC17AA0021204618F066FC394605A832
:10F8800016F0D6FC002012908C48069000200790BD
:10F8900017A80B904FF0FF30139000200E900F90A0
:10F8A00005AA1A21204612F001FB00200190312206
:10F8B0002046019918F0ECF80090009800F0FF0B3A
:10F8C00000BF0021204617F0FDFE049000200190AB
:10F8D00033222046019918F0DBF80090009800F0E0
:10F8E000FF0800BF204617F0D7F80390204617F016
:10F8F000CDF9029035F87E09002865D0E18A1C9880
:10F9000001440298081A00B20190A08AADF8800064
:10F91000208BADF87C004FF00009B5F87E000FFA9F
:10F9200080FABBF1020F1ADD0498002817DD08F0F9
:10F93000020040B10021204618F092F818B909F1F0
:10F9400001000FFA80F908F0010040B100212046C3
:10F9500017F0BAFF18B9AAF101000FFA80FA4E4663
:10F960002FE01A987043B5F87E10491E90FBF1F015
:10F9700000B2ADF88200BDF882100198084400B2D0
:10F98000ADF88200BDF88200ADF87E004B480690CD
:10F990000120079020A80E901FA80F90139605AA8B
:10F9A0001A21204612F082FA1FAB20AA17A9384666
:10F9B0000FF0C4FB05AA1B21204612F077FA701C39
:10F9C00006B25645CDDB00BFB5F88000002865D0F3
:10F9D000A18A1D9801440398081A00B20190E08A98
:10F9E000ADF88200608BADF87E004FF00009B5F8ED
:10F9F00080000FFA80FABBF1020F1ADD049800288C
:10FA000017DD08F0040040B10021204617F0B0FFD8
:10FA100018B909F101000FFA80F908F0080040B1A7
:10FA20000021204617F0D4FF18B9AAF101000FFAFF
:10FA300080FA4E462FE01B987043B5F88010491E9F
:10FA400090FBF1F000B2ADF88000BDF88010019895
:10FA5000084400B2ADF88000BDF88000ADF87C002D
:10FA6000164806900220079020A80E901FA80F901D
:10FA7000139605AA1A21204612F018FA1FAB20AAE5
:10FA800017A938460FF05AFB05AA1B21204612F091
:10FA90000DFA701C06B25645CDDB00BF4FF0FF30AB
:10FAA000139000200E900F9005AA1B21204612F003
:10FAB000FDF92198B86000BFA9E60000204A0408BB
:10FAC0002DE9F14F9AB01A9812F08BF907461A985F
:10FAD00012F0E8F905462C46122F7DD11A9812F043
:10FAE000DEF906463078022802D11BB0BDE8F08F5F
:10FAF00094F8380000F00300032805D094F838008B
:10FB000000F00300022802D101203070EDE794F8E4
:10FB10003800C0F38400042808D094F83800C0F3FB
:10FB20008400012802D001203070DEE74FF0000889
:10FB300046224146284617F0ABFF19901998C0B2EB
:10FB4000FF2802D001203070CFE7208E10B10120B5
:10FB50003070CAE71A9812F0A2F98146E08EB0F52B
:10FB6000807F09D1002205F114014846F7F7AEFF66
:10FB700098BB01203070B8E7284616F0BBFE8046DF
:10FB8000284618F0E9F9824604F13200E18E00239C
:10FB90004246CDE90010514618A8F8F757FABDF8CB
:10FBA0006000A98A084400B2ADF86000BDF8621098
:10FBB000E88A084400B2ADF86200BDF86400A98A82
:10FBC000084400B2ADF86400BDF86610E88A084445
:10FBD00000B2ADF8660001E00BE009E0002218A9D0
:10FBE0004846F7F773FF10B9012030707DE700BF7A
:10FBF00010E2152F01D0182FFAD1284618F0ACF9D1
:10FC00001990284616F076FE1890002632223146CA
:10FC1000284617F03DFF1090109800B2804600BFB4
:10FC200012223146284617F033FF109010984044B6
:10FC30000FFA80F900BF13223146284617F028FF3B
:10FC400010901098404400B2179000BF1022314627
:10FC5000284617F01DFF1090109840440FFA80FAC4
:10FC600000BF11223146284617F012FF109010985D
:10FC7000404400B21690608E484400B2ADF8540083
:10FC8000A08E504400B2ADF8560094F8390000F050
:10FC90000300012804D113A9284616F0D3FD26E05D
:10FCA00015A9E08ECDE90001208E03B213A8DDE98D
:10FCB0001821F8F7CBF9BDF84C00A98A084400B226
:10FCC000ADF84C00BDF84E10E88A084400B2ADF81B
:10FCD0004E00BDF85000A98A084400B2ADF85000AB
:10FCE000BDF85210E88A084400B2ADF8520005F1A0
:10FCF000140111A80CF0B7FF13A905F114000CF0C2
:10FD0000B2FFC5481A9916F0B9FC8346BBF1010F42
:10FD100000D0EAE611A905F114000CF0A4FF152F9C
:10FD20007DD1E08D08B1A08D00B9DEE6E08E00B98E
:10FD3000DBE61A9812F05DF8064605F114010FA8EB
:10FD40000CF091FF284613F01FFE0E9094F8390036
:10FD500000F0030001283CD1B4F92C10BDF9382083
:10FD6000891A481C00EBD071BDF83C20A2EB610160
:10FD700009B2ADF83C10B4F92C10BDF93820891A3D
:10FD8000481C00EBD071BDF84020A2EB610109B224
:10FD9000ADF84010B4F92E10BDF93A20891A481C6C
:10FDA00000EBD071BDF83E20A2EB610109B2ADF8C5
:10FDB0003E10B4F92E10BDF93A20891A481C00EB08
:10FDC000D071BDF84220A2EB610109B2ADF842103A
:10FDD00013E013A80DF009F8BDF83C100844401ECC
:10FDE00000B2ADF8400013A80CF085FFBDF83E103E
:10FDF0000844401E00B2ADF84200BDF83C00484443
:10FE000000B2ADF83C00BDF83E00504400B2ADF881
:10FE10003E00BDF840101798081A00B200E0F8E064
:10FE2000ADF84000BDF842101698081A00B2ADF8BF
:10FE3000420094F8380000F00300012805D094F83F
:10FE4000380000F0030000287ED108A80EF0F5FC71
:10FE500008AA0021284618F0A7F8E08EADF8220085
:10FE6000208E00B2ADF82000608EADF82400A18E87
:10FE7000ADF8261094F83800C0098DF83400BDF8AC
:10FE80004C00484400B2ADF81800BDF84E00504494
:10FE900000B2ADF81A00BDF850101798081A00B259
:10FEA000ADF81C00BDF852101698081A00B2ADF853
:10FEB0001E00B068059006AA06A8B168F7F7C5FD50
:10FEC00000B912E606A8B060B4F92800B4F92C1005
:10FED00090FBF1F201FB12000290B4F92A00B4F990
:10FEE0002E1090FBF1F201FB12000190BDF83E10C4
:10FEF0000198084400B2ADF80E00BDF90E00BDF93E
:10FF00003E10884206DDBDF80E00E18D401A00B2B9
:10FF1000ADF80E00BDF80E00E18D0844401E00B2A1
:10FF2000ADF812004AE0BDF83C100298084400B257
:10FF3000ADF80C00BDF90C00BDF93C10884208DD9D
:10FF4000BDF80C00A18D00E041E0401A00B2ADF810
:10FF50000C00BDF80C00A18D0844401E00B2ADF8A5
:10FF6000100015E003AA08A93046636A0EF014FCDD
:10FF7000BDF80C00BDF83810084400B2ADF80C0014
:10FF8000BDF81000BDF83810084400B2ADF81000FC
:10FF9000BDF90C00BDF940108842E3DBBDF80E004E
:10FFA000BDF83A10084400B2ADF80E00BDF81200DA
:10FFB000BDF83A10084400B2ADF81200BDF90E00C9
:10FFC000BDF942108842AEDB0598B06020E094F89D
:10FFD000380000F00300022811D106A80FF002F843
:10FFE00006AA0021284618F047F80020009005F1E5
:10FFF000140206A93046636A0EF03CFC08E000BF1C
:020000040801F1
:1000000000BF002305F11402194630460EF0C4FB70
:1000100000BF00BF00BF68E5648204082DE9F14F0E
:10002000DCB05C9811F03EFF05462C465C9811F060
:10003000E0FE5B9059A9284616F004FC0020CDE9AB
:1000400010506922DDE9100117F022FD0F900F9882
:1000500000B258900020CDE910506A22DDE910016D
:1000600017F016FD0F900F9800B25790BDF864116D
:100070005898081A00B2ADF86401BDF86811589894
:10008000084400B2ADF86801BDF866115798081A27
:1000900000B2ADF86601BDF86A115798084400B285
:1000A000ADF86A0159A80CF099FE834659A80CF0E6
:1000B0001BFE5690D4E90A10A0EB0109569883451F
:1000C00001DB012000E0002080460020559094F8DC
:1000D0005C0000F0030001280BD1A06A002808DAB8
:1000E000E06A002805DDA16A206B884201D1012069
:1000F00055900021284617F047FC549000212846CF
:1001000017F072FC53900021284617F0B5FC52906E
:100110000021284617F0E4FB519059A904F134005E
:100120000CF098FDA18E5498084400B2A086218F4F
:100130005398081A01B22187E18E5298084401B2FF
:10014000E186618F5198081A01B26187B8F1000FFA
:1001500013D004F134000CF0C7FD04280DDA5698D2
:1001600000EBD0714A10E98A1144891E0AB2E28676
:10017000E08E001D01B2618715E0B8F1000F12D1C9
:1001800004F134000CF02AFE04280CDA58460BEB7C
:10019000D071AA8A02EB6101891E09B2A186A08EE4
:1001A000001D01B2218704F134000CF017FE5090BD
:1001B00004F134000CF098FD4F90B8F1000F01D01D
:1001C000509800E04F988246B8F1000F05D004F136
:1001D0003406371DFE484C9004E004F13606371D06
:1001E000FC484C90A06D401CF8B1A36A216DC91A5F
:1001F00001FB0AF191FBF9F108B2A36A616DC91A1A
:1002000001FB0AF191FBF9F10AB2131AD4F858C0B4
:1002100003FB0CF1CB1701EB13631B121BB24D93C5
:100220004D99014409B24D9108E0A16A206B401A32
:1002300000FB0AF090FBF9F000B24D90A06C401C5E
:10024000E0B1A36A216CC91A01FB0AF191FBF9F133
:1002500008B2A36A616CC91A01FB0AF191FBF9F1BA
:100260000AB2131AD4F848C003FB0CF1CB1701EB08
:10027000136300EB23231BB24E9308E0D4E909017A
:10028000401A00FB0AF090FBF9F000B24E900020FB
:10029000119016222846119917F0FAFB1090109829
:1002A000C0B24B90B8F1000F0ED04B9801280BD183
:1002B00030463E4607464E99494209B24E914D9905
:1002C000494209B24D9100BFB8F1000F0AD0318800
:1002D0004E98084400B2388031884D98084400B2E6
:1002E00030800AE039884E98081A401C00B23080ED
:1002F00039884D98081A00B23880559878B3A26AA8
:10030000524202FB0AF292FBF9F211B2B8F1000F6D
:100310000CD032880A4410B2B7F90020824201DDC5
:1003200030801BE03A883280388017E03A88521AD1
:10033000521C10B2B6F90020824201DD388002E082
:1003400032883A803080B7F90020B6F900309A42FE
:1003500004DAB6F900003A883280388000BF559838
:1003600000BB04F134004C99884701281ADC684628
:100370005B9915F05DFF4FF400300D9096480190A9
:100380000020029004F1340003906A461A212846A6
:1003900011F08CFD6A461B21284611F087FD5DB0E7
:1003A000BDE8F08F04F1340149A80CF053FC3BA8E0
:1003B0000FF094FE3BAA4FF40031284617F042FF9D
:1003C00029A85B9915F034FF4FF40030369082482D
:1003D0002A9000202B903BA82D9004F134002C9003
:1003E00029AA1A21284611F061FD002011900B2244
:1003F0002846119917F04CFB1090109800B22890E5
:100400005698834501DA584600E056982790DDE972
:100410002701B1EB600F02DD279840102890BDF94D
:10042000EC0026904F995098884201DA509800E0ED
:100430004F982790DDE92601B0EB610F02DD279888
:1004400040102690B8F1000F08D004F134000CF0F1
:10045000C5FC01462698B1EB400F0BDCB8F1000F4C
:1004600028D104F134000CF03FFC01462698B1EB92
:10047000400F1FDD9DF8EF0011909DF806011090D0
:100480009DF80E010F9000208DF8EF008DF8060109
:100490008DF80E0104F134023BA95B980FF002FEC7
:1004A00011988DF8EF0010988DF806010F988DF8CF
:1004B0000E0100BFA98A5498084400B2ADF8780034
:1004C000298B5398081A00B2ADF87C00E98A52983B
:1004D000084400B2ADF87A00698B5198081A00B24E
:1004E000ADF87E0000231EA920A8289A0FF0E0FC9A
:1004F000002120A80EF066FE1D909DF822011C90A0
:100500009DF80E011B9000208DF80E018DF8220140
:1005100059A919A80CF09EFBBDF864105498084422
:1005200000B2ADF86400BDF866105298084400B2FD
:10053000ADF86600BDF868105398081A00B2ADF81F
:100540006800BDF86A105198081A00B2ADF86A0048
:10055000B8F1000F15D019A80CF0C6FB042810DA6A
:10056000569800EBD0714A10E98A1144891E09B2ED
:10057000ADF86610BDF86600001D00B2ADF86A0067
:1005800017E0B8F1000F14D119A80CF027FC0428CB
:100590000FDA58460BEBD071AA8A02EB6101891E73
:1005A00009B2ADF86410BDF86400001D00B2ADF8EA
:1005B0006800BDF9EC20002304F1340113A80FF00A
:1005C00077FC002113A80EF0FDFD129019AA05E09A
:1005D000DDCD0108E9CC0108488204083BA95B98FD
:1005E0000FF060FD1B988DF80E011C988DF822010C
:1005F00000208DF8EF008DF806018DF8220104F13E
:1006000034023BA95B980FF04DFD13A80FF0B4F82E
:1006100020A80FF0B1F812980FF032FD1D980FF0DE
:100620002FFD29AA1B21284611F040FC00BFB6E689
:100630002DE9FF4FA1B0064614462498807B00F0B8
:100640000F052298807E1F90032D00D10425012DD7
:1006500006D0022D0BD0042D10D0082D1DD114E092
:10066000DFF86C834FF0800A02201E901AE0DFF85A
:1006700064834FF0C00A04201E9013E0DFF8588313
:100680004FF0F00A10201E900CE0DFF850834FF07E
:10069000FF0A4FF480701E9004E000BF00BF25B039
:1006A000BDE8F08F00BF1F98FD2823DACC48017801
:1006B0001F98814203D1CB480068A84213D0002084
:1006C0000DE018F80010FF2901D11F9904E018F877
:1006D00000101F9A51430912C34A1154401C1E991D
:1006E0008842EED300BFDFF80083BD491F98087031
:1006F000BC4805602498B0F806B0249800891B9087
:100700000BFB05F01A90B4F90000B168B1F90010C4
:10071000884201DB002005E0B068B0F90000B4F9C0
:100720000010401A1990B4F900005844B168B1F9AA
:100730000410884201DC584606E0B068B0F90400B5
:10074000B4F90010401A401C1890B4F90200B168C6
:10075000B1F90210884201DB002005E0B068B0F971
:100760000200B4F90210401A1790B4F902101B9855
:100770000844B168B1F90610884201DC1B9806E014
:10078000B068B0F90600B4F90210401A401C169087
:100790001A9917984843199901FB050015902E994D
:1007A000159801EBD0002E90159800F007071C213A
:1007B0000DA814F0F2FE22988089ADF83C00229832
:1007C000807E8DF84C002298807FC0F3C2008DF8A7
:1007D0004D00F8F7F5F901900DF03EFF0C901B98D5
:1007E0000BFB00F10C98814201DD0C9802E01B9993
:1007F0000BFB01F00B900B9814F01CFC8146CDF81C
:10080000409000200A9021881998084400B2ADF861
:100810002000218818980844401E00B2ADF824003A
:1008200061881798084400B2ADF82200BDF8220094
:10083000ADF8260000BFBDF82400BDF82010401A16
:10084000401C00B2079000BFBDF82000ADF81400B6
:10085000BDF82200ADF81600BDF82400ADF8180070
:10086000BDF82600ADF81A0000BFBDF816101698A6
:10087000084400B2ADF81A0005A80EF0A1FF0490DC
:1008800008A80D901290C5F10800039019980BEB81
:1008900000011898081A6843029017981C9078E095
:1008A0000A9801902AFA07F0209019981D9028E0E4
:1008B0002E980078209908400399C91BC8401490CD
:1008C000149830B1149818F800100A9809F800101C
:1008D00003E000210A9809F800100398874204D227
:1008E0002F442098E840209005E00027CDF880A014
:1008F0002E98401C2E900A98401C0A901D98401C6F
:100900001D9018991D988842D2DB0498A0B1BDF9BA
:100910002620BDF92010019B09EB0300079B0EF078
:10092000FFFE8DF844009DF8440028B9019909EBB9
:100930000100079914F031FEDDE91801411A0A9807
:1009400001440B98814206D2BDF82600401C00B23B
:10095000ADF8260012E002208DF844000DA93046C3
:1009600010F00BF9BDF82600401C00B2ADF82200D3
:10097000BDF82200ADF8260000200A900298074436
:100980002E9800EBD7002E9007F007071C98401C0C
:100990001C9016991C98884282DBBDF92200BDF993
:1009A000261088420ED0BDF82600401E00B2ADF8D9
:1009B000260002208DF844000DA9304610F0DDF825
:1009C00000200A90484614F0B1FB00BF67E6000023
:1009D000A4480408A6480408B2480408C248040809
:1009E0003401002038010020CCDD01202DE9FF4F2B
:1009F0008FB00C4615461E46B4F90200401E0E90FC
:100A00000E9840100D900E9800F001010D980844CA
:100A10000C90B5F90000B6F90010884202DAB5F979
:100A2000000001E0B6F90000ADF82800B5F90000BB
:100A3000B6F90010884202DDB5F9000001E0B6F910
:100A40000000401E00B2ADF82C0069880C98081A0E
:100A500000B2ADF82A0069880D98084400B2ADF8DC
:100A60002E000F980AA982680AA8F6F7EEFF8246C0
:100A7000BAF1000F02D113B0BDE8F08FE08818B1D1
:100A8000A08808B1012000E00020834601200990E1
:100A90000AA80EF095FE10B10020099004E0BBF109
:100AA000000F01D0002009901C2102A814F075FD50
:100AB0000AA802902088ADF81000207A8DF8200056
:100AC000099820B102A90F9810F057F878E00AA809
:100AD0000CF068F90746BDF92E000190BDF82A0018
:100AE000ADF82E0000200090BBF1000F0BD0B4F940
:100AF0000600B4F904100844BDF9281091FBF0F287
:100B000000FB12100090384614F094FA8046CDF89D
:100B100014800AA80790BDF92A904AE03946404659
:100B200014F072FDBDF928103BB20FFA89F240466D
:100B30000EF0F6FD8DF81800BBF1000F27D09DF8E0
:100B4000180020B3009800211BE0B4F90420824271
:100B500007DBA3881B1A1AB28B1819B2831818B2B4
:100B60000BE0B4F90620B4F904301A44824201DCE7
:100B7000002002E0002208F801204A1C11B2421CA9
:100B800010B2B942E1DB02228DF8182000BF02A9A1
:100B90000F980FF0F2FFBDF82A00401C00B2ADF82C
:100BA0002A00BDF82E00401C00B2ADF82E0009F15D
:100BB000010901988145B1DD404614F0B7FA00BF44
:100BC00000BF58E72DE9FF4FC7B08B4691469A46C4
:100BD000B9F90200BAF90210884210DAB9F8020035
:100BE000ADF81A01BAF80200ADF81601B9F8000024
:100BF000ADF81801BAF80000ADF814010FE0BAF82A
:100C00000200ADF81A01B9F80200ADF81601BAF801
:100C10000000ADF81801B9F80000ADF81401BDF9F5
:100C20001401BDF91811441ABDF91601BDF91A11C4
:100C3000451A002C01DD204600E06042002D01DD58
:100C4000294600E06942884201DD012000E00020E1
:100C50004490BBF9026000204390449870B1002D8D
:100C600001DD284600E068424101002C01DD2046FC
:100C700000E0604291FBF0F043900DE0002C01DDBC
:100C8000204600E060424101002D01DD284600E0E1
:100C9000684291FBF0F04390E0494398085C704350
:100CA0003F30C611771006F0010000EB0708BDF9D0
:100CB0001801BDF91411884202DABDF9180101E0EA
:100CC000BDF91401801B00B2ADF80401BDF9180193
:100CD000BDF91411884202DDBDF9180101E0BDF92A
:100CE0001401304400B2ADF80801BDF91A01BDF994
:100CF0001611884202DABDF91A0101E0BDF91601A8
:100D0000801B00B2ADF80601BDF91A01BDF916113C
:100D1000884202DDBDF91A0101E0BDF91601304437
:100D200000B2ADF80A01479841A9826841A8F6F7D8
:100D30008CFE4090409810B94BB0BDE8F08F4498BD
:100D4000F0B3002C24DD0021BDF81601C01B00B259
:100D5000CDE90001BDF91431BDF81A01C01B02B282
:100D6000BDF9181135A80EF025FE0121BDF81601B8
:100D7000404400B2CDE90001BDF91431BDF81A01BB
:100D8000404402B2BDF918112AA80EF013FE4AE041
:100D90000021BDF81601404400B2CDE90001BDF9C3
:100DA0001431BDF81A01404402B2BDF9181135A83A
:100DB0000EF000FE0121BDF81601C01B00B200E0DC
:100DC0000DE0CDE90001BDF91431BDF81A01C01BD9
:100DD00002B2BDF918112AA80EF0ECFD23E00021A3
:100DE000BDF91601CDE90001BDF81401404403B27C
:100DF000BDF91A21BDF81801404401B235A80EF022
:100E0000D9FD0121BDF91601CDE90001BDF814019C
:100E1000C01B03B2BDF91A21BDF81801C01B01B2F5
:100E20002AA80EF0C7FD002135A80EF0CBF91390CB
:100E300000212AA80EF0C6F912904FF0FF30119051
:100E400010909BF80900C0F3001068BB0321BDF8A7
:100E50001A01204400B2CDE90001BDF81801401B81
:100E600003B2BDF91A21BDF918111FA80EF0A2FD99
:100E70000221BDF81601204400B2CDE90001BDF801
:100E80001401401B03B2BDF91621BDF9141114A8B9
:100E90000EF090FD00211FA80EF094F91190002192
:100EA00014A80EF08FF9109041A80BF07BFF0F9063
:100EB000F7F786FE01900DF0CFFB0D9041A80BF0E7
:100EC00028FF01460D98814203D241A80BF021FF73
:100ED00000E00D980C900C9814F0ACF80B90BDF954
:100EE0000A010A90BDF80601ADF80A010020099038
:100EF000DDE90B0114F088FB1C2102A814F04DFB66
:100F000041A80290BBF80000ADF810009BF8080063
:100F10008DF820000B98059041A80790BDF90601B7
:100F20000E9040E0BDF90411099B0B9AD0180F9A5E
:100F300013B20E9A12B20EF0F3FB8DF818009DF862
:100F4000180028B9099A0B9988180F9914F025FBF5
:100F50000F990998084409900F99099801440C9831
:100F6000814206D2BDF80A01401C00B2ADF80A0168
:100F700016E002208DF8180002A947980FF0FDFD39
:100F8000BDF80A01401C00B2ADF80601BDF806012B
:100F9000ADF80A0100200990DDE90B0114F034FBE3
:100FA0000E98401C0E900A990E988842BADDBDF941
:100FB0000601BDF90A1188420CD0BDF80A01401E95
:100FC00000B2ADF80A0102208DF8180002A9479876
:100FD0000FF0D3FD0B9814F0A9F835A80EF0CCFB58
:100FE0002AA80EF0C9FB1198401C10B11FA80EF0E2
:100FF000C3FB1098401C10B114A80EF0BDFB139851
:101000000FF03EF812980FF03BF811980FF038F8F7
:1010100010980FF035F800BF8EE60000C2490408B2
:101020002DE9FF4F91B00C4615461E46B4F902005B
:10103000401E1090109840100F90109800F0010181
:101040000F9808440E9029880E98081A00B2ADF83F
:10105000300029880F98084400B2ADF83400B5F983
:101060000200B6F90210884202DAB5F9020001E086
:10107000B6F90200ADF83200B5F90200B6F9021077
:10108000884202DDB5F9020001E0B6F90200401E17
:1010900000B2ADF8360011980CA982680CA8F6F7DA
:1010A000D4FC8146B9F1000F02D115B0BDE8F08F34
:1010B000E08818B1A08808B1012000E00020824635
:1010C00001200B900CA80EF07BFB10B100200B90C0
:1010D00004E0BAF1000F01D000200B901C2104A8FD
:1010E00014F05BFA0CA804902088ADF81800207A60
:1010F0008DF828000B9820B104A911980FF03DFD40
:1011000066E00CA80BF04EFE8346BDF93600039056
:10111000BDF83200ADF83600584613F08BFF029050
:10112000029807900CA8099000200190BAF1000FD6
:101130000BD0B4F90600B4F904100844BDF932101C
:1011400091FBF0F200FB12100190019FBDF932807B
:1011500037E05946029814F057FABDF930100FFAEB
:101160008BF30FFA88F202980EF0DAFA8DF820006D
:10117000BAF1000F13D09DF8200070B1B4F904004B
:10118000B84202DA00208DF82000B4F90600B4F964
:1011900004100844B84200DC0027781C07B204A9F8
:1011A00011980FF0EAFCBDF83200401C00B2ADF817
:1011B0003200BDF83600401C00B2ADF8360008F130
:1011C000010803988045C4DD029813F0AFFF00BF0B
:1011D00000BF6AE770B50446204610F063FE05467E
:1011E000204610F006FE0646314628460EF0B4FFB3
:1011F00070BD2DE9F14F90B0109810F053FE0546E8
:101200002C46109810F0F5FD06460EA9284615F05C
:10121000A5FA002794F84800C0F3001008B147F081
:10122000010794F84800C0F3401008B147F00207E6
:101230000021284616F06FFD42F2D171884205D197
:10124000688CC0F3C02008B947F0040706A80DF069
:10125000C9FEB4F84400ADF82E004620005BADF89E
:1012600030008DF8357006AA0021284616F004FFDC
:101270000DA8411E626A03780BB90123037000BFF9
:10128000284613F023F90790284613F019F908901F
:101290004FF6FF710798884223D00898884220D0E3
:1012A0004FF4802B55225946284616F0F1FB024692
:1012B000594601902846F7F722FA029002980390C7
:1012C000BDF80C00ADF8260000BF20225946284684
:1012D00016F0DEFB029002980390BDF80C00ADF80A
:1012E000280094F8480000F00700022805D094F880
:1012F000480000F0070003281FD19DF834000228A1
:1013000003D09DF83400032817D141F6FF71BDF9D1
:101310002A008DE88300BDF92C30069A03A8616A83
:101320001BF03CF80EA80BF067FDBDF90C108842CD
:1013300002DA01208DF8340000BF04F1300894F87F
:10134000480000F00700032805D00EA80BF0DAFCD7
:10135000B0F5806F01DA4FF000080EA904A8B2685A
:10136000F6F773FB8146B9F1000F02D111B0BDE869
:10137000F08F94F8480000F0070070B9284615F087
:1013800085FC8346CBF1000002B200210EA80BF0D1
:101390004BFD688BADF83E0000BF94F8480000F0AC
:1013A0000700022805D094F8480000F00700032841
:1013B0000ED1D6F808B004A8B060CDF800800EAA0F
:1013C00006A93046636A0DF055FAC6F808B007E082
:1013D000CDF800800EAA06A93046636A0DF04AFADD
:1013E000D6F808A004A8B06094F8480000F0070000
:1013F00003284FD141F6FF71BDF92A008DE8830023
:10140000BDF92C30069A03A8616A1AF0C7FF0EA82E
:101410000BF0F2FCBDF90C1088421BDA20221146B9
:10142000069810F0C7FE00EB4000B4F84410BDF879
:101430000C201144084400B2ADF82E004620005B99
:10144000ADF83000CDF800800EAA06A93046636AD8
:101450000DF010FA0EA80BF055FCBDF90E108842E5
:1014600017DAB4F84400ADF82E00069810F0BBFE71
:101470004621095BBDF80E201144084400B2ADF8C6
:101480003000CDF800800EAA06A93046636A0DF040
:10149000F1F900BFC6F808A000BF67E72DE9F74FD4
:1014A0008AB00C46904694F82A00022802DC0DB05F
:1014B000BDE8F08FE08C00B9F9E794F82A90B9F113
:1014C000FD0F01DD4FF0FF09414608A80BF0B9FB05
:1014D000208D401E05B2BDF82000401B00B2ADF8C3
:1014E0002000BDF82200401B00B2ADF82200BDF87C
:1014F0002400284400B2ADF82400BDF8260028449A
:1015000000B2ADF8260008A906A80BF09AFBBDF8BA
:101510001800E18C401A00B2ADF81800BDF81C00AC
:10152000E18C084400B2ADF81C00BDF81A00E18C53
:10153000401A00B2ADF81A00BDF81E00E18C084454
:1015400000B2ADF81E0008A80BF033FC824608A8D4
:101550000BF0B5FB0746B4F90060BA4501DA504616
:1015600000E038468346B6EB6B0F01DD4FEA6B06B1
:10157000E08C304400B20590A07894F82A10CDE9B0
:101580000210A08CADF8040030B2009008AA06A9A1
:10159000059B0A98FDF739FA00BF88E77CB5044639
:1015A000A06985686089002856D1A089002853D198
:1015B000E088218988424FDAE18808B21AF000FEFB
:1015C000B4F90410B4F90E20891A484321684988F7
:1015D00001EBE03000B2ADF80200E1885A3108B208
:1015E0001AF0EEFDA18810FB01F02168098801EBDB
:1015F000E03000B2ADF80400218908B21AF0E0FD35
:10160000A18810FB01F02168498801EBE03000B2AD
:10161000ADF8060021895A3108B21AF0D1FDB4F9AB
:101620000410B4F90E20891A48432168098801EB97
:10163000E03000B2ADF800002A4669466846F6F789
:1016400004FA06463EB1A169C1F808D0D4E90412F3
:10165000A0690EF027FDC2E0608910B1A0890028C2
:101660007BD16089D0BB20680088ADF8000020687D
:101670004088A188084400B2ADF80600E18808B2AD
:101680001AF09EFDB4F90410B4F90E20891A4843EB
:101690002168498801EBE03000B2ADF80200E18832
:1016A0005A3108B21AF08CFDA18810FB01F02168B4
:1016B000098801EBE03000B2ADF804002A46694623
:1016C0006846F6F7C2F906463EB1A169C1F808D0EE
:1016D000D4E90412A0690EF0E5FC00BFA08900283F
:1016E0007DD120680088A188084400B2ADF80400CC
:1016F00020684088ADF80200218908B21AF060FD28
:10170000A18810FB01F02168498801EBE03000B2AC
:10171000ADF8060021895A3108B21AF051FDB4F92A
:101720000410B4F90E20891A48432168098801EB96
:10173000E03000B2ADF800002A4669466846F6F788
:1017400084F906463EB1A169C1F808D0D4E9041273
:10175000A0690EF0A7FC42E0FFE76089A1898842FA
:1017600005D1608918B12089E188884211DB608940
:10177000022802D1A08901280BD06089032802D158
:10178000A089022805D06089032828D1A0890128D2
:1017900025D120680088ADF8000020684088ADF8A9
:1017A000020020680088A188084400B2ADF8040057
:1017B00020684088A188084400B2ADF806002A4697
:1017C00069466846F6F741F906463EB1A169C1F897
:1017D00008D0D4E90412A0690EF064FC00BFA0692F
:1017E00085607CBD7CB50446A06985686089012858
:1017F00056D1A089012853D1E088218988424FDA47
:10180000E18808B21AF0DCFCA18810FB01F0216825
:10181000498801EBE03000B2ADF80600E1885A31AA
:1018200008B21AF0CDFCB4F90410B4F90E20891AEC
:1018300048432168098801EBE03000B2ADF80400AC
:10184000218908B21AF0BCFCB4F90410B4F90E20D6
:10185000891A48432168498801EBE03000B2ADF8AD
:10186000020021895A3108B21AF0AAFCA18810FBA3
:1018700001F02168098801EBE03000B2ADF800000A
:101880002A4669466846F6F7E0F806463EB1A16981
:10189000C1F808D0D4E90412A0690EF003FCC7E037
:1018A0006089012802D0A08901287ED160890128A1
:1018B0003AD120680088A188401A00B2ADF8000033
:1018C00020684088ADF80200E18808B21AF078FC80
:1018D000A18810FB01F02168498801EBE03000B2DB
:1018E000ADF80600E1885A3108B21AF069FCB4F983
:1018F0000410B4F90E20891A48432168098801EBC5
:10190000E03000B2ADF804002A4669466846F6F7B2
:101910009CF806463EB1A169C1F808D0D4E904128A
:10192000A0690EF0BFFB00BFA0890128B7D12068D5
:101930000088401E00B2ADF8040020684088A188ED
:10194000084400B2ADF80600218908B21AF038FC4C
:10195000B4F90410B4F90E20891A48432168498863
:1019600001EBE03000B2ADF8020021895A3108B233
:101970001AF026FCA18810FB01F02168098801EB10
:10198000E03000B2ADF800002A4669466846F6F736
:101990005CF806463EB1A169C1F808D0D4E904124A
:1019A000A0690EF07FFB43E0FFE76089A1898842D0
:1019B00006D16089012803D02089E18888420FDBA5
:1019C000608910B9A08902280AD0608910B9A0895D
:1019D000032805D0608903282AD1A089022827D1AD
:1019E00020680088A188401A00B2ADF80000206885
:1019F0004088ADF8020020680088401E00B2ADF8B3
:101A0000040020684088A188084400B2ADF80600B0
:101A10002A4669466846F6F718F806463EB1A169B7
:101A2000C1F808D0D4E90412A0690EF03BFB00BF56
:101A3000A06985607CBD7CB50446A0698568608925
:101A4000022856D1A089022853D1E08821898842F2
:101A50004FDAE1885A3108B21AF0B2FBA18810FBC4
:101A600001F02168098801EBE03000B2ADF8000018
:101A7000E18808B21AF0A4FBB4F90410B4F90E20FE
:101A8000891A48432168498801EBE03000B2ADF87B
:101A90000600218908B21AF093FBA18810FB01F01F
:101AA0002168498801EBE03000B2ADF802002189DD
:101AB0005A3108B21AF084FBB4F90410B4F90E20BC
:101AC000891A48432168098801EBE03000B2ADF87B
:101AD00004002A4669466846F5F7B7FF06463EB158
:101AE000A169C1F808D0D4E90412A0690EF0DAFAAD
:101AF000CCE06089022802D0A08902287DD16089CB
:101B000002283CD120680088401E00B2ADF80400D5
:101B100020684088A188401A00B2ADF80200E18830
:101B20005A3108B21AF04CFBA18810FB01F0216871
:101B3000098801EBE03000B2ADF80000E18808B29E
:101B40001AF03EFBB4F90410B4F90E20891A484388
:101B50002168498801EBE03000B2ADF806002A4662
:101B600069466846F5F771FF06463EB1A169C1F8BE
:101B700008D0D4E90412A0690EF094FA00BFA0893D
:101B80000228B5D120680088A188401A00B2ADF8BB
:101B9000000020684088401E00B2ADF80600218990
:101BA0005A3108B21AF00CFBB4F90410B4F90E2043
:101BB000891A48432168098801EBE03000B2ADF88A
:101BC0000400218908B21AF0FBFAA18810FB01F089
:101BD0002168498801EBE03000B2ADF802002A46E6
:101BE00069466846F5F731FF06464EB1A169C1F86E
:101BF00008D0D4E90412A06900E002E00EF052FA25
